:100000000040002065800000A5800000A78000005F
:1000100000000000000000000000000000000000E0
:10002000000000000000000000000000A9800000A7
:100030000000000000000000AB800000AD80000068
:10004000AF800000055B000011840000AF8000005D
:10005000AF80000000000000AF800000AF80000013
:1000600095390000E5870000AF800000AF800000F8
:10007000AF800000AF800000AF800000AF800000C4
:10008000AF80000095840000AF800000AF800000CA
:10009000AF800000AF800000AF800000AF800000A4
:1000A000AF800000AF8000000000000000000000F2
:1000B0000000000000000000000000000000000040
:1000C00010B5064C2378002B07D1054B002B02D02E
:1000D000044800E000BF0123237010BD700200201F
:1000E00000000000B4F50000044B10B5002B03D055
:1000F0000349044800E000BF10BDC04600000000F6
:1001000074020020B4F50000164B002B00D1144BF4
:100110009D46402292029A1A924600218B460F4633
:100120001348144A121A0CF091F90F4B002B00D00F
:1001300098470E4B002B00D0984700200021040068
:100140000D000D48002802D00C4800E000BF0CF064
:100150003DF92000290008F0ADF90CF011F9C04676
:100160000000080000400020000000000000000027
:1001700070020020CC2F00200000000000000000D2
:1001800002000120104011D1042A0ED91368180969
:1001900080B2002809D001388000031D11180979A8
:1001A000002902D001309842F8D170470020FCE7C6
:1001B0000378002B03D05AB2002A01DB01307047CC
:1001C0003F229343C03B59424B41C01803789343AD
:1001D000802BF4D10130F9E710B500240378002B0F
:1001E00001D1200010BDFFF7E3FF0134F6E770B541
:1001F000002204000D00411C092003F0F3FE00283A
:1002000006D001236200134343600023A34200DBB6
:1002100070BD9A00A958821891600133F6E770B555
:10022000012803DC1C2001F06DFA70BD01230D686C
:1002300011201D42F7D04868184206D1042804D97D
:100240000F2302681340042B01D00E20EBE703F0CC
:1002500027FD6D100400002D03DDFFF7BDFFA84250
:1002600006DA1220DFE72000FFF7A2FF0400013DBD
:10027000012DF8D120787F2809DDDF280BDCF82359
:100280003F22DB00800118406378134018430123AC
:1002900040001843C9E7EF280BDCFC226378120109
:1002A0009B0113403F220007000C0343A07810403D
:1002B000ECE7F72812DCFC22637892021B03134060
:1002C000E0228004520310403F221843E378134099
:1002D000FC220343A07812018001E8E7012040429C
:1002E000D5E7F8B54D680F00EB0706D4042D04D907
:1002F0000F232E683340092B03D00B2001F002FAA4
:10030000F8BD6B683609B6B25C10731EA3420FD8F5
:100310000321200009F056FF6421642803DC01005A
:10032000032800DA03212800891903F08DFE050057
:100330002B6800201B099BB2013B9C42E0D23A682B
:10034000A31C9B005A510123013464001C436C60C0
:10035000D6E7F0B585B0012803DC1C2001F0D2F906
:1003600012E001274B683A000093022806D08B6800
:100370003B4203D05F10002F00DC17000125009BDB
:100380002B4203D00120404205B0F0BD009B042B5E
:10039000F8D91B680C680F261900314004292DD1AB
:1003A0002C4205D1042C03D923681E40042E01D011
:1003B0000E20D3E70098FFF7E3FEB842E2DB009897
:1003C00003F06EFC0600200003F06AFC03780100D5
:1003D000002BD7D0781E30180CF0EEFB041ED1D0C5
:1003E0003378002B01D0A64202D36800012521E01A
:1003F0003000FFF7DDFE01350600F1E709293ED1A7
:10040000009B5B685B1001939F42BBDC2C422ED1AA
:10041000042C2CD923683340042B28D1200003F06E
:100420003FFC039602907E1C009AB300D058844291
:1004300002D178002843A7E728420ED104280CD91E
:100440000368039A1340042B07D103F029FC010031
:1004500002980CF07BFB0028EBD0019B37009E42FA
:10046000E1DD8FE71F00019B9F4200DD8AE77B1CD7
:1004700000999A008A58A242F4D17800B6E703297D
:1004800000D07FE71A0992B25B0F92000B40D31A9B
:1004900001939F4200DD75E72C4229D1042C27D916
:1004A00022681640032E19D1100980B2520F800025
:1004B0003240251D801A019B2E181B1A0193009BA8
:1004C000781E0433019A904200DD5BE72A00191878
:1004D000B2420FD316D10130400087E7042E07D176
:1004E000200003F0DDFB05002000FFF749FEE2E7F6
:1004F0000F2033E70C78A4461478A44502D10131CB
:100500000132E5E70130DDE7F0B50D0085B00128E7
:1005100004DC1C2001F0F6F805B0F0BD01270868E6
:10052000384206D1042804D90F2102680A40042A5F
:1005300001D00E20EEE76A681740FAD1042AF8D9F4
:1005400013680B40042BF4D103F0AAFB0400686885
:1005500003F0A6FB02900CF003FB039000280FD1E0
:100560002000FFF739FE0190019B0122591C092050
:1005700003F038FD364E3060002815D10020CBE75F
:10058000029920000CF018FB001B4342434120005D
:100590000193019B5E1C0028E6D0039B0299C018C2
:1005A0000CF00AFB0196F4E70122019B5B00134368
:1005B0004360039B002B18D12000FFF7F9FD019B3E
:1005C0000500BB4201DC3068A6E7291B200003F0D0
:1005D00087FD0028D2D0BB1C32689B0098502800B1
:1005E000FFF7E6FD01372C00E9E7019B012B02D163
:1005F0002B68836090E7029920000CF0DDFA01255A
:100600000700019B002F13D0AB42DCDB391B20001D
:1006100003F066FD0028B1D032680135AB00985078
:10062000039B0299FC1820000CF0C6FA0700E8E7CB
:10063000AB42C8DB20000CF093FA0100200003F06D
:100640004FFD00289AD001353368AD00E850BAE775
:10065000E40F002010B503F007FB4300012018430E
:1006600010BD0000C30711D404280FD90F2302685E
:100670001340032B0AD119400133591AC0234907EB
:10068000DB051940024B1A40114301607047C04618
:10069000FFFFFF9F70B5002805DC1C2001F032F839
:1006A0000500280070BD01220C68144201D10D2004
:1006B000F4E701281CD04B681342F8D05B101320DC
:1006C000FF2BEBD81A0619040A431A431B021343E3
:1006D0006410E243D2171440E11C89101A00032071
:1006E00003F080FC051EDCD02100FFF7BBFFD8E73C
:1006F0000023EDE7F7B507000E001C20012F06DDF3
:100700004C68012322001A40009203D10D2000F012
:10071000F9FF53E0022F02D08A681A42F6D0012373
:1007200035681D4200D0A9E0042D00D8A6E01C4188
:10073000002C00DC1C000F2029680840092828D163
:100740006B685B100093022F05D0B368009A5B10B2
:100750009A4200DD0093009B01221D1B0135EB43F3
:10076000DB171D40691C092003F03CFC071E09D063
:1007700001236D001D430300326808334560009972
:10078000A14201DA3800FEBD0134A100515802C374
:10079000F5E7042845D1280003F082FAFFF71CFD95
:1007A0000190022F04D0B3685B10984200DD0193E2
:1007B000019BA34204DA002003F086FC0700E1E776
:1007C000280003F06DFA0700009BA34221DB2800FC
:1007D000009703F065FA05003800FFF7E9FC019B7C
:1007E00001340700A342F7DA009BC41A200003F08B
:1007F0006BFC071EC6D003F053FA0190306803F07B
:100800004FFA2200009B591B411801980BF002FE81
:10081000B8E73800FFF7CCFC009B070001330093DA
:10082000D2E703282AD10B099BB2490F9B00014054
:10083000591A022F04D0B2685210914200DD110003
:10084000A14205DA00220320110003F0CBFBB5E73B
:1008500003200E1B331DD9170140C918891000222F
:1008600003F0C0FB071E00D18CE7013631000334D2
:10087000FFF7F8FE381D29193200C7E7212046E7A7
:10088000F7B5002804DC1C2000F03CFF040014E055
:100890000D6801272E003E4011D03D41FF2D01D9AA
:1008A0001320F1E700223900032003F09BFB041E14
:1008B00003D03900FFF7D6FE25712000FEBD042DC0
:1008C000EED90F232A681340042B1BD12800FFF711
:1008D00057FCC31C07000320D9170140C918891011
:1008E000320003F07FFB041EE7D03900FFF7BAFEA9
:1008F000280003F0D5F9231D01003A0018000BF081
:1009000089FDDAE7092B1FD103206B6832005B10E9
:1009100001930333D9170140C918891003F062FB12
:10092000041ECAD00199FFF79DFE019B9E42C4DAC6
:10093000B300EB189B683B4204D05B10FF2BAFD891
:10094000A21913710136F0E7032BA9D12C00B4E7EB
:1009500010B57F2902DC0170013010BD1A4B99429D
:100960000CDC40238A115B42134303703F230B408E
:1009700080214942194341700230EEE7134B9942FE
:1009800010DC20230A135B4213433F2480220370B0
:100990008B1152422340214013430A43437082701B
:1009A0000330DAE70A4B9942D7DCF0230370603B4F
:1009B0004370113B8A11FF3B1A4382703F22114062
:1009C0001943C1700430C8E7FF070000FFFF0000B3
:1009D000FF0F0100F0B50D0085B0002803DC1C20DE
:1009E00000F090FE0DE009680122080010400AD0D6
:1009F00002AC11412000FFF7ABFF011B200003F008
:100A00006FFB04001AE004293FD90F230C68234030
:100A1000092B3AD14B685B10019303239C46019B41
:100A20009A420EDD03F050FB041E07D02E6801250C
:100A300003F036F92F00019B9D421DDD200005B01B
:100A4000F0BD01329300CC580123234001D127206F
:100A5000C6E764107F2C0DDD0D4E0223B44209DD84
:100A60000C4E6346B44205DD00270B4EE30FA64251
:100A70007B419B00C018D2E70135AB00F1583942E9
:100A8000E5D04910FFF764FFD5E70B20A8E7C04683
:100A9000FF070000FFFF0000FF0F010010B5012459
:100AA000044002D04410200010BD042810D90F23A8
:100AB00002681340042B07D103F0F2F821000A2248
:100AC0000CF016F90400EEE7032B01D10430F5E732
:100AD0000D2000F017FEE6E710B5040001200840E5
:100AE00010D104290DD90F230A681340042B08D113
:100AF000080003F0D5F8010020000CF027F843426D
:100B0000584110BD0020FCE7F7B50E00012803DCBA
:100B10001C2000F0F7FDFEBD4D68EB0706D4042D48
:100B200004D90F222B681A40092A01D00B20F0E7C4
:100B30006A681B099BB25410A34200D85C1E0127AF
:100B400031680F404810002F35D12648FFF7C4FF09
:100B500001230190002813D131682348FFF7BCFF1F
:100B6000002811D0002C0DD00122631C013C9440C0
:100B70009B005A5114436C6004E00137BA00AB503B
:100B8000BC42FADA0020C6E701233068184223D1BC
:100B9000042821D902680E331340042B1CD1FFF71F
:100BA0007DFF002807D131681048FFF795FF002826
:100BB00012D01220ADE70028FBDD8442F9DB830070
:100BC000EB180433844209DC0123621C013C9C4085
:100BD000920053511C43CEE711209AE75A68013026
:100BE0001A60EEE7EFDA0000F3DA0000F8DA00004E
:100BF000002310B50C000B70C30705D50D4942103A
:100C000020000BF067FF08E00B49002802D0042801
:100C100004D10A4920000BF07DFF10BD0428FCD947
:100C20000F2302681340042BF7D103F039F804496D
:100C30000200E5E784E60000FADA000000DB0000CD
:100C400005DB0000F0B593B0060002911C20012ED8
:100C50001DDD029B01251B681C002C4000D0ADE06F
:100C6000042B00D8E6E01A680F231A40092A4AD15B
:100C70000394039A029992008A5817002F4005D1D5
:100C8000042A03D910681840092806D0222000F051
:100C900039FD0190019813B0F0BD52685210A418AC
:100CA000039A013203929642E3D1611C012203F0C0
:100CB00099F90190002802D100230193EAE7019BF2
:100CC0006400190025435D600831029ABB00D058CA
:100CD00002684368120992B25B109A4200D8531E10
:100CE0000022934209DCDA43D21713409B00C91853
:100CF000039B01379F42E8DBCCE794000519AD6800
:100D000001320D51EDE72700032A59D10193029AD0
:100D1000BB00D3582B42B9D1042BB7D9186801991D
:100D20000140032939D1020992B2430F92000B40CE
:100D3000D31A1C190137BE42E9D10320E31CD9178D
:100D40000140C9188910002203F04CF901900028D5
:100D5000B2D000252100FFF785FC019B1E1D029AE1
:100D6000AB00D45801231C421FD1042C1DD90F21E4
:100D700023681940032918D1180980B25B0F80003D
:100D80000B40C01A0023834213DBC343DB17184018
:100D900001353618BD42E2DB7CE7042900D075E757
:100DA0001800FFF7EDF92418C4E72000FFF7E8F971
:100DB000E8E7E2181279F2540133E4E700273C0037
:100DC0000F25029ABB00D3580122134234D1042BC1
:100DD00032D9186801002940042935D11800FFF7DD
:100DE000CFF924180137BE42EBD1200003F06CF993
:100DF0000190002800D15FE7029FB600BB19041DD7
:100E0000029301233D681D4229D1042D27D90F26C5
:100E10002B681E40042E37D12800FFF7B1F90600D9
:100E2000280002F03DFF0100200032000BF0F2FA32
:100E3000A41922E02700C3E7180005A9FFF7D8FE90
:100E400005A80BF08DFECCE7032900D01EE70209B0
:100E500092B2430F92000B40D31A1C19C2E705A9A6
:100E60002800FFF7C5FE05A80BF07AFE05A90500CE
:100E7000020020000BF0CEFA6419029B0437BB423B
:100E8000BFD10023237005E7032EF6D11A0992B2D1
:100E90005B0F92001E40961B291DC5E7F0B50D00A3
:100EA00097B0002806DC1C2000F02CFC070038005E
:100EB00017B0F0BD0C68012123000B40009306D150
:100EC000042C04D922680F331A40092A01D00B20C0
:100ED000EAE7626852100392002A03DC009803F0EC
:100EE000F3F8E3E7504A019201280BD06868084202
:100EF00008D1042806D902681340042B02D102F05D
:100F0000CFFE019001980BF02BFE06000F27039BEC
:100F10000834013B05935E43039B02909B00E3185A
:100F2000049301232068184273D1042871D9016801
:100F30000B003B409C46042B03D1FFF721F9861997
:100F400009E0032B6CD162460B099BB2490F9B0051
:100F500011405A1A9619049B0434A342E1D130007F
:100F600003F0B2F8071EA2D02B680793029B002B58
:100F700003D0686802F094FE0190380002F090FE01
:100F80000400009B079A9B00D3189E68300002F073
:100F900087FE0123334005000693002B01D1042E68
:100FA00004D809A93000FFF723FE09AD28000BF093
:100FB000D7FD069B0490002B0ED1042E0CD90F21D7
:100FC00033681940032907D11A0992B25B0F9200C6
:100FD0000B40D31A351D04932000049A29000BF00E
:100FE00019FA049BE418029B002B0AD0059B009A77
:100FF000934206DD2000029A01990BF00BFA029B46
:10100000E418009B01330093009A039B9342B8D1EC
:101010004DE709A9FFF7ECFD09A80BF0A1FD8EE74C
:1010200002F03EFEF9E7C0461AE0000010B50122CA
:10103000002400280BDD0B681A40141E03D05C103E
:10104000E343DB171C400122904200D04A68611C38
:10105000092002F0C7FF002803D0012364001C43CD
:10106000446010BD0A6870B510000125284034D1D5
:10107000042A32D90F24136849681C40092C17D15F
:1010800054681B099BB22C41A34200D85C1E8442C9
:1010900005DC02200133984206DB00200FE08500CA
:1010A0005519A9600130F2E7840011510130F2E7CF
:1010B000032C12D1294203D1132000F023FB70BD71
:1010C0004910FF29F8D81B099BB204329B00D318A2
:1010D0009342E2D911700132FAE70B2000F012FBC3
:1010E000DBE700000123F7B500254E680C00334014
:1010F0000193AB420ED11D00042E0BD90F22336891
:101100001A40092A26D172681B099BB25510AB42BE
:1011100000D85D1E27687C10FB0746D439003D4887
:10112000FFF7DAFC002826D00BF070FC290009F04C
:101130002FF94C1C019B002B00D069E0042E67D9CD
:1011400032680F331340092B3BD10134A400A4595A
:101150002000FEBD042A04D13000FFF711F805007D
:10116000D8E7019D032AD5D11D09ADB25B0FAD00B3
:101170001340ED1ACEE739002748FFF7ADFC0028F1
:101180001DD1042F16D90F233A681340042B11D117
:101190003800FFF783FC041E07D139001F48FFF712
:1011A0009BFC002806D0122005E0002CFBDDA542A8
:1011B000C0DAF8E7112000F0A5FA0400C8E72C0017
:1011C000B8E7042B1CD1300002F06AFD0500012CA9
:1011D0000EDCFEF7EDFF461B300002F075FF041E2B
:1011E000B6D002F05DFD320029000BF013F9AFE735
:1011F0002B78013C002BD6D02800FEF7D9FFE5E77D
:10120000032B05D13419E37801245B001C439FE7CD
:101210000B20D0E7E8DA0000F3DA0000F8DA00008B
:10122000F7B54D680E002A0001210A402FD1042D88
:101230002DD90F242B68B7681C40092C14D169687C
:101240001B099BB24C100192A34200D85C1E31686E
:101250003448FFF741FC00282DD00F232A681340A3
:10126000092B1DD1012317E0032C10D10F4203D10C
:10127000132000F047FAFEBD7A100192FF2AF7D83A
:101280001A0992B25B0F92001C40141BDFE70B207F
:10129000EFE701339A00AF509C42FADA0020EAE708
:1012A000032BFBD12B0001335A1BA242F6DC6A460A
:1012B0001279DA70F7E736687010F30719D4310045
:1012C0001948FFF709FC002822D1042E1ED90F234C
:1012D00032681340042B19D13000FFF7DFFB0028E0
:1012E00007D131001148FFF7F7FB00280ED012207C
:1012F000BFE70028FBDD8442F9DB0F232A68134097
:10130000092B07D1013080004751C7E71120B0E712
:101310002000F2E7032BC1D16B461B792D18EB702F
:10132000BCE7C046EFDA0000F3DA0000F8DA0000AC
:1013300070B501240868204207D1042805D90F257B
:1013400001680D40092D02D14468200070BD032DB5
:1013500008D10A0992B24B0F92002B40D31A5B00BE
:101360001C43F2E7042DF0D102F09AFCFEF734FFA3
:1013700040000443E9E7000010B5034A0D2103488B
:1013800004F094FC10BDC04680DA000078DA00005A
:1013900000207047042070470120704710B50020DE
:1013A00002F092FE10BD0020704700207047002020
:1013B00070470020704700207047002070470020D1
:1013C000704700207047000010B5034A0C21034805
:1013D00004F06CFC10BDC0468CDB0000ECDB0000B0
:1013E00070470378002B03D05AB2002A01DB01308A
:1013F00070473F229343C03B59424B41C01803788A
:101400009343802BF4D10130F9E70000F8B50127B0
:10141000060014000800394227D104293FD90F23C0
:101420000A681A40042A3AD13C4213D1042C11D93B
:1014300022681340042B0DD102F032FC050020007D
:1014400002F02EFC010028000BF080FB00282EDBB0
:101450001FD127E0E30722D502F022FC0A22002157
:101460000BF046FC0500601010E0174015D1042A6F
:1014700015D90F2312681340042B10D120004D10F2
:1014800002F00EFC0A2239000BF032FC85420EDB22
:1014900008DD002E09DC00200CE04D10E3E70F22F0
:1014A000054B1A700136022EF5D8042002E0042004
:1014B00076173040F8BDC046B0020020F8B50600EF
:1014C00000242B4BE500ED182B79032B09D00134B8
:1014D000FF2CF6D1300004F0FDFB041E46D1013C88
:1014E00044E030000BF03CFBE3B202003100180096
:1014F00004F070FC002839D12A6851688842E6D08F
:101500008300D3189B680130F02BF7D101238000B2
:10151000083012181A42DAD1042AD8D90F211368D8
:1015200019400429D3D11B0998B20123013080004E
:1015300010181842CBD10428C9D90F2203681340D0
:10154000042BC4D102F0ACFB0327050009212800BD
:101550000BF0EEFA0028BAD0013F451C002FF5D160
:10156000310028000BF028FB8542B0D12000F8BDE7
:10157000A025002010B50124044002D04410200012
:1015800010BD042810D90F2302681340042B07D183
:1015900002F086FB21000A220BF0AAFB0400EEE712
:1015A000032B01D10430F5E70D22014B1A70E6E759
:1015B000B0020020012210B5024018D1042802D93F
:1015C00003681A0992B201230B4012D1042902D9EF
:1015D0000B681B099BB20024934206D104309B0088
:1015E0000431C318984206D30124200010BD002204
:1015F000E9E70023EFE704780A78002C01D1002AFC
:10160000F2D0013001319442ECD00024EDE700002B
:10161000F7B50700009101933049314B002A02D001
:1016200002220A70013A00261A601B68CE54BE429C
:1016300000DBF7BD009AB300D058294B274D1C683A
:10164000C8239B0065191C1B0123184206D0254A9C
:101650004310210028000BF00BFA09E0224A002871
:1016600002D004281BD1214A210028000BF000FAE7
:101670001A4C20000BF074FA194A019B1060002BE1
:101680000BD07B1EB34208DD194B984205D8431C92
:101690001360202222540022E2540136C7E70428B6
:1016A00019D90F2301680B40042B04D102F0F8FA7A
:1016B000104A0300CDE7092B03D143680E4A5B10A3
:1016C000C7E7032B08D10A0992B2490F92000B40D9
:1016D000D31A0A4ABDE70123094ABAE7B10200203A
:1016E000D405002084E60000FADA000000DB0000E8
:1016F0001F030000AFEC00005CDE00006BDE0000AA
:1017000076DE0000014B187000207047B002002008
:1017100070B502F065F8094C0100251D1F22280054
:101720000BF036FA28000BF01BFA04230430800873
:10173000000118432060200070BDC0468C020020CC
:10174000C368F0B59D00836889B05D190300183344
:1017500006930369069A9F00069B0290DF1943696E
:1017600001939B00D3180393D04B1B78002B26D1F9
:101770007F222B68CE491C1213409B005B58043516
:1017800001929F46029B587804F040FF0023029A82
:10179000137027E0C54B1B78002B10D12B68019AE2
:1017A0001C121340C24A9B009B580435E9E7069B74
:1017B0003A1DD11ABD4BD82928DD1A221A70029B76
:1017C000BA4C9B6821780193EA1A029B92109B788D
:1017D00012021A43029B587804F020FF0023029A59
:1017E00023701370029B069A9B680193ED1A029B6B
:1017F000AD10DD60069BFE1A029BB6101E61039BB6
:101800009B1A029A9B10536109B0F0BD39001B78F6
:1018100017000C60002BD2D12B68019A1C121340C8
:10182000A34A9B009B580435ABE7069B3A1DD11A8F
:101830009E4BD82902DD1A221A70C0E738001B78A7
:1018400017002A68291D0260002B01D00D00B6E7A1
:101850006B68019A1C121340954A9B009B580835EF
:101860008FE7069B3A1DD11A904BD82902DD1A2228
:101870001A70A4E73900A4001B782C1917000C601B
:10188000002B9CD12B68019A1C121340884A9B00A4
:101890009B58043575E7069B3A1DD11A834BD8290E
:1018A00002DD1A221A708AE739001700814AA40063
:1018B000A2581B780A60002B00D080E72B68019AA1
:1018C0001C1213407A4A9B009B58043559E7043F89
:1018D000784B3A68A400E250744B1B78002B00D080
:1018E0006DE72B68019A1C121340714A9B009B58AC
:1018F000043546E76F4BA400E058FFF73BFE6B4B07
:1019000006001B78002B09D1043F3868FFF732FE30
:101910000123861976001E43664BE650634B1B7805
:10192000002B00D04BE72B68019A1C121340604A31
:101930009B009B58043524E7069B391DCA1A5B4B54
:10194000D82A02DD1A221A7039E70698039C012270
:10195000A04202D222000C3A126838001B780F0015
:101960000260002B00D02AE72B68019A1C1213405A
:101970004F4A9B009B58043503E7069A3B1D991A72
:101980004A4AD82902DD1A23137018E706990398EA
:10199000814218D202000C3A12684749521064186A
:1019A000A41AA40022583A601F00404B1B78002B59
:1019B00000D004E72B68019A1C1213403C4A9B009C
:1019C0009B580435DDE6182111700022EBE7069BD9
:1019D000039A934219D213000C3B1B68364A5B10E2
:1019E000A418043FE41A3A68039BA400E2502F4B6A
:1019F0001B78002B00D0E2E62B68019A1C121340E2
:101A00002B4A9B009B580435BBE61822274B1A70C3
:101A1000EDE7069B039A934228D2274B043FE61832
:101A200014000C3C23685B10F31A9B009858FFF7D6
:101A3000A1FD04903868FFF79DFD2468049B6410A5
:101A4000341B1E18012376001E43039BA400E6509E
:101A5000164B1B78002B00D0B1E62B68019A1C12A4
:101A60001340134A9B009B5804358AE618220F4BFB
:101A70001A70EDE7069B3A1DD11A0C4BD82902DDEE
:101A80001A221A709BE639001700039AA400A25884
:101A90001B780A60002B00D091E62B68019A1C127B
:101AA0001340034A9B009B5804356AE6B0020020AD
:101AB0005CDC0000982D0020FDFFFF3F043F039BEE
:101AC0003A68A400E250D64B1B78002B00D076E693
:101AD0002B68019A1C121340D24A9B009B58043574
:101AE0004FE6039BA4001C192368043F38685E106E
:101AF000FFF740FD0123361876001E43C84B2660D1
:101B00001B78002B00D05AE62B68019A1C12134058
:101B1000C44A9B009B58043533E6069BA4003F1B38
:101B2000BF4CBB420CD82378002B00D047E62B6873
:101B3000019A1C121340BB4A9B009B58043520E6B7
:101B4000B94802F09DF82378002B00D037E62B68C7
:101B5000019A1C121340B34A9B009B58043510E6AF
:101B6000A300ED18002C00DA3CE6AD4B1B78002BEF
:101B700000D024E62B68019A1C121340A94A9B004E
:101B80009B580435FDE5043F3B68042B04D1A300BA
:101B9000ED18002C00DA25E6A14B1B78002B00D0B5
:101BA0000DE62B68019A1C1213409E4A9B009B581D
:101BB0000435E6E5043F3B68042B04D0A300ED1890
:101BC000002C00DA0EE6964B1B78002B00D0F6E5D1
:101BD0002B68019A1C121340924A9B009B580435B3
:101BE000CFE501233E1F306818420AD01841013862
:101BF000002809DB01234000A40018432D193060A0
:101C0000F0E5FFF7B7FCF2E7854B1B78002B01D01E
:101C10003700D4E52B68019A1C121340814A9B00BF
:101C20009B5837000435ACE5FF20610040000140BF
:101C3000FE38FF380143396002993B00896824125D
:101C400004916D1A0299AD1089782D020D438540DB
:101C500005437D6006991700039A521A921082403C
:101C600002439A60029B029A9C70E4B26F4BE400BC
:101C7000E35893606A4A1278002A03D008331D00A3
:101C800003979CE51D00019A9B680C351C121340BC
:101C9000644A9B009B58039773E53B1F1C68039A9B
:101CA000069B934232D10A20E30711D4042C18D9A1
:101CB0000F2322681340042B16D1200001F0F0FFFF
:101CC0000AF04EFFC8239B00984200D91800063046
:101CD000643004F0B3F800280FD1043D069B039351
:101CE00080E50720042CF3D02000431E9841FA23FE
:101CF0004042FF3318400730EAE7029B2100587842
:101D000004F09EFC0023029A1370E7E7039B039AFA
:101D10000C3B1B6802995B109B00D31A0C3B1C60A8
:101D20001F1D1300083B1B685A108A70D2B23F492E
:101D3000D2005B0055589B0A029A9B009560ED18F3
:101D4000039B069A043B1B685B109B00D31803930C
:101D5000334B1B78002B00D031E52B68019A1C1205
:101D60001340304A9B009B5804350AE53B1F186816
:101D7000FFF700FCA40006003F1B1E2827DC0028FC
:101D80000DDC274B1B78002B00D018E52B68019A3F
:101D90001C121340234A9B009B580435F1E401F0C8
:101DA00005FD033E361801F001FD214B801B9842D2
:101DB000F9D81B4B1B78002B00D000E52B68019A4B
:101DC0001C121340174A9B009B580435D9E4012389
:101DD000029A137001F0EAFC029B0A3886195E60D1
:101DE00000E53B1F1868FFF7C5FBA40006003F1B7A
:101DF00000280DDC0A4B1B78002B00D0DFE42B6899
:101E0000019A1C121340074A9B009B580435B8E402
:101E1000084B984210DD1D22014B1A70CFE4C046DA
:101E2000B00200205CDC000088DE0000A02500205D
:101E30003F420F0080EE36000123029A137001F03A
:101E4000B5FCFA239B005E430A3E3018029B5860A3
:101E5000C8E4A300FF1A002320001A003900FFF78E
:101E6000D7FBD74ED74C3168200002F039F9D64B5A
:101E700031681860200004F0A3FA3168200004F0F3
:101E8000E6FBD24B1B78002B00D098E42B68019A1C
:101E90001C121340CE4A9B009B58043571E4CB4B77
:101EA000A4001B783F1B002B00D088E42B68019A0C
:101EB0001C121340C64A9B009B58043561E40298EB
:101EC00004F020F8C14B1B78002B00D077E42B687E
:101ED000019A1C121340BE4A9B009B58043550E4E3
:101EE0003B1F1B68002B58D13B0001260C3B186898
:101EF00006402FD046103A0001217300083A0B43E8
:101F00001360002E00DC95E0012173000B433A1FA3
:101F100013603B00083B1B680B419B1B04933B0079
:101F20000C3B186808423BD0049BA4005B188B4014
:101F30000B43039AA350A54B1B78002B00D03EE423
:101F40002B68019A1C121340A14A9B009B58043530
:101F5000FFF717FC04281BD90F2302681340092B35
:101F600002D143685E10C6E7042B08D101F098FE49
:101F70000378002BBFD0FFF734FA0136F8E7032BC4
:101F800006D11609B6B2520FB6001340F61AB2E7E0
:101F900019228E4B1A70FFF712FC5B105E1EB0E721
:101FA000042842D90F2302681340092B05D1049B52
:101FB000A40002339B001B58BBE7042B2BD1039BCF
:101FC000A4001B19079301F06BFE0600049C01346A
:101FD000012C10DC3000FFF704FA831B1800049377
:101FE00002F072F8041E0ED001F05AFE049A31007D
:101FF0000AF010FA07E03178013C002906D11222DC
:102000000C00724B1A70079B1C6094E73000FFF7BE
:10201000E8F90600DCE7032B07D10122049BA400AA
:10202000C01803795B00134383E71922674B1A70CA
:10203000FFF7C5FB04357EE7A300069AFB189B1A41
:10204000D82B08DD1A22614B1A70FFF7B8FB01226A
:102050001C003A600437631E002CF8DC5B4B1B78D5
:10206000002B01D0FFF7ABFB2B68019A1C12134029
:10207000574A9B009B580435FFF783FB069A3B1D8C
:102080009B1A524ED82B03DD1A233370FFF797FBB0
:10209000069B039AA40093422AD23B1F1868FFF7BD
:1020A00069FA011E21DD039B0C3B1A685210824223
:1020B0001BDB9007801A474B4018C018039B800019
:1020C000C2583B1B1A60414B3F1B1B780437002B47
:1020D00001D0FFF774FB2B68019A1C1213403C4A95
:1020E0009B009B580435FFF74CFB20233370EAE735
:1020F0001823FBE7344BA4001A683B1B1F001A602F
:10210000324B04371B78002B01D0FFF758FB2B68AC
:10211000019A1C1213402E4A9B009B580435FFF76E
:1021200030FB3A1F1368042B02D13A00A4002D198A
:10213000264B1B78002B02D01700FFF740FB2B68C3
:1021400001991C120B4022499B005B581700043573
:10215000FFF717FB043F3B68042B04D00023A400C7
:102160003B602D190437194B1B78002B01D0FFF76A
:1021700026FB2B68019A1C121340154A9B009B58A2
:102180000435FFF7FEFAA3009C46F81A002C23DC66
:102190001C2200260D4B1A706346FF1A0B4B06607B
:1021A0001B780437002B01D0FFF709FB2B68019A3D
:1021B0001C121340064A9B009B580435FFF7E1FAB6
:1021C000D4050020B102002008000020B002002049
:1021D0005CDC0000FCFFFF3F002103685B10012670
:1021E0008A008258164003D10D22D54B1A70D3E7CE
:1021F0005210934200DD130001318C42EFDC5E008F
:1022000001231E43C8E7A3009C46F81A002C17DCE4
:102210001C220026CA4B1A706346FF1AC84B066080
:102220001B780437002B01D0FFF7C9FA2B68019AFD
:102230001C121340C34A9B009B580435FFF7A1FAB8
:10224000002103685B1001268A008258164003D1E2
:102250000D22BB4B1A70DFE75210934200DA1300D5
:1022600001318C42EFDC5E0001231E43D4E73B00CA
:102270000122083B1968A40011421DD03B1F1B68B6
:10228000134219D0114113410022994200DA04325D
:102290003B1B1A60AA4B3F1B1B780437002B01D055
:1022A000FFF78DFA2B68019A1C121340A54A9B0078
:1022B0009B580435FFF765FA02203B1F1A6840421D
:1022C000FFF7A4F83E1B3060E4E73B000120083B29
:1022D0001968A40001421ED03B1F1A6802421AD09E
:1022E00001415010CB0FD217884253413A1B9B003B
:1022F0001360934B3F1B1B780437002B01D0FFF773
:102300005EFA2B68019A1C1213408E4A9B009B5860
:102310000435FFF736FA01203B1F1A684042FFF7E9
:1023200075F83E1B3060E4E73B00083B18683B1F34
:102330001968A600BE1B0423814202D0042802D8DB
:102340000023336016E001231842F9D10F230268FD
:102350001A40042AF4D1033A1142F1D10429EFD9E9
:102360000A681340042BEBD1FFF724F9431E984170
:1023700080003060724BA4001B783F1B0437002B99
:1023800001D0FFF71CFA2B68019A1C1213406D4A0A
:102390009B009B580435FFF7F4F93B00083B186895
:1023A0003B1F1968A600BE1B0023814202D00428EF
:1023B00002D80423336016E001231842F9D10F2319
:1023C00002681A40042AF4D1033A1142F1D10429D7
:1023D000EFD90A681340042BEBD1FFF7EBF8434227
:1023E000584180003060564BA4001B783F1B0437D7
:1023F000002B01D0FFF7E3F92B68019A1C12134060
:10240000504A9B009B580435FFF7BBF93B00012263
:10241000083B1968A40011421ED03B1F1B681342E1
:102420001AD05B104A10D80FC9179A4241413B1B82
:1024300089001960424B3F1B1B780437002B01D0E9
:10244000FFF7BDF92B68019A1C1213403D4A9B000F
:102450009B580435FFF795F93B1F1A680120FEF7DA
:10246000D5FF3E1B3060E5E73B000122083B1968C1
:10247000A40011421DD03B1F1B68134219D011410B
:1024800013410022994200DD04323B1B1A602C4BA1
:102490003F1B1B780437002B01D0FFF790F92B6806
:1024A000019A1C121340274A9B009B580435FFF7E2
:1024B00068F93B1F1A680220FEF7A8FF3E1B306038
:1024C000E5E73B1F1B68A400043B5A1E93413A1BDF
:1024D00017009B0013601A4B04371B78002B01D0A8
:1024E000FFF76DF92B68019A1C121340154A9B00E7
:1024F0009B580435FFF745F93B00083B1868FFF788
:1025000039F83B1F06001868FFF734F80121A400D2
:102510003B1B1F00321852000A431A60084B043755
:102520001B78002B01D0FFF74AF92B68019A1C1287
:102530001340044A9B009B580435FFF722F9C0461C
:10254000B00200205CDC00003B00083B1868FFF78D
:1025500011F83B1F06001868FFF70CF80121A400D2
:102560003B1B1F00321A52000A431A60E44B043727
:102570001B78002B01D0FFF722F92B68019A1C125F
:102580001340E04A9B009B580435FFF7FAF83B00E4
:10259000083B1868FEF7EEFF3B1F06001868FEF7C1
:1025A000E9FF02000121A4003B1B1F0072435200FF
:1025B0000A431A60D24B04371B78002B01D0FFF777
:1025C000FEF82B68019A1C121340CE4A9B009B58C0
:1025D0000435FFF7D6F83B1F1868FEF7CBFF061E41
:1025E00017D11F23C64A1370A4003B1B1F001E6097
:1025F000C34B04371B78002B01D0FFF7E0F82B68A2
:10260000019A1C121340BF4A9B009B580435FFF7E8
:10261000B8F83B00083B1868FEF7ACFF310007F044
:10262000D1FD012346001E43DEE73B1F1868FEF77D
:10263000A1FF061E17D11F23B14A1370A4003B1B34
:102640001F001E60AE4B04371B78002B01D0FFF734
:10265000B6F82B68019A1C121340AA4A9B009B589B
:102660000435FFF78EF83B00083B1868FEF782FF41
:10267000310007F08DFE01234E001E43DEE73B1FB5
:102680001868FEF777FFC217801850400122A40097
:102690003B1B1F00400010431860994B04371B7808
:1026A000002B01D0FFF78BF82B68019A1C12134006
:1026B000944A9B009B580435FFF763F8A300FE1A69
:1026C0003068012C25D1FEF755FF012307900493B4
:1026D0000AF09CF90799002900DC012107F058FE57
:1026E000049BA400C918012349001943844B3F1BD4
:1026F0001B7831600437002B01D0FFF760F82B689E
:10270000019A1C1213407F4A9B009B580435FFF727
:1027100038F8FEF72FFF04907068FEF72BFF049B3C
:102720000130C31A0793D3E7A300FE1A310020003B
:10273000049301F05BFE049B3060FF1A704B04377A
:102740001B78002B01D0FFF73AF82B68019A1C1276
:1027500013406C4A9B009B580435FFF712F83B006E
:10276000083B1868FEF706FF3B1F06001868FEF7D7
:1027700001FF02000121A4003B1B1F003240520058
:102780000A431A605E4B04371B78002B01D0FFF719
:1027900016F82B68019A1C1213405A4A9B009B584A
:1027A0000435FEF7EEFF3B00083B1868FEF7E2FE3B
:1027B00006003B1F1868FEF7DDFE32000121A40071
:1027C0003B1B1F00024352000A431A604C4B043764
:1027D0001B78002B01D0FEF7F2FF2B68019A1C1228
:1027E0001340484A9B009B580435FEF7CAFF3B0044
:1027F000083B1868FEF7BEFE06003B1F1868FEF790
:10280000B9FE32000121A4003B1B1F0042405200D0
:102810000A431A603A4B04371B78002B01D0FEF7AD
:10282000CEFF2B68019A1C121340364A9B009B581E
:102830000435FEF7A6FF3B1F1868FEF79BFEC0435A
:102840000122A4003B1B1F004000104318602C4BCA
:1028500004371B78002B01D0FEF7B1FF2B68019ADB
:102860001C121340274A9B009B580435FEF789FF32
:102870003B00083B1868FEF77DFE06003B1F18680A
:10288000FEF778FE320082400121A4003B1B1F00AE
:1028900052000A431A601A4B04371B78002B01D0F0
:1028A000FEF78DFF2B68019A1C121340154A9B00FE
:1028B0009B580435FEF765FF3B00083B1868FEF7A0
:1028C00059FE06003B1F1868FEF754FE3200024115
:1028D0000121A4003B1B1F0052000A431A60084B51
:1028E00004371B78002B01D0FEF769FF2B68019A93
:1028F0001C121340034A9B009B580435FEF741FF0E
:10290000B00200205CDC00003B000C3B1868FEF7C6
:1029100031FE3B00083B06001868FEF72BFEF1175E
:102920000200C317300007F085FD3B1F049005919E
:102930001868FEF71FFE02000498059907F02EFDA7
:102940000123A4003E1B370040001843E54B3060D4
:102950001B780437002B01D0FEF731FF2B68019A5A
:102960001C121340E04A9B009B580435FEF709FFF8
:10297000A300FE1A310020000493FEF757FB049BCE
:102980003060FF1AD74B04371B78002B01D0FEF7BD
:1029900016FF2B68019A1C121340D34A9B009B58C8
:1029A0000435FEF7EEFEA300FF1A39002000FEF703
:1029B00059FBCC4B1B78002B01D0FEF700FF2B6896
:1029C000019A1C121340C84A9B009B580435FEF71D
:1029D000D8FEA300FE1A310020000493FEF782FB0C
:1029E000049B3060FF1ABF4B04371B78002B01D0CB
:1029F000FEF7E5FE2B68019A1C121340BA4A9B00B1
:102A00009B580435FEF7BDFEA300FF1A39002000D5
:102A1000FEF706FCB34B1B78002B01D0FEF7CFFE70
:102A20002B68019A1C121340AF4A9B009B58043537
:102A3000FEF7A7FEA300FE1A310020000493FEF764
:102A400077FC049B3060FF1AA64B04371B78002BE1
:102A500001D0FEF7B4FE2B68019A1C121340A24A63
:102A60009B009B580435FEF78CFE3B1F186801F055
:102A700017F93A000121083A12680300A4000A423B
:102A800029D1042A0CD910680F22104001380828D7
:102A90000FD807F003FB052026220E0E0E0E240091
:102AA000924918000AF052F8434258413B1B8000FB
:102AB00018608C4B3F1B1B780437002B01D0FEF7AE
:102AC0007EFE2B68019A1C121340874A9B009B587C
:102AD0000435FEF756FE8649E3E78649E1E7864975
:102AE000DFE78649DDE7069B3E1DF31A7D4CD82BB8
:102AF00003DD1A232370FEF762FE00F061FE01225F
:102B00003B0040001043186023783700002B01D0B1
:102B1000FEF755FE2B68019A1C121340724A9B0067
:102B20009B580435FEF72DFE069B3E1DF31A6D4C97
:102B3000D82B03DD1A232370FEF741FE00F036FE8A
:102B40006F4A4000104001223B0010431860237878
:102B50003700002B01D0FEF732FE2B68019A1C12C1
:102B60001340614A9B009B580435FEF70AFE069A03
:102B70003B1D9B1A5B4CD82B03DD1A232370FEF7F9
:102B80001EFE00F01DFE5F4B1A68831A904201D2B0
:102B90005D4A9B1801213A005B000B4313602378C8
:102BA0000437002B01D0FEF70AFE2B68019A1C1295
:102BB00013404D4A9B009B580435FEF7E2FD00F0A0
:102BC000FFFD504BA4001860464B3F1B1B78002BA9
:102BD00001D0FEF7F4FD2B68019A1C121340424A03
:102BE0009B009B580435FEF7CCFD00F0F7FDA300D9
:102BF000002810D1FF1A3B4B1B78002B01D0FEF7A9
:102C0000DEFD2B68019A1C121340374A9B009B582B
:102C10000435FEF7B6FD3E00FF1A012320001A001E
:102C20003900FEF7F5FC394C2068643003F006F9F2
:102C3000002803D1043D3700FEF7D4FD029B216834
:102C40005A78334803F015FD0123029A137000F0FF
:102C5000ADFD304B22681B68063253431818FFF74E
:102C6000F5F800F0BBFDA300002810D1FF1A1D4BA2
:102C70001B78002B01D0FEF7A2FD2B68019A1C12D5
:102C80001340194A9B009B580435FEF77AFD3E001D
:102C9000FF1A2000012300223900FEF7B9FC1B4C6B
:102CA0002068643003F0CAF80028C3D0184803F045
:102CB00071FAC9E7A4003E1BFEF72AFD3700094B55
:102CC00030601B780437002B01D0FEF778FD2B68AD
:102CD000019A1C121340044A9B009B580435FEF7CE
:102CE00050FDC046B00200205CDC000098DE000011
:102CF000A0DE0000A7DE0000AEDE0000B3DE0000B4
:102D0000FEFFFF7FDC05002037894100D40500204D
:102D1000B102002004000020FB4BA4001B783F1BE5
:102D2000002B01D0FEF74BFD2B68019A1C121340BB
:102D3000F64A9B009B580435FEF723FDA4003E1B7A
:102D4000300000F078FD3700EF4B30601B7804371F
:102D5000002B01D0FEF733FD2B68019A1C121340A3
:102D6000EA4A9B009B580435FEF70BFDA4003E1B6E
:102D7000300000F062FD3700E34B30601B78043711
:102D8000002B01D0FEF71BFD2B68019A1C1213408B
:102D9000DE4A9B009B580435FEF7F3FCA300FE1AA5
:102DA00031002000049300F025FC049B3060FF1AE2
:102DB000D54B04371B78002B01D0FEF700FD2B68A4
:102DC000019A1C121340D14A9B009B580435FEF710
:102DD000D8FCA4003F1B380000F032FDCA4B1B7822
:102DE000002B01D0FEF7EBFC2B68019A1C1213405C
:102DF000C64A9B009B580435FEF7C3FCA300FE1A8D
:102E000031002000049300F027FC049B3060FF1A7F
:102E1000BD4B04371B78002B01D0FEF7D0FC2B688C
:102E2000019A1C121340B94A9B009B580435FEF7C7
:102E3000A8FCA4003F1B380000F048FDB24B1B78F3
:102E4000002B01D0FEF7BBFC2B68019A1C1213402B
:102E5000AE4A9B009B580435FEF793FC01212000ED
:102E600000F01CFDA84B1B78002B01D0FEF7A7FC3F
:102E70002B68019A1C121340A44A9B009B580435EE
:102E8000FEF77FFC0021200000F008FD9E4B1B7820
:102E9000002B01D0FEF793FC2B68019A1C12134003
:102EA0009A4A9B009B580435FEF76BFCA4003E1B1E
:102EB000300000F039FD3700934B30601B78043749
:102EC000002B01D0FEF77BFC2B68019A1C121340EB
:102ED0008E4A9B009B580435FEF753FCA4003E1B12
:102EE000300000F035FD3700874B30601B78043729
:102EF000002B01D0FEF763FC2B68019A1C121340D3
:102F0000824A9B009B580435FEF73BFCA4003F1B04
:102F1000380000F0F1FC7C4B1B78002B01D0FEF751
:102F20004EFC2B68019A1C121340784A9B009B5858
:102F30000435FEF726FCA4003F1B380003F09EFF7B
:102F4000714B1B78002B01D0FEF739FC2B68019ADE
:102F50001C1213406D4A9B009B580435FEF711FC70
:102F6000A4003E1B300004F043F83700664B30608D
:102F70001B780437002B01D0FEF721FC2B68019A47
:102F80001C121340614A9B009B580435FEF7F9FB65
:102F9000A4003F1B380003F00BFF5B4B1B78002B9A
:102FA00001D0FEF70CFC2B68019A1C121340574A03
:102FB0009B009B580435FEF7E4FBA4003E1B300049
:102FC00003F010FF3700504B30601B780437002BA4
:102FD00001D0FEF7F4FB2B68019A1C1213404B4AF8
:102FE0009B009B580435FEF7CCFBA300FF1A390069
:102FF000200001F06FFD444B1B78002B01D0FEF741
:10300000DEFB2B68019A1C121340404A9B009B5820
:103010000435FEF7B6FBA300FF1A3900200001F0CB
:1030200079FB394B1B78002B01D0FEF7C8FB2B68CE
:10303000019A1C121340354A9B009B580435FEF739
:10304000A0FBA300FF1A3900200001F0FBFB2E4B70
:103050001B78002B01D0FEF7B2FB2B68019A1C12E3
:1030600013402A4A9B009B580435FEF78AFBA300B5
:10307000FF1A3900200001F00DFC234B1B78002BB8
:1030800001D0FEF79CFB2B68019A1C1213401F4ACB
:103090009B009B580435FEF774FBA300FE1A310019
:1030A0002000049304F08EF8049B3060FF1A164B46
:1030B00004371B78002B01D0FEF781FB2B68019AA7
:1030C0001C121340114A9B009B580435FEF759FB14
:1030D000A300FE1A31002000049304F07BF8049B47
:1030E0003060FF1A084B04371B78002B01D0FEF725
:1030F00066FB2B68019A1C121340044A9B009B58E4
:103100000435FEF73EFBC046B00200205CDC000048
:10311000A300FE1A31002000049304F063F8049B1E
:103120003060FF1AAA4B04371B78002B01D0FEF742
:1031300046FB2B68019A1C121340A64A9B009B5821
:103140000435FEF71EFBA300FE1A31002000049395
:1031500003F00CFD049B3060FF1A9D4B04371B7875
:10316000002B01D0FEF72BFB2B68019A1C12134099
:10317000984A9B009B580435FEF703FBA300FF1AF7
:103180003900200001F026FC914B1B78002B01D068
:10319000FEF715FB2B68019A1C1213408D4A9B0009
:1031A0009B580435FEF7EDFAA300FF1A3900200002
:1031B00001F098FB864B1B78002B01D0FEF7FFFA3D
:1031C0002B68019A1C121340824A9B009B580435BD
:1031D000FEF7D7FAA300FE1A31002000049301F095
:1031E000FDFA049B3060FF1A794B04371B78002BE3
:1031F00001D0FEF7E4FA2B68019A1C121340754ABD
:103200009B009B580435FEF7BCFAA300FF1A390057
:10321000200001F0ABFA6E4B1B78002B01D0FEF7BB
:10322000CEFA2B68019A1C1213406A4A9B009B58E5
:103230000435FEF7A6FA002C79DD3B1F1E68012C31
:103240000CD1264207D1042E05D90F233268300055
:103250001340042B11D001235B4213E0022CFAD15E
:103260003B00083B186801231842F4D10428F2D926
:1032700002680E331340042BEDD100F011FDFEF770
:103280001DF90300A200BF1A5A1C50D00020022CC6
:1032900011D101223240824223D1042E21D90F21A3
:1032A0003068014009291CD171684810C0B2810002
:1032B000914211D17F18FF2B1BD81C0204433A0006
:1032C000069B0C32D31AD82B01DCFEF7ADFC1A2278
:1032D0003F4B1A70FEF773FAB418A468BC5004325E
:1032E000E6E70B223A4B1A7000233B600437FEF7E7
:1032F00066FA069A0299BA1A86009210BE1B0A61F3
:10330000310098470022344B371D1A60304B306033
:103310001B78934201D0FEF752FA2B68019A1C12D7
:1033200013402C4A9B009B580435FEF72AFA0023D1
:103330003B60274B3A1D1B78002B02D01700FEF78D
:103340003EFA2B6801991C120B4022499B005B58E6
:1033500017000435FEF715FA069B029AFB1A9B101C
:103360001361A300FF1A3900200002F051FF184B2F
:103370001B78002B01D0FEF722FA2B68019A1C1251
:103380001340144A9B009B580435FEF7FAF9069B3C
:10339000029AFB1A9B101361A300FE1A3100200051
:1033A000049302F035FF049B3060FF1A084B04378A
:1033B0001B78002B01D0FEF702FA2B68019A1C1231
:1033C0001340044A9B009B580435FEF7DAF9C046C7
:1033D000B00200205CDC0000E40F00200023F7B501
:1033E0005A1E0192002B07DA01F08AFB03F028F83D
:1033F00003F09EF91923019300263000194B196838
:10340000B14212DD184B1A6801328A420FDAF024F9
:103410001A601D68154F6C43E35D002B1FD0E41943
:10342000022B06D12000FEF78BF9019BD8E7002282
:10343000EDE7012B0DD1002801D100F0B7F9F02202
:103440006A43BB185B680A49C31A8B4201D802233E
:10345000BB54F0235D43054BEB5C022BE2D00136FD
:10346000CCE7C046D805002000000020401C00200A
:103470003F420F0080220B4B52001A600121A8220C
:10348000A920094BD20019649A58C00005321A507D
:1034900006481A50C122C020920000039850044BE5
:1034A0001970704700E100E0008000404C0500000A
:1034B0000306002004207047F8B550C901232200FC
:1034C0001A40101E2DD03340181E2AD06410002040
:1034D0001C2C26D81D4B761035009E4200DD1D00A9
:1034E0001B4F3B5D012B05D00121200005F0C6F9E3
:1034F00001233B55174B1B78002B01D1FFF7BAFF77
:103500000023154A9E420DDCFF2514491448D65C61
:10351000B44202D15E007052D5540133042BF6D16F
:103520000420F8BDD15C8C4203D10C4A5B009D5253
:10353000F6E70133042BF5D10023D15CFF2901D13B
:10354000D454F2E70133042BF7D1E9E788130000E4
:10355000E4050020030600201C0000200E000020CF
:10356000DC05000070B530C9012322001A40101E8E
:103570001BD02B40181E18D064101C2C00D900241E
:10358000154E335D012B05D00121200005F076F9A1
:103590000123335569100800104A1038104B90422F
:1035A00004D9012252421A60042070BD1C600D48EB
:1035B00006F008FE0C4B040018800C4B1B78002B07
:1035C00001D1FFF757FF0122094B9A64A922D200CB
:1035D000995864189C50E7E7E405002090860100A4
:1035E0001800002020A107000C0000200306002086
:1035F00000800040F8B501240B6806000D0023424E
:1036000004D10D20FEF77EF82000F8BD5B102000ED
:10361000052BFAD80E4A9B009C580E4F3B5D002BA1
:1036200005D00021200005F029F900233B55012E8B
:1036300006DD6B68042B03D10221200005F01EF982
:10364000200004F0C9FF012440002043DDE7C0460C
:1036500028DF0000E405002070B501240D68254234
:1036600004D10D20FEF74EF8200070BD6D101C2D0A
:1036700017D80024012804DD4C68043C63425C41F7
:103680006400094E735DA34204D02100280005F0B8
:10369000F5F87455280005F025F903000420012BE6
:1036A000E3D00020E1E7C046E4050020F8B501269C
:1036B0000D683400B04200DD4C682B003340181E0A
:1036C0000BD023003340181E07D06D10002D05DCF1
:1036D000A12300201E4ADB00D650F8BD6410002054
:1036E0001C2CFAD81B4F3B5D012B04D0012120007C
:1036F00005F0C4F83E552900174806F063FD0A217D
:10370000053006F05FFD154BA400E258144B120281
:103710001343A2221349D2008B50134C0C4B9C50E4
:10372000124C1951012412495C50124B19690021A5
:103730009950114A904200DD1000A8228021D20049
:103740009850012289005A5004201A60C5E7C046EB
:1037500000F00140E405002000B4C40474F000004F
:10376000030003000060004040A100401405000079
:103770000405000000A00040FFFF0000030010B59A
:103780000120002B02DC1B30FDF7BCFF10BD042024
:10379000704710B5002803DC1C20FDF7B3FF10BDF7
:1037A0000B680020DB07FAD40D30F6E70122034B4B
:1037B0001A64A822D20098587047C0460080004082
:1037C0000122054B10B51A64A822FA21D20098589C
:1037D000890006F06DFC10BD00800040012070479C
:1037E0000048704740DF00001D20704770B5054E4F
:1037F0000400335C0D008B4202D005F03FF83555D4
:1038000070BDC046E405002070B50024084D635D1E
:10381000012B09D10021200005F04EF800212000E5
:1038200005F02CF80023635501341D2CEED170BD3A
:10383000E405002070470D2070473B2070470000D2
:10384000F8B501260568354202D04468344203D1F8
:103850000D20FDF757FFF8BD6D101C2DFBD80A4F4A
:103860007B5D012B04D03100280005F007F87E5560
:10387000064964108C4202DCE143C917214028004C
:1038800004F030FFE7E7C046E4050020FF03000036
:1038900010B50800FFF7D4FF002010BD70B504007C
:1038A0000D001C280ED8084E335C012B04D00121DA
:1038B00004F0E4FF01233355290020004D1EA941E7
:1038C00004F0FAFF70BDC046E4050020036810B59F
:1038D000DA0703D40D20FDF715FF10BD416858101D
:1038E00004394A425141FFF7D9FFF6E710B5080005
:1038F000FFF7ECFF002010BD37B569460A00064B04
:1039000030CB30C203680220042B02D100F09AFFB2
:1039100037BD00F0BFFFFBE7C0DE000010B50800B8
:10392000FFF7EAFF002010BD10B5084C6379002BAB
:1039300005D00021052004F0A1FF002363710520BC
:1039400004F0D0FF43425841800010BDE405002040
:1039500010B5084CE37A002B05D000210B2004F0B1
:103960008DFF0023E3720B2004F0BCFF434258415B
:10397000800010BDE4050020A02200230349D200EE
:103980008B50034910328B507047C04600F0014005
:1039900000600040F7B52F4D2F4EEB6C002B14D07C
:1039A000A9240023E4003759EB642C4B1868002845
:1039B0000BDB2B4B19784A425141C9B2197004F004
:1039C0007BFF284B1B88DF1937512B6D002B38D01C
:1039D0000021254B254FF45829653A780193244D51
:1039E0008A4206D02B68032B03D8224AD05C04F00D
:1039F00063FF2B68204A0133134004D50422013BA6
:103A00005242134301331B4900228C462B60042B86
:103A100018D06046C05C591CFF2802D10B0001225F
:103A2000F5E7002A00D02B60012104F045FF0123B7
:103A30003B702B68114A5B009B5A0C34E418019BC5
:103A4000F450F7BD01235B422B6000233B700C4B0D
:103A5000F4E7C046FC8000400080004018000020D1
:103A6000020600200C0000204C050000010600208A
:103A7000E00500201C000020030000800E00002054
:103A80005C460000084B094AFF201A805A809A8041
:103A9000DA800023064A07491370074A0870487005
:103AA0008870C870136070470E000020DC050000AD
:103AB000010600201C000020E00500200122024B2E
:103AC00052421A607047C0461800002010B5034AE1
:103AD0000C21034802F0EAF810BDC046C8DE000021
:103AE000B6E70000E12170B54902194804F0EAFA8E
:103AF000002401220320174B17491A615C5004313E
:103B000058508018083158501A60063004F05EFD95
:103B1000FF21124AA15401341D2CFBD101220020A7
:103B20000F4B01001A6004230E4A0F4D1468002C3D
:103B3000FCD02C680002013B20431160002BF5D122
:103B400001220A4B1A6004F079FC01F025F970BDDE
:103B5000C81B00200080004004050000E405002090
:103B600000D0004000D1004008D5004004D0004003
:103B7000F8B50B4E070030000D0004F0EBFA04001E
:103B8000A84200DD2C003D00EB1B9C4205DD30000F
:103B900004F0EAFA28700135F6E72000F8BDC046C7
:103BA000C81B002010B50100014804F093FA10BDB5
:103BB000C81B002010B5054C200004F099FAE12143
:103BC0002000490204F07EFA10BDC046C81B002048
:103BD000C3070CD4064B1B68834208D8054B1B68EF
:103BE000984204D8031F1B68002B00D018007047B0
:103BF0000C060020080600200023012210B50A4808
:103C0000990001334250642BFAD1084C084B002133
:103C10001A602000074A08F019FC074B074A636046
:103C2000074B1A6010BDC046982D002010060020DA
:103C300008000020D40900003027000014060020EE
:103C40000406002010B5044B044A1A60044B054AD0
:103C50001A60FFF7D1FF10BD0C06002010060020EF
:103C600008060020E40F0020044B1B6818680009B8
:103C700080B20238C343DB171840704704060020A7
:103C800000B59BB00200054901A808F023FF01A878
:103C900002F09CFA02F04CFDFCE7C0460AE000008E
:103CA0000B4BC20704D4042804D80A4B00D00A4B9B
:103CB000180070470F2203681A40031D042AF7D02A
:103CC000064B092AF4D0064B032AF1D0054BEFE747
:103CD000E4DF000000DB0000FADA0000EEDF0000A5
:103CE000FEDF0000F5DF00000020064A0649131F32
:103CF000186013681B099BB202339B00D2188A42DA
:103D0000F5D3704714060020E40F0020F7B50F2408
:103D10000126314B314A1968314B324D186813680E
:103D20001F002740072F26D813681B099BB20233B8
:103D30009B00D218AA42F2D300242B4EA500AD1945
:103D40002868FFF745FF01342860642CF6D1274C22
:103D50002068FFF73DFF2060254C2068002802D036
:103D6000FFF736FF20600025224B1B680093009B65
:103D70009D4214DBF7BD1B099BB29B00D3189A42EE
:103D8000D2D01F68374208D1B94206D2B84204D314
:103D9000043F3F68002F00D01F60043BEFE7F02393
:103DA0006B43154A9B181A78002A01D10135DEE7CA
:103DB0001F693C2300266B43DB199B0001930136EE
:103DC000BB1BF3D4019BB4001C1B0B4B1C19A0693B
:103DD000FFF7FEFEA061F2E70C06002014060020AB
:103DE00008060020E40F0020982D00200800002085
:103DF000E40F0020D8050020401C0020F7B5012466
:103E0000204246D1234B1B689C46984241D3224B0B
:103E10001B68019398423CD8031F1B68002B38D1C4
:103E20000200036800941B099BB2002B0FD100997C
:103E3000131F196090422CD015682B1F1B68990026
:103E400069180C68013B14600A602A00EDE79D00C8
:103E500055192968009C214219D18C4517D8019C1D
:103E60008C4214D30E1F3468002C10D10F680F340D
:103E70003C40072C08D92F60151F2B600B680A6087
:103E80001B099BB20A00D0E700993160CDE7013BE6
:103E9000CBE7F7BD0C060020080600200D4970B5E1
:103EA0000A000D4D1368141F1B0926689BB2981C4D
:103EB000002E0BD000238A4200D00B002360830029
:103EC000C91880001218AA42ECD370BD1B01136000
:103ED000F7E7C04614060020E40F0020F8B5124CA6
:103EE00027000F223B681D09ADB213420DD06E1C96
:103EF000B600A74204D032003900200008F093FA3F
:103F00000022A3190436A4191A600235AD00074B2C
:103F10007F199F42E5D31B1B9B10013B1B012360B4
:103F2000034B1C60F8BDC04614060020E40F0020BF
:103F300004060020F0B59BB0FFF738FC0024070012
:103F4000214AA300D0580134FFF758FF642CF7D161
:103F50001E4B1868FFF752FF1D4B1868002801D050
:103F6000FFF74CFF00261B4B1B689E4217DBFFF739
:103F700095FFFFF7CBFEFFF7B1FFFFF717FC164BDE
:103F8000C21B1B6815491B6801A81B099BB2023B99
:103F900008F0A0FD01A802F019F91BB0F0BDF02552
:103FA00075430F4BED182B78002B01D10136DAE762
:103FB0002B695C1E002CF9DBA300EB189869FFF756
:103FC0001DFF013CF6E7C046982D002008000020A8
:103FD000E40F0020D805002004060020C4DF000004
:103FE000401C0020F7B5174D4F1C2B6806001B68BE
:103FF0000C001B099BB201929F420BDBFFF79AFF5B
:104000002B681B681B099BB29F4203DB0A20FDF74C
:1040100079FBFEBD2868A71CBA00DB1B81181B01B9
:104020000B6029600021031F19600F231E4003004D
:104030002401264340C3083A9A189A42E9D90199C3
:1040400002C3FAE704060020F7B50300012213407B
:1040500004000D000193002B2BD1174B1B688342EA
:1040600027D8164B1B68834223D90F23144F38607F
:1040700000681840FFF7B6FF019B3C68061E3B60D6
:1040800017D0236804301B099BB29D4200DD1D0040
:10409000AA00211D251F08F0BDF9FFF725FE2E609F
:1040A000FFF734FE00232B602268064B1340236089
:1040B00034002000FEBDC0460C060020080600208B
:1040C000E40F0020F0FF0F000323043010B5C117E8
:1040D00019400918891000220420FFF783FF10BD42
:1040E00070B5050008000C00FFF7EEFF0023002864
:1040F00004D170BDE95CC21811710133A342F9DB30
:10410000E343DB171C40002304192371F1E7F0B5EA
:104110000C009BB0022804DC1C20FDF7F3FA1BB056
:10412000F0BD01230868184206D1042804D90F26DF
:1041300001683140042901D00E20EEE761680D00CE
:104140001D40F9D10429F7D90A683240042AF3D175
:10415000A2681A4201D10D20DFE7FFF7A1FD06009A
:104160006068FFF79DFDA768010001AC7F1030007B
:10417000257003F0D1FB39006423220003F031FCE9
:10418000200008F0EDFC01002000FFF7A9FFC6E7C2
:1041900010B51C4CA544041E02D1FFF795FF0BE09F
:1041A00003F0D2FA0138062828D805F077FF09096C
:1041B00011182904240000208023DB009D4410BD39
:1041C000200003F03DFB011B2000FFF789FFF3E710
:1041D000200003F0E3FA430001201843ECE78022BB
:1041E0006946D200200003F0F0FA684608F0B8FCF7
:1041F00001006846E9E704210348E6E70020CCE730
:104200000420D9E700FCFFFF50E0000070B50C006F
:10421000022803DC1C20FDF775FA70BD0123086835
:10422000184206D1042804D90F2501682940042921
:1042300001D00E20EFE761681942FAD10429F8D9BC
:104240000A682A40042AF4D1A2681A4201D10D203A
:10425000E1E7FFF725FD05006068FFF721FDA46891
:1042600001006410280003F057FB210003F094FBC9
:10427000FFF78EFFD1E770B50D00012803DC1C208D
:10428000FDF740FA70BD01240868204206D10428D9
:1042900004D90F2102680A40042A01D00E20EFE75A
:1042A0006A682242FAD1042AF8D913680B40042B19
:1042B000F4D1FFF7F5FC06006868FFF7F1FC010098
:1042C000300003F029FB03F0ABFB40002043D9E7AB
:1042D000F8B507000C001C20012F0BDD0125086834
:1042E000284206D1042804D90F2102680A40042A72
:1042F00003D00E20FDF706FAF8BD62682A42F8D115
:10430000042AF6D913680B40042BF2D1FFF7C8FC3E
:1043100006006068FFF7C4FC0100022F14D0A468F7
:104320002C4211D06410300003F0F6FA050003F0BF
:104330000BFA012811D1002C02DD0135012C06D128
:104340002800FFF725FFD7E701246442EBE72800A8
:1043500003F083FA013C0500F0E70228F0D1002CBD
:10436000EEDD0135012CEBD000222800110003F016
:10437000A6FA03F072FA013C0500F3E710B5012438
:104380000868044016D04410200006F0AFF9154923
:1043900006F07AF807F060FF04F0B2FB0022124B3F
:1043A00007F014F904F054FB07F0E6FE4300012087
:1043B000184310BD042810D90F2302681340042BA2
:1043C00007D1FFF76DFC21000A2208F091FC0400E0
:1043D000DAE7032B01D10430F5E70D20FDF792F960
:1043E000D2E7C046D30237390000D040086870B524
:1043F00001240500254006D1042804D90F230268B2
:104400001340042B03D00E20FDF77CF970BDFFF79D
:1044100047FC03782900233B5A4253411022C0181D
:1044200008F066FC80239B05C218044B9A4201D910
:104430001420E9E740002043E8E7C046FFFFFF3FC4
:1044400010B5034A0621034801F030FC10BDC046F8
:1044500020E000001BE000000020704710B51E2087
:10446000FDF750F910BD10B51E20FDF74BF910BD3A
:1044700010B51E20FDF746F910BD10B51E20FDF742
:1044800041F910BD10B51E20FDF73CF910BD10B567
:104490001E20FDF737F910BD10B51E20FDF732F9CB
:1044A00010BD10B51E20FDF72DF910BD10B51E2052
:1044B000FDF728F910BD10B51E20FDF723F910BD3A
:1044C00010B51E20FDF71EF910BD10B51E20FDF71A
:1044D00019F910BD10B51E20FDF714F910BD10B567
:1044E0001E20FDF70FF910BD10B51E20FDF70AF9CB
:1044F00010BD10B51E20FDF705F910BD10B51E202A
:10450000FDF700F910BD10B51E20FDF7FBF810BD3A
:1045100010B51E20FDF7F6F810BD10B51E20FDF7F2
:10452000F1F810BD10B51E20FDF7ECF810BD10B568
:104530001E20FDF7E7F810BD10B51E20FDF7E2F8CC
:1045400010BD000010B5034A1821034801F0AEFB6E
:1045500010BDC0468CE000004CE100000120034B80
:104560001860034B1B6883401843704700100020FD
:10457000E80F0020F0B5EFF310810123194083F319
:104580001088134AA1261268124D013A9340A022C6
:10459000114FD205F600002B17D02C68945103421E
:1045A0000BD0C046C046C046C046C046C046C04606
:1045B000C0462C68D4515B08EDE7D451C046C046D4
:1045C000C046C046C046C046F5E781F31088F0BD3E
:1045D00020000020F40F00200C05000030B585B04D
:1045E00001AD0C220649280007F014FF0024285DC5
:1045F00001210134FFF7FAF80C2CF8D105B030BDD9
:1046000088E20000F7B56A463B4B01AE13800A23EF
:1046100093703A4B33801C23B370FFF7C7F8384BC5
:10462000384DC0182B68984201D200232B602C68AB
:10463000002C41D1375D01213800FFF7D7F8013454
:104640000021380004F038F9032CF3D100240127AD
:104650006B461E5D39003000FFF7C8F801343900A1
:10466000300004F029F9032CF2D1C8200138C046EB
:10467000C046C046C046C046C046C046C046C0460A
:10468000C046C046C046F1D16B4600211878FFF7FE
:10469000ADF86B4600215878FFF7A8F86B4600216B
:1046A0009878FFF7A3F8FFF781F8FA2300241B019D
:1046B000C01828602000FEBDFFF778F82B680024A2
:1046C0009842F7D3032003F087FF0600042003F08D
:1046D00083FF36180A2003F07FFF0B4B9B1B181A31
:1046E0000A4BA04206DB18600023094A2B601360C6
:1046F0000124DFE71C60F7E7030400001A1B000039
:1047000010270000F80F0020E3030000E80F00204E
:10471000001000200022054B10B51A60044B1B68E6
:10472000934201D002F0B0FF002010BDFC0F00202A
:10473000EC1A002010B5041E0CDA0024084BA4006B
:10474000E2581F231A401E3B9340064A1360064A54
:10475000136010BDFFF748F8A042EEDDEEE7C0465B
:1047600074F00000F40F00201805005002000868E3
:1047700010B5C3070FD540101823012A03DD4A687E
:10478000042A00D10833054A1360FFF753F8FFF7F6
:10479000D1FF002010BD01204042EDE720000020A5
:1047A00010B50124044002D04410200010BD04289C
:1047B00010D90F2302681340042B07D1FFF770FABA
:1047C00021000A2208F094FA0400EEE7032B01D13D
:1047D0000430F5E70D20FCF795FFE6E70868F8B52B
:1047E000C3071AD5FFF7DCFF0300203B5E2B25D85B
:1047F0000520434301221D180020114E9D4219D06F
:1048000005211024F75C3C4200D080180139520089
:1048100064100029F7D10133F0E704280ED90F22E4
:1048200003681A40042A09D11B099BB2002B05D04A
:104830000379DAE7012340001843F8BD0120FCE7C3
:1048400094E2000070B508680D00FFF7A9FF0400AE
:104850006868FFF7A5FF621E0100042A14D8451EF0
:10486000042D11D805236B439B18012215009D4090
:104870002B00064805682B430360054B1B68002B83
:1048800002D0200002F001FF002070BDFC0F0020CC
:10489000EC1A002070B508680D00FFF781FF0400D6
:1048A0006868FFF77DFF621E0100042A13D8451EC9
:1048B000042D10D805236B439B1801229A4007480A
:1048C000036893430360064B1B68002B03D0002250
:1048D000200002F0DAFE002070BDC046FC0F002070
:1048E000EC1A0020F0B5050089B008680C00FFF74D
:1048F00057FF0690022D36DD6068FFF751FF0190EB
:10490000A068FFF74DFF04000127231D661E0793D3
:10491000731C0293079B9E4235D005237343059376
:10492000019B019D05330493049BAB421ED0042ED2
:1049300016D86B1E042B13D80122059B2349013B7B
:104940005B199A409446224A0B681068069A3A40CE
:1049500003920DD062461A430A60012200280DD14D
:104960007F000135E0E701240194CDE7029ECFE707
:10497000624693430B600028F2D0039A0299280004
:1049800002F083FEECE7019B1E1D042E1AD8012CB9
:1049900018D1002505273B0021006B439B19994046
:1049A0000B000A4A013511689943094B11601B68D5
:1049B000002B05D0019B0022581D290002F065FE46
:1049C000052DE8D1002009B0F0BDC046FC0F002045
:1049D000EC1A0020F0B53B4B85B01B680C00002B97
:1049E00003D101204042FFF7A5FE012627683E4083
:1049F0003CD1042F3AD90F233A681340092B35D103
:104A00007B685B100293029B9E4258DAB300FB184E
:104A10009868FFF7C5FEFF23050004140012184034
:104A20001C4029492B404043019305F0CBFB030474
:104A3000200025496043039305F0C4FB039C00025A
:104A4000044301982049404305F0BCFB1F4B204321
:104A50001B68202B06D1AD00AD0E1D4BAD00EC58F0
:104A600000022043FFF786FD0136CCE73800FFF750
:104A700097FEFF26050007140012304012494043FC
:104A800005F0A0FB3740040438000F49784305F0D7
:104A900099FB2E400002044330000B49704305F09F
:104AA00091FB0A4B20431B68202B06D1AB009B0EC9
:104AB000074A9B009B5800021843FFF75BFD00204C
:104AC00005B0F0BDF40F00205906000020000020C2
:104AD00070E40000086810B5C30703D5FFF760FE57
:104AE000054B1860054B1B68002B03D0024B186860
:104AF00002F0CCFD002010BDFC0F0020EC1A0020BD
:104B00007FB5A04C2368002B0AD19F4A1268002A67
:104B100006D19E4B1B68002B01D0FFF773FD7FBDB4
:104B20009B4D2A68002A26D1984A1268002A1BD079
:104B3000FFF768FD0028F2D0FFF750FD924B246884
:104B40001A681C60002A16D0002C14D101AD0C226A
:104B50009049280007F05EFC285D00210134FEF733
:104B600045FE0C2CF8D1DAE7874A1268002AE5D115
:104B7000002BE3D0E0E700211A2003F09DFE002186
:104B80001B2003F099FE00211C2003F095FE2E68E7
:104B9000012E5CD0022E00D1A2E0002E50D10136B1
:104BA0003100794C03202368994303F085FE0420EB
:104BB000216801404B42594103F07EFE10212368D9
:104BC0000A2019404B42594103F076FE80212368A8
:104BD000090119404B425941062003F06DFE802126
:104BE0002368090219404B425941072003F064FE33
:104BF00080212368490219404B425941092003F0A2
:104C00005BFE80212368890219404B4259411920DB
:104C100003F052FE80212368C90219404B425941DA
:104C2000182003F049FE802321681B0319404B42E2
:104C30005941172003F040FE31001A2003F03CFEDA
:104C40002B680321581C05F0A3FB296067E70221AC
:104C50004D4C1720236819404B42594103F02CFE5C
:104C600008212368182019404B42594103F024FEC3
:104C700080212368C90019404B425941042003F0A8
:104C80001BFE80212368490119404B4259410A20EB
:104C900003F012FE80212368C90119404B4259419B
:104CA000032003F009FE80212368890319404B4249
:104CB0005941092003F000FE802321681B0419409C
:104CC0004B425941192003F0F7FD3100062003F053
:104CD000F3FD3100072003F0EFFD31001B20ADE7AD
:104CE0002021294C1720236819404B42594103F0D9
:104CF000E3FD40212368182019404B42594103F03D
:104D0000DBFD80212368192019404B42594103F0F3
:104D1000D3FD80212368490019404B4259410920A5
:104D200003F0CAFD80212368890019404B42594194
:104D3000072003F0C1FD80212368890119404B42FF
:104D40005941062003F0B8FD80212368490319402A
:104D50004B4259410A2003F0AFFD80212368C9036B
:104D600019404B425941032003F0A6FD80232168DE
:104D70005B0419404B425941042003F09DFD012181
:104D80001C205BE7FC0F0020F00F0020001000202B
:104D9000EC0F002088E20000012010B54042FFF730
:104DA000C9FC10BD10B5034A0921034800F07EFF7D
:104DB00010BDC04670E50000B8E500008023F0B5E6
:104DC00002255B051A690A4C0A4BA1261D510327CF
:104DD0008025F600ED00BA43884202D300221A5122
:104DE000F0BD5F59002FFCD098518018F4E7C04601
:104DF0000405000000E0014010B5002806D1C020E5
:104E0000B02140028902FFF7D9FF10BDB0208021F8
:104E10008002C902F7E7000043425841064B404276
:104E20001840B0239B02C018036800201A0E532AB2
:104E300001D11B02180A704700C0FEFF30B50124E3
:104E40008025054B054AED009C505C59002CFCD098
:104E500001600021995030BD00E0014004050000D0
:104E600043425841074B40421840B0239B02C018B0
:104E7000A62310B50902DB05090A1943FFF7DEFF77
:104E800010BDC04600C0FEFFF0B5012480260D4BCA
:104E90000D4DF6005C51002902DC00225A51F0BD94
:104EA000577814783F022743947824042743D47812
:104EB000043224063C439F59002FFCD010C0013916
:104EC000E9E7C04600E001400405000070B50500B8
:104ED0004B680A009C1C2100A400FFF7D5FF28198D
:104EE00070BD0000134B1B68002B0CD08022B02338
:104EF000D2029B0200280BD11A1D5B681B0E522B9D
:104F000000D110007047B022C02392025B02F1E78B
:104F100082420DD903681B0E522B09D1436802331C
:104F20009B00C018824203D903681B0E522BE9D0A4
:104F30000020E7E704110020F0B50020B7B00024FE
:104F4000FFF7D0FF270005002600002D2ED1284DA9
:104F50002868FFF761FF32003B000190009425496B
:104F600004A807F0B7FD04A801F030F9224B642033
:104F70001C682B68A0215A425341204A5B421340CF
:104F8000B02292029B18E41A6043490205F01AF914
:104F9000A0225202030000921949220004A807F03F
:104FA00099FD04A801F012F937B0F0BDFF226B683B
:104FB00029689C460233FF180B12013613409C42AD
:104FC00000DA1C00FF200A140240039262460140EE
:104FD00001920091039A0B4904A807F07BFD04A8F5
:104FE00001F0F4F82800FFF77DFF0500ADE7C046AB
:104FF00004110020C2E600000811002000C0FEFFDE
:105000006CE60000AEE6000070B50020FFF704FF7C
:1050100004000120FFF700FF844200DA04000A4B7D
:105020001D686A42554128001D60FFF7E5FEA02279
:105030006B4252021340054A28009B18044A611C27
:105040001360FFF70DFF70BD041100200480010004
:1050500008110020F8B50020FFF7DEFE0700012050
:10506000FFF7DAFE3E00204D0643204C0DD1802193
:10507000C020C9024002FFF7A1FE01213000FFF766
:10508000EFFE1B4B2E6023601DE0874209DD0023ED
:10509000B0212B60164B8902236023680020012574
:1050A00017E0012380212B60124BC9022360F4E733
:1050B000120E522A08D0002800D023600E4801F0BA
:1050C00085F8FFF7A1FFF8BD28005A680232920068
:1050D0009B188B4205D21A68561CE9D10028F2D0E1
:1050E000D1E72160EFE7C04604110020081100203D
:1050F0000480010004C0020087E6000070B50020B3
:10510000FFF7F0FEFF260500002801D1280070BD42
:1051100003681C143440FFF7E5FEDA2CF4D10500D7
:10512000F2E70000FF2270B5134CD20000212000EE
:1051300007F08CF9FF25FFF7E1FF0026002800D1DA
:1051400070BD03681A142A400A2A0AD11A122A408A
:10515000FF2A03D0D200A1180B71A050FFF7C2FEA6
:10516000ECE7132AFAD11B122B40FF2BF6D0DB0001
:10517000E2181671E650F1E7A025002010B59AB0AC
:10518000FFF768FFFFF7CEFF00231A000A48D90097
:10519000415801334C1EA1415218FF2BF7D107494A
:1051A00001A807F097FC01A801F010F8044801F0ED
:1051B0000DF81AB010BDC046A0250020F7E600008B
:1051C0000BE700008022F0B55200A1B00021684832
:1051D00007F03CF9802200215200664807F036F9BA
:1051E000654BFF271B681A00049353425A41100075
:1051F0000592FFF701FE049C0020631E9C415F4B5B
:1052000064421C405E4BE418FFF778FF0600002E56
:105210002FD10498FFF700FE411C0598FFF720FEF0
:10522000059A554B574D1A602C60FFF77BFFFEF730
:10523000C1FC514B64201B68A0215A4253414F4A84
:105240005B421340B0222C6892029B18E41A604320
:10525000490204F0B7FFA0225202030000924A491B
:10526000220007A807F036FC07A800F0AFFF21B026
:10527000F0BD3268131412123A403B4003921A00F8
:105280000A3A092A49D83A4B039A995C002931D144
:1052900010223E4807F0DAF835002B6803991A12FD
:1052A0003A40914209D11A143A400B2A27D0132AC6
:1052B0002DD00A2A01D1354B1D602800FFF712FEC0
:1052C000051EEAD1314B196800290FD02000FFF7E5
:1052D000FDFD04002D4B5B195968002903D0200007
:1052E000FFF7F4FD040004350C2DF3D1204B012110
:1052F000039A99543000FFF7F5FD060087E73B401D
:10530000022BDADC214A9B00D3185D60D5E710221E
:1053100000211E4807F09AF8CFE71A00153A082A2C
:10532000E8D8144A0399525C002AE3D13500152BC2
:1053300000D01500300003681A143A40152A0FD027
:105340001D2A00D10025FFF7CDFD0028F3D1002D47
:1053500004D020002900FFF7B9FD0400054BC6E783
:10536000039A1B123B409A42EDD10500EBE7C04681
:10537000041000200C1100200411002000C0FEFFCA
:1053800004C002000811002051E60000282F002070
:1053900010B5FFF717FF10BDF0B585B003920322DB
:1053A0000333DC17294D1440E4182B68284F5A4268
:1053B000534180225B42D202A4103B409B18A21CA6
:1053C0000291244E910000910190316800980A18D2
:1053D000934215D2FFF7F6FE2B685A4253418022C2
:1053E0005B421F40D202BF183368009A9B189F424D
:1053F00006D2194800F0EAFE0025280005B0F0BDED
:10540000029B356819066B461A7BA423DB05134300
:10541000FF222F00090C1943019B12041B041340A7
:1054200019432800FFF70AFD0837281D21003760BF
:10543000FFF704FD002C04D00A9A21003800FFF782
:1054400023FD009B083BFF183760D6E704110020BE
:1054500000C0FEFF081100202BE600000021094BD0
:10546000094A59600131516059680029FCD0002176
:105470001961012393600222044B8131FF315A509C
:105480001A607047FC1000400010004000E100E08E
:105490000222064B0121DA670022054B5A61054AB8
:1054A00011615A69002AFCD07047C04604E100E04F
:1054B000FC1000400010004010B5044C2378002B75
:1054C00001D0FFF7E5FF0020207010BD0D12002075
:1054D000802301205B055B6E5B0018437047000072
:1054E0000120024B1B685B0018437047901200209C
:1054F0000120024B1B685B0018437047240000200A
:105500000120024B1B685B00184370479412002077
:1055100070B504000D001600FEF752F9802301213A
:105520005B055A6E2670002653006170E17062724E
:10553000010A5A0A6071A171A272010C5A0C000E84
:105540005B0EA6702571E1712072E272237370BD4B
:1055500010B5044C200007F003FB01002000FEF70B
:10556000BFFD10BD991200200E4B10B51B680E4CEC
:105570005A1C0FD00D4C002B0CD00D4C012B09D018
:105580000C4C022B06D0094C042B03D00A4C052BE3
:1055900000D1074C200007F0E3FA01002000FEF7DD
:1055A0009FFD10BD280000209CE70000A0DE000049
:1055B000A7E70000A7DE0000A1E7000070B5214CBE
:1055C0002278002A3DD1204B01215A608022D20549
:1055D00011605A68002AFCD0002207201B4B1C498E
:1055E00001255A500439585008315A5019481A495F
:1055F00058501A491A485A501A495A50A622D200ED
:105600009D50082218495A50043158500220174919
:1056100058501749174858501748043958501820FF
:1056200016495850C12189005A500539FF39585838
:10563000921802435A501249124A9950FFF70EFF2E
:10564000257070BD0D120020FC00004000100040CD
:105650000C050000746962751C050000240500003B
:10566000200004022C050000140500003405000091
:105670003C050000FFFF0000211001005405000060
:105680000E1200200405000070B50E4B06001B78BA
:10569000002B01D1FFF792FF00200B4D2C788442A4
:1056A0000ED00A4B202219780323091B1940084BFE
:1056B0004901C918300006F0ADFE0120013C2C70F4
:1056C00070BDC0460D120020981200200C12002060
:1056D0000E120020002370B588B0984235DD0D68A9
:1056E00001262C0034409C422FD12300042D2CD9BC
:1056F0000F222B681A402300092A26D16A683F2A04
:1057000023DD6846FFF7C0FF230000281DD06B464D
:1057100019783300A14203DB6B461B5D5B0033430A
:10572000A200AA1801349360202CF2D10921694407
:105730004A780B7812021A438B781B041A43CB78F1
:105740001B061343024A13600423180008B070BDFF
:105750009412002070B5454B8AB01B78002B01D104
:10576000FFF72CFF02AC2000FFF78EFF002802D1CC
:1057700000200AB070BD23780B2BF9D96378012B78
:10578000F6D1E378012BF3D100231120384E394DA7
:1057900033602B7068442379374A4178136002786C
:1057A00009021143827812041143C27812060A4397
:1057B00032490A60002B0ED1152169444A780B78D2
:1057C00012021A438B781B041A43CB781B0613432F
:1057D0003360002318E0012B1AD1152169444A785F
:1057E0000B7812021A438B781B041A43CB781A21C8
:1057F0001B06134333600E23627C6944934200DD31
:10580000130000229A422CD100220420EA54B0E76F
:10581000022B03D1627B10331621EEE7042B0DD14E
:10582000152108226944684606F0F4FD00980199A4
:1058300003F07EF806F0A0FC3060CAE7052BC8D163
:10584000152108226944684606F0E4FD0098019994
:1058500003F06EF806F090FC3060627D0A231E2192
:10586000CBE7885CA8540132CCE7C0460D1200207B
:10587000901200209912002028000020941200208D
:1058800010B5134B04001B78002B01D1FFF796FED7
:10589000FFF7FEFD00200F4A0F49104B545058608F
:1058A0000130106058680028FCD0002018610130D9
:1058B000906018690028FCD0094B0A481B785B01EE
:1058C0001B185350FFF7E4FDFFF7C8FD10BDC0469D
:1058D0000D1200200010004004050000FC100040E4
:1058E0000C1200200E12002010B588B000281DDD1B
:1058F0000A68012113000B4018D1042A16D90F2081
:1059000014682040092811D150683F280EDD980006
:10591000101880680024084201D04010C4B26846C4
:10592000C4540133202BF2D1FFF7AAFF002008B0A6
:1059300010BD000010B5002813DD0C68E30710D57A
:105940006410532C0DD8084B1B78002B01D1FFF7A6
:1059500035FEFFF79DFDA123044ADB00D450FFF77D
:105960007DFD002010BDC0460D120020001000403B
:1059700010B500280EDD0C68E3070BD56410FF2C72
:1059800008D8054B1B78002B01D1FFF717FE034AFF
:10599000034BD450002010BD0D1200200010004019
:1059A0002405000013B5002814DD0C68E30711D5A9
:1059B000094B64100093094B0193072C0AD8084B3C
:1059C0001B78002B01D1FFF7F9FD6B46054A1957EB
:1059D000054BD150002016BDE2ECF0F4F8FC0004B9
:1059E0000D120020001000400C05000070B588B0BA
:1059F000002820DD0124086804401CD104281AD99D
:105A00000F2302681340042B15D1FEF749F9060055
:105A100007F0A6F80500122800D912252A00022155
:105A20000D326846FFF774FD6B465D73A54205DCD9
:105A30006846FFF725FF002008B070BD2300325DE7
:105A40006B449A730134F1E7F0B50D008BB0012877
:105A500032DD08680122040014402DD104282BD91E
:105A60000F2301680B40042B26D16B68134223D00F
:105A7000FEF716F96E6807007310019307F070F8CF
:105A800005000E2800D90E252A000121113202A896
:105A9000FFF73EFD6A46127902AB5A7302AA7312EF
:105AA0009373019B76141B0ED67313745574A54221
:105AB00005DC02A8FFF7E4FE00200BB0F0BD3A5D64
:105AC00002A963189A740134F1E730B589B000284F
:105AD00014DD0C68E30711D5102268460021FFF79A
:105AE00017FD6B466A4665105D73684663122D0E9E
:105AF00064149373D4731574FFF7C2FE002009B0C9
:105B000030BD0000174B184A5968002903D0002106
:105B1000596001319160196900291FD00020186176
:105B20008023DB00D3581149012B18D1A923DB00B6
:105B3000D3585B420B600E490B78032B01D801331D
:105B40000B7003200B490B78013303400B700A499B
:105B50005B015B180949535001239360704708604B
:105B6000FAE7C046FC10004000100040240000206E
:105B7000981200200C1200200E12002004050000D4
:105B800010B5034A1021034800F090F810BDC0463C
:105B90001CE7000013E70000044A05491368C854D5
:105BA00001339B059B0D13607047C046C81600204B
:105BB000C812002070B5114C114A2368834202DCE0
:105BC0000023236016E0155C411C2E00FA3E012ED6
:105BD00005D899420FDA555C013D1F2D01D9080007
:105BE000ECE70100151A565C6E5401318B42FADC69
:105BF000181A206070BD1570FAE7C046D41A00204C
:105C0000D416002010B5FDF7D1FD064B1A6882426C
:105C100001D900221A601B68C31A034898428041C8
:105C2000404210BDC4120020204E000010B5094CA7
:105C3000094A23681268934200D110BD074AD05C1C
:105C4000FDF7B0FF0028F8D0236801339B059B0DBA
:105C50002360ECE7CC160020C8160020C8120020F4
:105C600010B50400064B074A1B6812689B1ADB43F9
:105C70009B059B0DA34200DB10BDFFF7D7FFF1E7AB
:105C8000C8160020CC16002070B5FFF737FAFF25A4
:105C90000400002801D1200070BD03681B142B40B4
:105CA0001D2B00D10400FFF71DF9F2E770B5074E78
:105CB00033680B2B08DC0C255D43054C0133285160
:105CC00064196160A260336070BDC046D0160020C8
:105CD000382F0020F0B5B7B0040006F041FF0128CE
:105CE00002D8002037B0F0BD23785B2BF9D1013802
:105CF00025182B785D2BF4D101343A21200006F0D1
:105D000017FF061EEDD0071B002FEADD210000243F
:105D10003A0004A806F03CFF04AB711CDC556F1A76
:105D2000A742DEDD1DAD3A00280006F031FF134B1F
:105D3000EC551B6803950193019BA342D1DD0C2612
:105D400066430F4B04A9F618306806F0FFFE051EE7
:105D500005D17368B6680293029B9D4201DB013452
:105D6000EAE73068039906F0F1FE370008360028AC
:105D700001D17868B6E70135EEE7C046D0160020BD
:105D8000382F002010B5FBF7F7FAFFF70BF8FBF7F9
:105D90001BFBFDF79BFEFEF753FBFEF7D3FBFFF764
:105DA000EFFE01F03FF801F045FC01F071FC01F05D
:105DB000BBFE10BD962210B512010021034806F06B
:105DC00045FB0022024B1A6010BDC046401C00205B
:105DD000D805002070B514007F22174BC000C058B2
:105DE0000D00836813401C2B01D0002070BDC368D8
:105DF000190011400429F8D101690A40192AF4D187
:105E00001B0A01339B000C30C018FDF749FF0378D3
:105E100006000120002BE9D0300006F0A1FE00238F
:105E2000A042E2D1A34201DB0120DFE7F15CEA5CA2
:105E30009142DAD10133F5E7A0250020064B074A4D
:105E40001B6812689B1ADB439B059B0D0122834252
:105E500000DC002210007047C8160020CC1600207D
:105E6000F8B505000C0016001F1E0ED10320FFF729
:105E7000E5FF002808D0FA20FFF78EFEE8B2FFF712
:105E80008BFEE0B2FFF788FEF8BD501DFFF7D6FF8E
:105E90000028F9D0FB20FFF77FFEE8B2FFF77CFE79
:105EA000E0B2FFF779FEF0B2FFF776FE3012C0B233
:105EB000FFF772FE3C00E31B9E42E5DD2078FFF712
:105EC0006BFE0134F7E7000070B50024F0250B4BA2
:105ED0001B68A34202DCFFF76DFF70BD2B0063431C
:105EE000074A9B181A78002A05D0597800231120F8
:105EF0001A00FFF7B5FF0134E9E7C046D8050020D6
:105F0000401C0020F8B507000024F0252B00634357
:105F10000C4A01349E18B74211D0317800290BD0B9
:105F20000133D15C002311201A00FFF799FF2A00EA
:105F30000021300006F08AFA0A2CE7D1F8BD024BA6
:105F40001C60F9E7401C0020D8050020F0B51500C2
:105F500001222F007A4C1740A54401900291002F96
:105F600011D005AB1A706A105A70120E1A71052200
:105F7000691299706D140299DD70FFF771FFCF23DC
:105F80009B009D44F0BD042D2AD90F2428680440AD
:105F9000042C32D1022304AA28001371FDF780FEDD
:105FA000050006F0DDFDC82302009B00984200DDDD
:105FB0001A007C1C97420DD1984206D9614804AB67
:105FC00003226149C01806F025FA220005AB0299A8
:105FD0000198D2E72700611E695C05ACE155E8E74E
:105FE000042D00D0A7E0032304AA043D13716B42E3
:105FF0005D4105AB55710222E9E7092C7ED10422EF
:1060000005AB1A706A6851100091694652120978FE
:106010009A70009A59701F2A01DD202200926A4668
:10602000127806ACDA70009BBB4202DC05ABE21AC8
:10603000CDE70126BB00EB189868064006D104287E
:1060400037D90F210368194002290CD1012323708D
:106050004310637042121B0E4014A270E070237153
:1060600005340137DFE7042921D102232370FDF72E
:1060700017FE039006F074FDA31C0C2809D860706D
:10608000864201D19C19ECE7039A925D9A5501363C
:10609000F6E70C226270039A925D9A550136092E3A
:1060A000F9D12E23E372237363730E34D9E70129E8
:1060B00007D10323043823704342584160700234EF
:1060C000CFE7092909D10423237043685A1062706D
:1060D0005B12A370E6700434C3E703290BD10523D8
:1060E00023700068020992B2430F92000B40D31A4A
:1060F00063701B12EDE726700134B2E7032C00D069
:106100003DE7052205AB01091A7089B2420F8900EB
:1061100022408A1A11125A709970642A00DD642292
:106120000421DA70081F824201DC04324FE7685C08
:1061300058540131F6E7002D00D020E753E7C04660
:10614000C4FCFFFF220300000ADB000070B5020060
:106150000024F0210D4E08006043801945789542D7
:1061600003D001340A2CF6D170BDF022002106F0D4
:106170006DF9074A1368013BA34200D11460002364
:1061800029001A001120FFF76BFEEDE7401C0020EC
:10619000D805002010B5B2B002236A46040013707F
:1061A00006F0DEFCC72800D9C7200023984207DC90
:1061B000421C6B46FE211420FFF752FE32B010BD88
:1061C000694601335A1EA25CCA54EFE730B5B3B03A
:1061D00002236A460500137006F0C2FC0400C728BB
:1061E00000D9C72400239C420BDC20003230FFF78B
:1061F00037FD621C6B46FF211420FFF731FE33B0E0
:1062000030BD694601335A1EAA5CCA54EBE7000050
:10621000F0B5BDB005900C00012803DC1B20FBF796
:1062200071FA55E02C4B08680393C30709D404287E
:1062300007D90F2302681340042B02D1FDF730FD6C
:106240000390254B60680493C30709D4042807D939
:106250000F2302681340042B02D1FDF721FD0490A7
:1062600000261E4B1B680893089BB3420BDC049B63
:106270001B4A0093C821039B0AA806F0F9FB0AA851
:10628000FFF7A4FFCAE70C257543164B0399ED18D9
:10629000286806F05BFC071E05D16B68AD680993A2
:1062A000099B9F4201DB0136DEE7286804990795C8
:1062B00006F04CFC0835069000280BD1210005980B
:1062C000079B08315B6802389847074B069A1A60AB
:1062D0003DB0F0BD0137E3E71AE00000D016002022
:1062E00078E80000382F0020E40F0020F7B5234B9A
:1062F00006001B68F02100930023009A9A4211DCEB
:106300000024F0231A006243019201991C4A551897
:106310002F78002F12D001340A2CF3D11948FFF73F
:1063200055FF29E00A005A43154882185078B042B8
:1063300002D11278002A1FD10133DEE7F0223900A2
:10634000280006F083F802230D4A0199EB605354AC
:106350000D4AF1008A58009B6E70AE70AA602F61E2
:106360006F61A34202DC054B01341C600023310045
:106370001A001020FFF774FDF7BDC046D8050020B5
:10638000401C0020C1EC0000A025002010B5FFF744
:106390009BFDFF24084AE3005B429B18074AD35C3D
:1063A000043B012B03D8E043C0B2FFF79FFF013C41
:1063B000002CEFD110BDC046FC070000A025002036
:1063C000F8B505000E00FDF78BFEFF240D4B18609D
:1063D0000D4AE3005B429B180C4AD35C062B01D0AC
:1063E000032B0BD1E743FFB2320029003800FFF73F
:1063F000F1FC002802D03800FFF778FF013C002CA8
:10640000E6D1F8BD08000020FC070000A025002010
:1064100070B50500FF24084AE3005B429B18074A59
:10642000D35CAB4203D1E043C0B2FFF75FFF013C56
:10643000002CF0D170BDC046FC070000A025002054
:10644000F7B5FDF7B3F9574B1A68824201D900221C
:106450001A601A685449821A8A420DD9FF22534998
:106460001860D3005248CB1A1B181B78073B022B2D
:106470000CD9013A002AF4D1F7BD0720FFF7C8FF75
:106480004C4B27E00820FFF7C3FF38E0FDF798F9F1
:10649000071E00D101270020FDF746FA01900020D9
:1064A000FDF756FA019B0090434C444D002B12D04F
:1064B0002368002B6ED12B682760002B6ED0404BD9
:1064C00001261B78002BD8D10920FFF7A1FF394BFB
:1064D0001E703B4B1E70009B002B12D02B68002BB4
:1064E0000FD123682F60002B1ED0324B01261B7862
:1064F000002BC7D10920FFF78BFF2E4B1E70304BAE
:106500001E702368002B0FD02A4E3278002A0BD140
:106510009F4200D227602368FB1A312B04D9072041
:10652000FFF776FF012333702B68002B0FD0244E2A
:106530003278002A0BD1BB4200D92F602B68FF1A9A
:10654000312F04D90820FFF763FF0123337023683C
:10655000002B0CD0019B002B09D1164E3378002B59
:1065600002D10720FFF754FF0023236033702B680C
:10657000002B00D180E7009B002B00D07CE7104C63
:106580002378002B02D10820FFF742FF00232B6065
:10659000237071E7009A002AA0D1B5E7009B002B79
:1065A0009FD1AEE7C01200200F270000A0250020D9
:1065B000FC070000B4120020B0120020B812002026
:1065C000BC12002037B500240500FFF77DFC01A8B0
:1065D0000194FDF791F921002000FEF79BF8FEF7EA
:1065E0008FFAFDF7C9F9FDF74DFAFDF767FAFEF7E7
:1065F000D3FBFDF709F9A54204D0FDF7FDFA0248E7
:10660000FFF7E4FD37BDC046B2EC0000002310B533
:1066100001001A001120FFF723FC10BD07B56B46DF
:10662000197069465A7013128B701314120ECB70C6
:106630000A716B46010005221320FFF711FC07BD0C
:1066400010B50A0001001220FFF780FC10BD70B5E4
:1066500005000C00FDF7C2F8002809D020003230F8
:10666000FFF7FEFA2B00220000211B20FFF7F8FBAA
:1066700070BD10B50C000300110014202200FFF7BC
:10668000EFFB10BD012370B5FF24084A41185B429F
:10669000884201D3D84370BD06781D0A2340734059
:1066A0009B009B5801306B40F2E7C04694E8000025
:1066B00013B50400FE2813D80A4BC200D058002896
:1066C0000ED0436808309900FFF7DCFF01900920E5
:1066D000FFF7C6FA01AB042221001720FFF7C0FB29
:1066E00013BDC046A0250020F7B50190FFF7CCFAF6
:1066F00001250400FF276D42002C01D12800FEBDBA
:10670000266833143B40152B0DD121000198083128
:1067100006F01CFA002801D135123D402000FEF79A
:10672000E1FB0400E8E71D2BF8D101256D42F5E7F8
:10673000F0B58027A1B0FFF779FAB84CB84D2068C2
:10674000FF00391A4019FDF713FA23680600C31831
:106750002360002B0ED121B0F0BD2068391A281813
:10676000FDF706FA236806001B182360FDF71EF8E4
:10677000AC4B1860002EF0DC2B78FA2B00D014E123
:106780002368022B07DCFFF73DFA0028E3D0012045
:10679000FFF710FADFE76B78AC78981E182800D95D
:1067A000F8E003F07BFC0D2024282B34F73E707AB0
:1067B0007E94D3E4F7F7F7F7F7F7F7F7F7F7F20078
:1067C000FF2C0ED02000FFF7C1FC0022964BE10009
:1067D000CA505B181A712100009213001320FEF7B3
:1067E000DBFD0320D4E72000FFF780FDF9E7200060
:1067F000FFF7ACFCF5E7FFF7C9FDF2E7FFF764FB35
:106800000020FFF7DFFE8948FFF7E0FCE9E7632C93
:10681000E7D8874BA200D25821001520FFF796FB3E
:10682000DFE7FFF731FAFF270400002CD9D02568F5
:106830002B143B40152B04D02000FEF753FB040023
:10684000F3E72000083006F08BF906000530FFF76B
:1068500007FAFB20FFF7A0F92D121D20FFF79CF986
:10686000E8B2FFF799F9F0B2FFF796F93012C0B22B
:10687000FFF792F925002B1B9E42DDDD287AFFF7FA
:106880008BF90135F7E700211D2000910B000A006C
:10689000FEF782FDFDF7B0F9A3E72000FFF708FF40
:1068A0009FE7FCF79DFF07AC624A64210090624BB2
:1068B000200006F0DDF802232000237006F050F9D6
:1068C0002300020000211620FFF7CAFA89E75B4B7C
:1068D000FA21186803F076FC00260490524AF3006F
:1068E0009B181C68002C28D01B790593636808341A
:1068F0009F00B81D0393FFF7B3F9FB20FFF74CF996
:1069000001207D1CFFF748F9F0B2FFF745F9E8B226
:106910002D12FFF741F9E8B2FFF73EF90598FFF7AE
:106920003BF9E719A7420CD8FFF780F9049B0398BD
:10693000584301F0A1FDFFF779F90136FF2ECDD1C3
:106940004FE72078FFF728F90134EBE70024FFF741
:10695000BBFA2200210000942300DA20FEF71CFD80
:10696000FF222100D200304805F070FD92E7012C93
:1069700002D1FEF7E1FA34E7022C02D1FEF708FD5E
:106980002FE70120FFF71EFE2BE7002321001A004E
:106990001A2099E71A00C83A052A00D921E70022EF
:1069A00018001100FAF71CFD1BE7FB2B00D0EEE6E8
:1069B0002268042A00DCE6E62E79E878204B3602CD
:1069C00006439E4200DDE2E6331D9A4200DCDAE631
:1069D000EB5CFE2B00D0DAE66878AC78771E1B28DB
:1069E00000D17FE030D8072865D008283AD00128A8
:1069F0002FD1FF2C10D02000FFF7A8FB6D79114A92
:106A0000B31E009221002A000A20FEF7C5FC064BA7
:106A1000E400E0501B191D71701DB9E6D41A002066
:106A2000D4160020C4120020A025002094EC000001
:106A3000982D0020ABEC0000A6EC00000400002024
:106A4000F6030000DA1600201D285DD04FD31E2863
:106A500071D00300C83B052BDED8404A3900FAF755
:106A6000BFFCD9E7632CD7D86A79022A13D0032A4E
:106A70001BD0012AD0D1E979AB79090219432B7ACD
:106A8000A4001B0419436B7A1B060B435B001343E2
:106A9000334AA350C0E7002FBEDDB11E3148FDF7D9
:106AA0001FFB2F4BA400E050B6E7AB79A4005A1EA1
:106AB00093419B00ECE7632FAEDC07AD3A0027491A
:106AC000280005F0A7FC00232800EB55FFF70CFE7B
:106AD0000028A1DB224B8000C25821001520FFF7BF
:106AE00035FA99E739001D48FFF76AFC94E7FF2C57
:106AF00092D06A79022A8FD81A490B20009121007E
:106B0000B31EFEF749FC87E7632F00DD63270023F0
:106B100007A99F420ADCFB430022DB173B40CB184E
:106B20001A70152000917B1C2100EAE7EA185279BF
:106B3000CA540133EDE7012C00D06DE7002F00DCD3
:106B40006AE76B79002B03D01C00322B00DD322466
:106B500064235C43044B1C605EE7C046D9160020EA
:106B6000982D0020DA160020040000200122094B95
:106B70001A60094A1368002BFCD00322074B1B68DC
:106B8000D8171040C0180123801006384000184361
:106B90007047C04600C0004000C1004008C500402A
:106BA0000120704710B5064C200001F0D1F80549CE
:106BB000200001F001F90122034B1A6010BDC0460C
:106BC000101B0020801A0600D81A00201FB50021D3
:106BD0000E20FCF70BFE01210F20FCF707FE012120
:106BE0000D20FCF703FE1C4C200001F00FF81B4B9E
:106BF0001B4A1B6812681B49D2B28B420BD88023F8
:106C00009B04019301AB1A710199029A00232000A1
:106C100001F018F81FBD14498B4202D88023DB0411
:106C2000EFE712498B4202D880231B05E9E71049A0
:106C30008B4202D880235B05E3E70E498B4202D8E2
:106C400080239B05DDE70C498B4202D88023DB05BE
:106C5000D7E780231B06D4E7F01A0020300000207D
:106C60002C00002048E8010090D0030020A107007C
:106C700040420F0080841E0000093D0010B500282E
:106C800015DD01240B68234211D023410C4A136007
:106C90000C4AA04209D04B68234206D02341022B64
:106CA00009D0032B09D0A34203D002231360002094
:106CB00010BD0023FAE70323F8E71460F7E7C046A6
:106CC000300000202C000020F8B50125086828427B
:106CD00003D10D20FAF716FDF8BD4010FCF7AAFD10
:106CE000041E2DDBFCF780FDA04229DB00212000E3
:106CF000FCF77CFDFA222900D200200001F0EEFB17
:106D000000281DD0002500270726FA220121920025
:106D1000200001F0E3FB002812D0282802DD012327
:106D2000B3401F43013EF0D20D4EAF550135052D46
:106D3000E9D1012206210920FDF754F9002801D1EB
:106D40000020C9E70B23012443600023F25C990073
:106D500052004118224301338A60052BF6D1BBE76C
:106D6000DC1A002070B500281EDD0D68EB071BD46F
:106D7000042D19D90F242B681C40032C14D11A0997
:106D800092B25B0F92001C40141B2E00FFF71EFFF7
:106D9000731B06489C4205DD317900F059FF01362E
:106DA000F070F5E700F053FF002070BDF01A0020EE
:106DB00010B504680D20E30703D56410FF2C03D938
:106DC0001720FAF79FFC10BDFFF700FFE1B2044C5B
:106DD000200000F03DFF200000F039FF0020F2E726
:106DE000F01A002070B5FFF7F1FE064D00212800D3
:106DF00000F02EFF0400280000F029FF01206400AD
:106E0000204370BDF01A002010B5002001F0E4FB13
:106E1000800810BD10B5FFF7F7FF430001201843AD
:106E200010BD000010B5034A0E210348FEF73EFFD7
:106E300010BDC046D8EC000048ED00000D4B70B509
:106E40001B6804000E001500002B01D1FFF7AAFEFD
:106E5000E1B2094C200001F046F8F1B2200000F048
:106E600043FFE9B2200000F03FFF200001F0A6F848
:106E700070BDC046D81A0020101B002010B5012498
:106E80000368234205D04168214202D08268224231
:106E900003D10D20FAF736FC10BD5810802801D917
:106EA0001520F7E74910FF2901D91620F2E7521003
:106EB000FF2A01D91720EDE7FFF7C0FF0020EBE71D
:106EC000F7B501221400904226DD0D682A4223D036
:106ED0002D4B15411B684C68002B01D1FFF762FE5A
:106EE0002A4EE9B2300000F0FEFF270001221740D1
:106EF00014D01441FF2C02D91720FAF703FCE1B299
:106F0000300000F0F1FE300001F058F80024A042FB
:106F100002D02320FAF7F6FB2000FEBD042CF2D9A4
:106F20000F2523681D40092D1CD1636801925B1059
:106F30000093009BBB42E6DDBB00E3189D68019B0C
:106F40001D420BD06D10FF2D02D91720FAF7DAFB86
:106F5000E9B2300000F0C8FE0137EAE71720FAF77F
:106F6000D1FBF9E7032DCED127001A0992B25B0FAE
:106F700092001D40551B3B1B9D42C4DD39793000FA
:106F800000F0B2FE0137F6E7D81A0020101B0020EF
:106F9000154B70B51B6805000E00002B01D1FFF7E3
:106FA00001FE124CEDB22900200000F09CFFF1B26E
:106FB000200000F099FE0021200000F09FFF002833
:106FC00001D0404270BD72B601222900200000F0BD
:106FD00085FF62B6200000F078FE0028F2D0200085
:106FE00000F078FEEEE7C046D81A0020101B002003
:106FF00010B501240368234202D04168214203D125
:107000000D20FAF77FFB10BD5810802801D91520FC
:10701000F7E74910FF2901D91620F2E7FFF7B8FF7B
:1070200040002043EFE7000070B50D211D20FFF761
:10703000AFFF184C5A280CD101222A2122703D386A
:10704000FFF7FCFE022001F017FA0122124B1A6032
:1070500070BD0F211920FFF79BFF332805D10223B4
:107060008F22237020211A38EAE70D211E20FFF716
:107070008FFFC7280AD1032500222A21A9382570AD
:10708000FFF7DCFE2A002A211E20D9E70023237007
:10709000D8E7C04634000020E41A002010B50028CC
:1070A00003DC1C20FAF72EFB10BD01240B681C40EA
:1070B00001D10D20F6E75B10012B2BDD022B03D055
:1070C0000224042B00DD0134194B1B68002B01D175
:1070D000FFF7AAFF174B1B785BB2022B1CD0032BC8
:1070E0001ED0012B11D1032C00D1013C00222A21FA
:1070F0001D20FFF7A3FE22000E211D20FFF79EFE9C
:1071000001222A211D20FFF799FE022001F0B4F987
:107110000020C9E70024D7E7220123211920F2E744
:10712000032C00D1013C22000E211E20EBE7C046BB
:10713000E41A002034000020204B10B51B68040026
:10714000002B01D1FFF770FF1D4B1B785BB2022BA8
:107150000AD0032B29D0012B2CD121001D20012482
:10716000FFF716FF644205E0012C13D129211920F5
:10717000FFF70EFF7F2801DD0138FF3803007F3362
:1071800001DA7F204042C8237F21584303F01AF8D8
:10719000604310BD032C0BD12B211920FFF7F8FE03
:1071A000043CE7E72D211920D9E721001E20D6E76E
:1071B000052CF7D0012400206442E4E7E41A002003
:1071C0003400002010B50120FFF7B6FF4300012076
:1071D000184310BD10B50320FFF7AEFF4300012098
:1071E000184310BD10B50520FFF7A6FF430001208E
:1071F000184310BD144B70B51B68002B02D1012041
:10720000FFF79AFF114B1B785BB2013301D1FFF7F7
:107210000BFF0120FFF790FF04000320FFF78CFF16
:1072200005000520FFF788FF6D4364434043641960
:10723000201804F0D7FF01F0ABFC04F09DFF4300E1
:107240000120184370BDC046E41A0020340000201D
:10725000414B70B51B680500002B01D1FFF7A2FC64
:107260003E4C23787F2B00D872E007210E20FFF7D9
:107270008FFEC42833D101220E26394B10211A70FB
:10728000384B30001A702670FFF7D8FD802211218C
:107290003000FFF7D3FD0021615600291EDB324E7E
:1072A000C9B2300000F01FFE2D4B3000197800F0FD
:1072B0001BFD300000F082FE21780622300000F035
:1072C0000DFEAC1D300000F000FD002806D030009F
:1072D00000F000FD28700135A542F3D170BD0F21EB
:1072E0001920FFF755FE33280FD168221C4B1E26AC
:1072F0001A7000221B4B60211A7030000C3226706D
:10730000FFF79CFD02226121C2E700211820FFF750
:107310003FFEFA28BFD14222114B10261A700022DC
:10732000104B4B211A70300001322670FFF786FD9A
:10733000042001F0A1F838224C213000FFF77EFD37
:107340000F2251213000FFF779FD1B2252219FE7C8
:1073500000216156A3E7C046D81A0020350000205E
:107360003700002036000020101B002073B50026D7
:1073700006220021684605F069F86846FFF768FFB5
:10738000FFF7D6F91A4B6A469E576C466B469178C2
:107390001878D5785B7812796479002E1FD00002B6
:1073A0000902034329431BB209B2120211482243C6
:1073B000007812B240B2102802D15210DB10C9106E
:1073C000D8171B184340C817091841400120591805
:1073D000D317D2185A408A185200104376BD1B02A8
:1073E0002D02034329431BB209B22402DEE7C04643
:1073F0003600002035000020F8B501231C0098421B
:107400002BDD0F683B4228D04E6835001D4024D14B
:10741000042E22D90F2231680A40092A1DD173682F
:107420005C10202C00DD2024144B1B68002B01D1A4
:10743000FFF7B8FB72B67F10F9B2114F2200380087
:1074400000F04CFD62B6A54214DA380000F03DFCB5
:10745000002804D101246D002C432000F8BD380021
:1074600000F038FC0122AB004000F3181043986094
:10747000AD18E8E764000125EEE7C046D81A002001
:10748000101B002010B5054C2368002B02D01B20D8
:10749000FAF738F90020206010BDC046E81A002035
:1074A00010B5002803DC1C20FAF72CF910BD0B687E
:1074B000DA0706D4042B04D90F221B681340032BD0
:1074C00001D02420F0E7034B25201B68002BEBD0D4
:1074D0001B20E9E7E81A002010B5002803DC1C2077
:1074E000FAF710F910BD0B68DB0701D40D20F7E7A0
:1074F0001B20FAF707F90020F4E700001D4B70B5D8
:107500001B680C00002B03D12520FAF7FBF870BD97
:10751000012801DC1C20F8E708680121084207D196
:10752000042805D90F2302681340DD1E8D4201D9BE
:107530002420EAE765680D4201D11120E5E7042B1C
:107540000BD1FCF7ADFB05F00BFB63685B10013B57
:1075500001D4834208DB1220D7E7100980B2520021
:107560008000920F801AF0E71B20FAF7CBF8012079
:10757000CDE7C046E81A002010B50400802803DDDE
:107580002620FAF7BFF810BD002CFCDD1B20FAF70F
:10759000B9F8FEF755FFFFF7CBF8012000F06CFFBC
:1075A000F2E7000010B5002805DC1C20FAF7AAF865
:1075B0000400200010BD184B1B68002B01D12520B2
:1075C000F4E70124086804400FD04010FF2801D9D7
:1075D0002820EBE71B20FAF795F8FEF731FFFFF7BD
:1075E000A7F8012000F048FFF4E70428E1D90F21B3
:1075F00002681140042906D1FCF752FB05F0B0FAED
:10760000FFF7BAFFD5E70329D3D1100980B2520F93
:1076100080000A40801AF3E7E81A0020044B10B5F6
:107620001B682520002B00D01B20FAF76BF810BD3B
:10763000E81A002010B5034A06210348FEF736FB7E
:1076400010BDC046E4ED000014EE000000207047BD
:1076500001207047002070470020704700207047CD
:1076600001207047002070470020704700207047BD
:1076700000207047002070470020704700207047AE
:107680000020704700207047704770477047000027
:1076900010B5034A0F210348FEF708FB10BDC04692
:1076A0003CEE0000B4EE00000378013B1F2B00D934
:1076B00070470130F8E710B5FFF7F6FF0378002BAD
:1076C0000BD00130222B11D10378002B03D0421CA8
:1076D000222B03D11000FFF7E7FF10BD5C2B03D175
:1076E0004378002B00D0821C1000EDE73A2BF2D03B
:1076F0002C2BF0D07B2B0BD1FFF7D6FF0378002B80
:10770000E9D07D2B01D10130E5E7FFF7D4FFF5E7A4
:1077100020225B2B14D1FFF7C7FF0378002BDAD0B0
:107720005D2BF0D0FFF7C7FFF7E7202BD3DD2C2B25
:10773000D3D0190091435D29CFD0222BCDD0013079
:107740000378002BF1D1C6E7002210B5904216D085
:10775000FFF7AAFF03780422222B10D0023A7B2BDA
:107760000DD0013A5B2B0AD01900303902320929B9
:1077700005D92D2B05D14178303909290AD81000B7
:1077800010BD0522742BFAD00132662BF7D00132DE
:107790006E2BF4D0581E83415A42F0E770B5FFF7C4
:1077A00083FF037801222D2B01D18018023A002398
:1077B0000A2502E06B430130CB1801783039CCB296
:1077C000092CF7D95A43100070BDF8B50C0015000C
:1077D000FFF76AFF0378222B02D000232370F8BD45
:1077E0000D236A1E210008250C260A279C4601301D
:1077F0000378222B02D100230B70F0E7002BFAD084
:10780000441C5C2B0BD14378841C622B0ED0662B5E
:107810000ED06E2B0ED0722B0ED0742B0ED0002AF1
:10782000E9DD0B70013A01312000E1E72B00F6E7BA
:107830003300F4E73B00F2E76346F0E70923EEE7A5
:1078400010B50400FFF737FFA04203D90378013BCE
:107850001F2B00D910BD0138F6E710B5002815D050
:107860000378002B13D0FFF71FFF202103780200BD
:107870008B4300205D2B09D01000FFF71CFF03781D
:107880002C3B5A425341C018FFF70EFF10BD1800A1
:10789000FCE70300002070B50C0081420EDD1A7871
:1078A0005B2A0BD1581CFFF7FFFE0125AC4205D027
:1078B000FFF7D3FF002801D00135F7E770BD70B5A1
:1078C0000C001500002901D000230B70002820D0E7
:1078D0000378002B1ED0FFF7E7FE037806002C2B61
:1078E00003D10130FFF7E0FE0600337800207D2B46
:1078F0000FD0844204D02A0021003000FFF765FF3A
:107900003000FFF7D8FE03783A2B02D10130FFF7A1
:10791000CBFE70BD1800FCE7F0B50D0004009DB073
:107920002E78002E35D02E21280005F001F9071EF3
:1079300014D0431B0193303E092E14D82800FFF7C2
:107940002DFF01002000FFF7A4FF0400002C20D031
:10795000002F1ED0019B0133ED18E1E7280005F050
:10796000FFF80190E7E723787B2B11D1601C64229C
:1079700003A9FFF7A4FF041E0BD0019A290003A856
:1079800005F0F5F80028E1D02000FFF794FEEEE7BF
:10799000002420001DB0F0BD70B5050000200C00D3
:1079A00081421DDD2800FFF7CFFE0300681C012B7C
:1079B00014D00020022B13D10022681C1100FFF705
:1079C0007EFF012C0CD0FFF748FF00221100FFF7CB
:1079D00076FF013CF5E7FFF740FF013C012CFAD1AF
:1079E00070BDF8B5050000200C0016001F00814294
:1079F0000DDD2800FFF7A8FE03000020022B06D1B2
:107A0000681C3A003100FFF75AFF012C00D1F8BD85
:107A1000FFF723FF3A003100FFF751FF013CF4E785
:107A200010B50024A04218D0FFF73EFE03787B2B50
:107A30000AD1013000221100FFF741FF00280CD0CD
:107A4000FFF739FE0134F5E75B2B06D10130FFF774
:107A500004FF002801D00134F9E7200010BDF8B57B
:107A6000002816DD0D68EB0713D56D10013D0124CC
:107A7000FDF744FB0026FF27644200280CD1002EAE
:107A800021D0300005F06CF801003000FCF728FB35
:107A9000F8BD01256D42EAE703681A143A40152A39
:107AA0000BD11B123B409C4200DA1C009D4201D1CD
:107AB00006000836FDF716FADFE71D2AFAD1012481
:107AC00000266442F6E70120013464002043DFE72A
:107AD00010B508680C00FCF7E3F8FEF705FE002877
:107AE00003DB6268024B8000C250002010BDC0461C
:107AF000982D002010B50868FCF7D2F8FEF7F4FDC9
:107B00000123002802DB024B8000C358180010BD7F
:107B1000982D002010B50868FCF7C2F8FEF7E4FDC8
:107B2000C043C00F800010BD10B5034A04210348B4
:107B3000FEF7BCF810BDC04650EF00004AEF000051
:107B400010B5FBF7CFFFFCF77DF8FEF71BF90448F3
:107B5000FEF73CFBFDF712FBFEF718FC10BDC0461C
:107B60009FEF000010B5FBF739FC10BD70B5002584
:107B700004AC24780573A94205D10A4B0A4A252191
:107B80000A4804F0D9FB01600949920052589B0051
:107B900002715B58A40083716358856043710223AE
:107BA000C37170BDB7EF000016F00000C5EF000014
:107BB00074F00000037B002B04D1437383730361D3
:107BC00001330373704700001FB50191A021002409
:107BD0000068C900D2B24450012A10D0A24209D094
:107BE000032A0AD0074A8350074B019AC250012347
:107BF00043501FBD02221343F4E70422FBE7062291
:107C0000F9E7C046540500002405000010B5040043
:107C1000FFF7D0FFA1222368A179D20099506179A2
:107C2000064A20009950217904329950044B196872
:107C30005A689B68FFF7C8FF10BDC0460C050000DE
:107C4000041B00201FB5FFF7BFFF05B000BD704744
:107C50000368074A99501A00FC32D1680029FCD009
:107C6000A321C90058580023C0B2D3607047C04652
:107C70001C05000007B58022074BD2051A600022C0
:107C80009A6002321A710F230C3200930349023BAF
:107C90000348FFF76BFF07BD041B002000300040C6
:107CA000F01A0020F8B505000E0017000024BC42B1
:107CB00008D02B68315D1B6828009847002801D048
:107CC0000134F4E72000F8BD704710B51C3000F017
:107CD000AFF910BD10B51C3000F09CF910BD10B507
:107CE0001C3000F0ABF910BD70B5437E0D00002BC9
:107CF00001D1002070BD6430040000F0A8F9002814
:107D0000F7D12000290000F076F90120F2E7000009
:107D1000F7B50193FA23002504009B0083600B4B09
:107D20004560083303601C300F00160000F058F95E
:107D30002000643000F054F96B461B7927616675AA
:107D40006576A5762000A375FEBDC04654F0000000
:107D5000012330B5A024C375837D13499B005A5875
:107D6000437DC132114DFF32E40592009B005B5808
:107D70001551CC22C133FF339B001D5104690C4BBC
:107D80005204E25005220469243BE250837D0469D9
:107D90009B005A58A123DB00E250437D02699B00FF
:107DA0005958044BD15030BD74F000000C0600004F
:107DB000240500000C050000A022002310B5046972
:107DC000D200A3500A4CA1420FD90A4C8C425B410D
:107DD00009495B420B40CD21C9045B18046907497E
:107DE000635005210369995010BDCC235B04F5E76E
:107DF000A086010090D00300000098FD240500003B
:107E0000F7B5040000200D000193824265D01600F2
:107E1000402A00D9402627001C37380000F0F6F829
:107E2000B1232269DB00D550802201232169920011
:107E30008B50A27E002A03D122691362226913604B
:107E40000025731EAB4207D1019B002B04D080227A
:107E50000221236992009950012223691A62236941
:107E6000FC33DA68002A02D19A6A002AF9D09A6AA9
:107E7000002A0BD1DA60A3232269DB00D158380035
:107E8000C9B2013500F0B7F8B542DAD3019B2269D7
:107E9000002B0FD11300FC339B6A002B0AD1013356
:107EA000A376D3612369FC33DA6C002AFCD000226C
:107EB000DA640AE000230121A37651611A002369E4
:107EC000FC3399680029FCD09A602369FC339A6AD4
:107ED000002A01D000229A62E8B2FEBD10B501234B
:107EE000FFF78EFF10BD0300AC3310B5040019700E
:107EF000643000F08BF80123637610BD002302008C
:107F000070B5AC3243760D001178B12204000069DF
:107F1000D20081508022216992008B502269013366
:107F200013622269936026006436300000F080F806
:107F3000002812D0300000F06DF81E4B2269D0509E
:107F40002369FC331A6A002A02D19A6A002AF9D0FE
:107F50009A6A002A01D11A62E5E723690122002DFD
:107F60000DD11900FC31896A002908D1DA61236931
:107F7000FC33DA6C002AFCD00022DA6407E05A6194
:107F80002369FC339A68002AFCD000229A60002002
:107F90002369FC339A6A82420BD098622169064AAF
:107FA0008B588B501800022B03D0181F431E98418A
:107FB000033070BD1C050000C404000010B5012191
:107FC000FFF79CFF10BD000010B5132314220249D7
:107FD0000248FFF79DFE10BD00400040101B00202E
:107FE00010B540220021040004F030FA00232000E4
:107FF0002364636410BD10B53F24026C531C2340FE
:10800000446C9C4201D08154036410BD002303647E
:1080100043647047436C026C934206D03F21C25CBC
:1080200001330B4043641000704701204042FBE7DE
:10803000036C406C181A00D540307047436C026CDA
:10804000934201D0C05C704701204042FBE73F22D1
:10805000036C406C01331340181A43425841C0B2BC
:108060007047000003210A4802680A430260094879
:1080700002680A4302600849084A094B9B1A03DD5B
:10808000043BC858D050FBDC00F012F8F8F73CF87D
:108090002405004054050040C0F500000000002009
:1080A00070020020FEE7FEE7FEE7FEE7FEE7FEE7E0
:1080B000014B024A1A607047380000200024F40087
:1080C0000120704710B503681322DB69984710BD83
:1080D00070470000054B0269D1500369FC331A6AEE
:1080E000002AFCD0002201201A6270471C05000003
:1080F000030010B55C331A781F231A401E3B190089
:108100009140114AD167C222042104699200A15012
:10811000026953600269D360A02300220169DB0079
:10812000CA5001230169094A5B428B500169084A20
:108130008B5001690C3A8B50016908328B50143016
:10814000FFF764FF10BDC04604E100E00C0500002D
:108150001405000010B51430FFF76AFF10BD10B50C
:108160001430FFF76BFF10BD10B51430FFF752FF4E
:1081700010BD0000030070B55E331A780469724BBD
:10818000E25003005D331A780469704BE25003003B
:1081900061331C7802696E4B012C00D09EE0050013
:1081A0005F352E78A225ED00565102006032157819
:1081B000A1220669D200B5500269D4509623DB0093
:1081C000994200D88CE096231B01994200D88AE09E
:1081D00096235B01994200D888E096239B0199423F
:1081E00000D885E0E1239B01994200D882E09623E4
:1081F000DB01994200D880E0E123DB01994200D8FD
:108200007DE096231B02994200D87AE0E1231B020D
:10821000994200D877E096235B02994200D874E037
:10822000E1235B02994200D871E0E1239B0299426D
:1082300000D86EE0474B994200D86CE0E123DB02A6
:10824000994200D86AE0E122002312038A425B418E
:10825000414A5B421340802252059B1801693F4A04
:108260008B50A02304220169DB00CA50002103695E
:10827000FC33D9600369FC331962012301690B6087
:1082800001698B60C1210469890062501F215C3043
:1082900002780A4093406231314AFF315350002145
:1082A000415600293CDA0F230B40083B2D4C9B081C
:1082B0009B001B1903242140A140FC348C40DD6944
:1082C000A5432C00C0258D4029002143D9611F23DF
:1082D000017819401E3B8B40136070BD00246CE791
:1082E0009E23DB02BAE79D231B03B7E71E4BB5E7CE
:1082F0001E4BB3E7EC239B03B0E71D4BAEE71D4BD2
:10830000ACE71D4BAAE71D4BA8E71D4BA6E71D4B8D
:10831000A4E71D4BA2E78023DB049FE71B4B9DE7EF
:108320008C080F4BA400E41803230B40FF21C02549
:10833000DB009940AD0066598E433100C0269E4057
:1083400033000B436351C2E70C0500001405000025
:108350006C05000090D0030000D0BEFE2405000094
:1083600000E100E000ED00E000B013000050270045
:1083700000A04E0000F0750000509D0000F0EB00E2
:1083800000903A0100E0D70100B0AF0300705F0732
:10839000F7B5009308AB1B7800250193FA2304007E
:1083A0009B0083600E4B45600833036014300F0060
:1083B0001600FFF715FE23005C3327611E70009B3B
:1083C000084A9B00995823005D331970019B2000D7
:1083D0009B009A5823005E33DD701A70FEBDC046C4
:1083E000F8F0000074F00000036910B51A00FC32C8
:1083F000D2680400002A0AD0A322D200995814306F
:10840000C9B2FFF7F8FD00222369FC33DA6010BD22
:1084100010B50248FFF7E8FF10BDC046C81B00209A
:10842000162307B5022200930249013B0248FFF7D9
:10843000AFFF07BD00200040C81B002010B500287A
:1084400001D004F0BFFA10BD0849094A094B10B524
:108450001B688858FA22190A1B0618439200002349
:1084600001F0E8FF4904C00B084310BD00100140B3
:10847000040500002C1C002070B5041E09D0FFF775
:10848000E3FF050000F014F8FFF7DEFF401BA042F9
:10849000F8D370BD0022044B9A60044A136801337C
:1084A000DBB213607047C046FC1001402C1C00205A
:1084B0007047704710B500F05FF8FFF7FAFF012032
:1084C000FFF7DAFFFFF73CFBFFF74CFB024B002BFB
:1084D000FAD000E000BFF7E700000000F8B54C1E3E
:1084E000A1410125104B114F8000C3584C42386800
:1084F0000F499D40160001F0DBFD0A21704301F099
:10850000D7FD2C400300220029000A4800F016F88D
:10851000FA21094C89004443386801F0C9FD010083
:10852000200001F0C5FDF8BD74F000003800002007
:1085300040420F00100500501027000030B50468BD
:108540000C40944206D1013B002BF8D112E0013BD4
:10855000002B0FD004680C409442F8D10024056829
:108560000D40954204D101349C42F8D1002002E034
:10857000201C00E0181C30BDC420114B80001A588C
:1085800010491140C02212020A431A50C021802211
:10859000490092025A501A608023A3220021DB0571
:1085A000D20099500122F9309A60074BFF301950E0
:1085B000C120023180001950403019501A607047B4
:1085C00000E100E0FF00FFFF00100140014B1860D8
:1085D0007047C04684000020F7B5002320285AD8F1
:1085E000384B8000C258042A5BD007D8022A54D0E6
:1085F00055D80423012A09D000234CE0062A54D080
:1086000051D31A2A53D002231B2AF5D12E4A1168BE
:1086100008294ED909294FD00A240226A020012575
:108620002A4AC00015502A482A4D07681C20BF005E
:1086300007402948019700685759009027481B02B6
:1086400007401F43C02300989B020340FF2057515F
:108650005759000207401F43019B1F43009B5801CD
:108660006023184007433E43565101251C4B1560BB
:1086700058680028FCD000205860A1230125DB00A9
:10868000D3585560A025ED0050511BB2A14202D035
:1086900015D2611ACB401800FEBD0823B6E710239F
:1086A000B4E72023B2E74023B0E78023AEE70123FD
:1086B000ACE708240026B1E70C000126AEE7091B51
:1086C0008B40E8E774F0000080000020007000405C
:1086D0003C0000200405000040000020FF00FFFFD8
:1086E000FC700040F0B520285BD8364B8000C258A3
:1086F000354B1E68002E30D1C227344BBF00D859ED
:10870000334C03250440C02000022043D851C0242C
:1087100080206400800018512E4F18602E4B803C42
:10872000D859FF3CA043D8510437D859A843204317
:10873000D8510837D8590C35A843844607206546D8
:108740002843D851A820C0001E50C1208026800098
:1087500076021E501C601C4B1C60142500202B0050
:108760001E4C2E0046433659771C1BD14343E25022
:10877000A0230325C132FF329200DB05D550184BF0
:108780001A68082A14D114234343E3189A6812483C
:108790005132FF32920059601150DA68C1239B00B8
:1087A000C250F0BD9642E1D001300328D9D1F8E79C
:1087B000082A02D9083AD140E5E708239A1A9140DD
:1087C000E1E7C04674F00000301C002000E100E04A
:1087D000FF00FFFF0405000000900040440000205F
:1087E000840000202149F0B54A6C2148002A14D0A9
:1087F000A025A12600230124ED05F600C258571C30
:1088000006D0C7187F68002F02D027009740AF51CD
:1088100014333C2BF2D100234B64A0230121DB0550
:1088200000260F009C4614234B43C3181A1F1268DE
:10883000104C0E4D920014195219526C002A10D08F
:108840001A00143A1268551C09D0103B1B68FF2B04
:1088500005D03B00934065461A00074BEA50FC34B4
:10886000666401310429DED1F0BDC046FC900040B1
:1088700044000020009000400C05000000B52028B6
:1088800010D80C4A8000835803290BD8A022080076
:10889000C133FF33D2059B0001F000FC020905073C
:1088A0000021D15000BD0C21FBE70421F9E7032191
:1088B000F7E7C04674F0000020280AD8074B800074
:1088C000C25801239340A022D205002902D10449B5
:1088D00053507047A121C900FAE7C04674F0000068
:1088E0000C05000003000020202B0AD8A021A222A2
:1088F000C905D2008858034A9B009B58D8400123E1
:108900001840704774F00000F7B506000D000C0029
:108910008B180193019B671B9C4207D03368217819
:108920001B683000984701340028F3D13800FEBDA1
:10893000F0B5C64600B5CB0F9846404A4B005B0DDC
:108940009A1882B00D000400132A2FDC002A49DB9C
:108950003B4F17413E000E40064323D07F083900AD
:1089600029400C430AD03749BD438C4663445C42DE
:108970005C418023DB021341E4071D434146CE00E6
:1089800031492B008E1922003468756820002900B7
:1089900001F0F6FE009001910098019922002B0051
:1089A00003F086F802B004BC9046F0BD332A08DD1F
:1089B0008023DB009A42F5D102000B0001F0E0FEBB
:1089C000F0E7224A9446012263445242DA400242CE
:1089D000E8D052080242D1D094438022D2051A41F5
:1089E0001443CBE74B005B080343DBD00B031B0BAB
:1089F0001C436342234380244D0C24031B0B234060
:108A00006D042B4319004346DA000F4B9B181C687A
:108A10005D6802000B002000290001F0B1FE00900B
:108A200001910098019922002B0003F041F8424681
:108A30004B005B08D60733431900B3E701FCFFFF87
:108A4000FFFF0F00EEFBFFFF28F10000EDFBFFFF33
:108A5000F8B5274A4B005B0D9A180C000700132A43
:108A600010DC002A36DB234B13410B423AD0802422
:108A700024031441002064189C43060025003000A4
:108A80002900F8BD332A0EDD80230600DB000D002F
:108A90009A42F4D102000B003800210001F070FE70
:108AA00006000D00EBE7144D0600AC4601256344BB
:108AB0006D42DD40AC4663460D000342DFD03323F8
:108AC0009A1A323B93401818874200D94C1C6346CF
:108AD0009843D2E7C90FCC070020531CCDD1074BD8
:108AE0001C43CAE706000D000028C0D1C7E7C046F6
:108AF00001FCFFFFFFFF0F00EDFBFFFF0000F03F59
:108B000030B5214A4B0087B05B0893421EDD1F4AF7
:108B1000934205DD02000B0002F0CAFF07B030BD32
:108B200002AA00F095F803231840049A059B012837
:108B300013D002281DD0002814D00298039900F009
:108B40006FFB80231B069C466144E7E7002300225D
:108B50000093002301F0DEF8E0E70298039900F0AB
:108B60005FFBDBE7012402980399009401F0D2F83F
:108B7000D4E7012402980399009401F0CBF88023F4
:108B80001B069C466144C9E7FB21E93FFFFFEF7FDD
:108B9000F0B54746CE4680B58DB004000D0000F01C
:108BA00067FA294B06001B780F005BB29846013329
:108BB00010D022002B002000290003F0C1FA8146CA
:108BC000002807D1002200232000290001F00AFC20
:108BD000002806D1300039000DB00CBC90469946F3
:108BE000F0BD01230293194B0694079503934B465E
:108BF0000A93434604940595002B15D000230022C8
:108C00001900100002F0D8F8434608900991022B91
:108C10000ED103F0AFFB212303600A9B0193002BCD
:108C20000CD1089E099FD5E70023002408930994DE
:108C300002A801F0C1F90028EFD1EAE703F09AFB9E
:108C40000A9B01930360ECE78800002038F10000E4
:108C5000F0B54E464546DE465746E0B5E14B4C0082
:108C60008FB09046894664089C4200DC87E0DE4B6A
:108C70009C4222DCDD4A002900DC92E0DC4B02F061
:108C800017FFDB4B06000F009C4200D17EE1D94A62
:108C9000D94B02F00DFF02000B00414630000A6084
:108CA0004B60390002F004FFD34BD24A02F000FFC0
:108CB000434601259860D9606BE0D04B9C4200DCB4
:108CC0008FE0CF4B9C4200DD55E1CE4A2315924602
:108CD0009A4451460905631A19001D00040003F067
:108CE0004BFA03F07FFA02000B00200029000892E3
:108CF000099302F0DDFE0022C34B02F067FC0F0077
:108D0000060003F039FA03F06DFA04000D000200CA
:108D10000B00300039000A940B9502F0C9FE0022C6
:108D2000B94B02F053FC002200230C900D9101F08E
:108D300053FB002800D192E10023002220002900EB
:108D400001F04AFB434243410133B04A414601929C
:108D5000022208A80092524600F07CFB4B46050018
:108D6000002B16DA802243461206944642465B6880
:108D7000454263445360D3686344D36009E00B0009
:108D8000020041460A604B600022002300258A60F1
:108D9000CB6028000FB03CBC90469946A246AB463B
:108DA000F0BD934B01F0ECFC914B06000F009C4290
:108DB00000D13DE18F4A904B01F0E2FC02000B0034
:108DC000414630000A604B60390002F071FE894A6A
:108DD000894B01F0D5FC012543466D429860D9606E
:108DE000D7E701F049F88A4A8A4B06000F0002F0E3
:108DF000EDFB0022884B01F0C3FC03F0BDF9050038
:108E000003F0F0F9794A7A4B0490059102F0DEFB09
:108E100002000B003000390002F04AFE754A0600DD
:108E20000F0004980599744B02F0D0FB0290039157
:108E30001F2D00DCC7E0029A039B3000390002F0CE
:108E400037FE83468A4653465B0024155B0DE31AC2
:108E5000102B6CDD04980599D322674B520502F064
:108E6000B5FB02000B00300039000292039302F0C0
:108E70001FFE0A000100130006910792020039004C
:108E8000300002F015FE029A039B02F011FE06006C
:108E90000F0004980599614A614B02F097FB32007C
:108EA0003B0002F005FE069E079F0B000200390002
:108EB00030000292039302F0FBFD4B005B0D8346F2
:108EC0008A46E41A312C32DD04980599B822544BB5
:108ED000920502F07BFB03000C0002000293039456
:108EE0000B000698079902F0E3FD02000B00060054
:108EF0000F000698079902F0DBFD029A039B02F02F
:108F0000D7FD484A0290039104980599464B02F018
:108F10005DFB029A039B02F0CBFD02000B003000C8
:108F200039000292039302F0C3FD83468A465A46F3
:108F30005346414630000A604B60390002F0B8FDEC
:108F4000029A039B02F0B4FD44460B000200A260AB
:108F5000E3604B46002B00DB1BE75B46236080236E
:108F60001B065344636080231B069C466144A0603B
:108F7000E1606D420DE70B00020002F099FD4346EF
:108F800000259860D9601860596002E7D3221A4B17
:108F9000520502F08DFD214A214B0D00040002F024
:108FA00087FD02000B00414620000A604B6029004B
:108FB00002F07EFD1A4B194A02F07AFD4346012564
:108FC0009860D960E5E602000B003000390002F03D
:108FD0006FFD6B1E154A9B009B5883468A46A34231
:108FE000A5D130E7FB21E93F7BD902400000405486
:108FF000FB21F93F3163621A61B4D03DFB21394155
:10900000FFFFEF7FEAFBFFFF00007041C0F10000AF
:1090100083C8C96D305FE43F0000E03F7370032EEA
:109020008A19A33BC14920259A837B3940F100006E
:10903000D3220C4B520501F0A3FB0B4A0B4B04004F
:109040000D0001F09DFB02000B00414620000A606C
:109050004B60290002F02CFD034A044BB9E60323C0
:1090600073E6C04661B4D03D7370032E8A19A33BEA
:10907000F8B54746CE46674B80B50A000F00190089
:1090800005003940994200D19BE004000100002F07
:1090900069DD3F1500D1B4E05F4B12039C4680238D
:1090A000120B5B0313435B00CA0F67449B184A0013
:1090B000F80703D5D20F5B009B188A0079108C4605
:1090C000002180201624894680030D189D4202DC71
:1090D00029185B1B8144D50F5B00013C5B195200D2
:1090E0004008002CF1D10020804680202025002758
:1090F000000609E08B425CD0D40F5B00013DE31811
:1091000052004008002D16D0C4198B42F2DD2718FA
:109110000E00002C49DB5B1AA242894149425B1ACE
:10912000121BD40F5B00013D80443100E318520054
:109130004008002DE8D113434ED143465B08374920
:109140004A468846494652104244C90702D5802102
:1091500009060B4361460F05BD18180029000CBC19
:1091600090469946F8BD7B005B0803433900002B0D
:10917000F5D0002F3CD1E30A153A6405002BFAD054
:109180008020400303423FD1002700E00F005B0036
:10919000791C0342FAD0250020208D40401A290076
:1091A000D71B2200C2401A4376E7FE43F60F8E1902
:1091B000B1E79442A0D82718002CF6DB1E0000234C
:1091C000AEE702003B002800390002F0FFF92A0058
:1091D0003B0001F0D5FAC2E74346013303D04346D2
:1091E00001335B08ABE7012398460023C144A6E79F
:1091F0003B00020002F05CFC02000B0001F0DCFD11
:10920000ADE713000022BBE70127210020207F42A9
:10921000C6E7C0460000F07F01FCFFFF0000E03F12
:10922000F0B54746CE4680B587B000920193754BA6
:109230004F00814688467F089F4263DC02F09CFF16
:10924000002800D1D4E04A4643464846414602F051
:10925000BDF904000D006C4A6C4B02F0B7F96C4A82
:109260006C4B01F08DFA22002B0002F0AFF96A4A34
:109270006A4B02F01DFC22002B0002F0A7F9684A9D
:10928000684B01F07DFA22002B0002F09FF9664A3C
:10929000664B02F00DFC22002B0002F097F9644AA5
:1092A000644B01F06DFA22002B0002F08FF902905E
:1092B00003910022604B2000290002F087F9029AF6
:1092C000039B06000F002000290002F07FF9009A9E
:1092D000019B04000D004846414602F077F9020068
:1092E0000B002000290002F0E3FB02000B0030001D
:1092F000390002F0DDFB02000B0000204F4902F0B4
:10930000D7FB70E002000B0002F060F904000D00D2
:109310003D4A3E4B02F05AF93D4A3E4B01F030FACD
:1093200022002B0002F052F93B4A3C4B02F0C0FBFA
:1093300022002B0002F04AF9394A3A4B01F020FA98
:1093400022002B0002F042F9374A384B02F0B0FB02
:1093500022002B0002F03AF9354A364B01F010FAA0
:109360002B00220002F032F9354B029003919F420C
:109370009FDD344B00229F423DDC334900207B18A7
:109380002E4916001F0002F093FB04900591002265
:10939000294B2000290002F019F932003B0002F0AD
:1093A00087FB029A039B06000F002000290002F0B1
:1093B0000DF9009A019B04000D004846414602F059
:1093C00005F902000B002000290002F071FB0200E9
:1093D0000B003000390002F06BFB02000B00049818
:1093E000059902F065FB07B00CBC90469946F0BDAC
:1093F00000201249F7E7154B002604920593144FFD
:10940000C5E7C046FFFF3F3ED43888BEE9FAA8BD95
:10941000C4B1B4BD9EEE213EAD529C804F7E923EC3
:109420009015CB19A001FA3E7751C1166CC1563F79
:109430004C5555555555A53F0000E03F0000F03F05
:109440003233D33F0000E93F0000E0FF0000E73F78
:109450000000D23FF0B5DE464E4645465746E0B5E1
:10946000DC4CA5440D9114001900A49A0993DA4B21
:109470009200D6584D1E03901821E01E06960295C4
:1094800000F0A0FEC3430100DB1719404B1C9A00FB
:109490009B1ADB001B190B9105934C1B771918D4F1
:1094A000A59BA5009C463F1922AE6544013707E005
:1094B000286802F097FE013403C60435BC4208D088
:1094C000002CF5DA00200021013403C60435BC422B
:1094D000F6D1069B002B01DA00F0FDFB069B0399F9
:1094E0000133DB009A46099BDA0094460092002281
:1094F000914672AA0492B94A6144934688469AAB4F
:1095000063449B44029B002B00DABCE15D460026CD
:109510000027039C4D442A686B6803CC02F056F880
:1095200002000B003000390001F02AF9083D060066
:109530000F004445EFD1049B4B441E605F6008233D
:109540009C46E144D145DDD10EA804218446494220
:1095500061448C46069A93009C44614684460A9175
:109560000399083B63448C460C93009B0092634430
:109570009B46009A0498D10003008C4663440891EE
:109580001E685F68002A33DD954980468C46624438
:10959000D300984470AB9A460EAB99460022914B8B
:1095A0003000390002F012F802F0E6FD02F01AFE77
:1095B00000228D4B04000D0002F008F802000B00A1
:1095C0003000390002F074FA02F0D6FD4B4601C3B8
:1095D0009946434620001A685B68290001F0D0F8DC
:1095E00008235B429C46E04406000F00D045D5D1DD
:1095F000059B30001A003900984600F0DFFCFF237D
:1096000000229B0504000D0001F0E0FF00F038FC93
:109610000022764B01F0DAFF02000B002000290047
:1096200002F046FA0D00040002F0A6FD814602F0A9
:10963000D9FD02000B002000290002F039FA0600D3
:1096400040460F00002800DCEEE0009B18215A1E67
:1096500092000EAB9B58091A1D000D41A9448D4084
:109660005D1B0EAB9D5017231B1A1D41002D2DDDD8
:1096700001239C46009BE144002B00DC1CE20E9C75
:109680000123002C00D0B5E0009A012A09D09900EE
:109690000EAA54580133002C00D0ACE0009A9A4234
:1096A000F5D1059B002B0EDD012B00D1A8E1022B8B
:1096B00009D1009B0EA95A1E92000EAB9B5807932E
:1096C0009B029B0A8B50022D00D1C1E00023002297
:1096D0003000390000F080FE009B002800D194E2A9
:1096E000069A591E8A4210DC414A0A9894460EAAEC
:1096F0006344944600229B0063441C68043B22435D
:109700008342FAD1002A00D0C0E0069B0EAA013B9A
:109710009B00D358002B00D0B3E001220C9B043BEC
:10972000596801320029FAD0009B9C46624411001E
:1097300007921A0001338B4246DC0B986346804641
:10974000A59C4344A046099C9B00A1464A449844DA
:10975000D30022AA9146049A99449446089BA59A5C
:1097600063448446614494469A468B006344009364
:109770004346586802F036FD4B4618605960029B1C
:10978000002B24DB4D46039C0026002701E02868BF
:1097900069680CCC01F01AFF02000B0030003900A0
:1097A00000F0EEFF083D06000F005C45EFD1534688
:1097B0009E60DF6004239C460433E0449C46009B8B
:1097C000E144E2449845D3D1079B0093D1E60026BB
:1097D0000027ECE794FDFFFF08F3000018FEFFFFF1
:1097E000FFFFFF1F0000703E00007041000020409E
:1097F000FFFFFF3F002180225204141B0EAA545089
:10980000009999420EDD0EA884469B000EAA89009D
:10981000D25861446344CF4800E01A68821A04C3F6
:109820008B42FAD101243CE7059B002B06D1009B1B
:109830000EAA013B9B00D558ED1517E70022C64B39
:10984000300000F0EDFD002800D024E100253DE7C8
:1098500032003B000020C14902F02AF906000F0047
:10986000002C00D132E7059A0020BC4900F0A6FB8D
:1098700002000B003000390002F01AF906000F0058
:1098800024E7012250E70026002754E64B46059ABC
:10989000079388468B000EA9CB58183A0895059275
:1098A000002B0DD18C464146AD4B43449B00634495
:1098B000043B58680139183A0028F9D088460592C7
:1098C000059A0020A54900F079FB434604000D00ED
:1098D000002B00DA05E29E000EAB9C464346DB00FF
:1098E00066449C46059370AB9946049F6744009775
:1098F000306802F077FC22002B0001F067FE0022A6
:1099000038607960974B2000290001F05FFE083F26
:1099100004000D00043EB945EAD14AAB03939B46CF
:1099200000239A46069B42469946434601320292DC
:1099300004934B46002B00DAAAE080208A4B009D5E
:109940009846C005894900260027002408E008231E
:109950009C460835E044544511DC43461868596874
:109960002A686B6801F032FE02000B0030003900FB
:1099700000F006FF013406000F00A145E7DA5B4660
:10998000C0C39B4601239C46009BE244083B0093D6
:10999000029B9A45CDD1049B9846A49B022B00DDE7
:1099A0008EE0002B37DC1FD1059B00271D00039B99
:1099B00000249C461E006544083E2A686B683800F7
:1099C000210000F0DDFE083D07000C00AE42F4D19E
:1099D000089B002B03D080231B069C4664443A005E
:1099E00023000D990A604B600720079B18409B23BA
:1099F0009B009D443CBC90469946A246AB46F0BDB8
:109A0000009B0EA95A1E92000EAB9B5807935B0257
:109A10005B0A8B5057E64346002B00DA70E10020CA
:109A20000021DB004AAAD61848AF32687368083EA6
:109A300000F0A6FEB742F8D1089B002B00D025E12C
:109A40000B0002004A984B990D9C2260636002F063
:109A50002FF8434607000C00002B13DD01254CAE08
:109A6000B14638002E0021004C4601360CCC00F0E7
:109A700087FEA146B045F7DA089B07000C00002BD3
:109A800000D015E13A0023000D998A60CB60ABE766
:109A90000026002773E701239C46009BE144022532
:109AA000002B00DDEBE532003B0000202B4901F0EC
:109AB000FFFF06000F0009E60024F2E54AAB03931E
:109AC000A49B032B00D08FE74346002B00DC14E15E
:109AD000039ADB009B46130091465B441E685F6857
:109AE000234B43440293DB00994448AB9A464B46D0
:109AF0005C681B681800210032003B000090019157
:109B000000F03EFE04000D0002000B0000980199D9
:109B100001F0CEFF3B00320000F032FE4B46986071
:109B2000D9601C605D6008235B429C46E1442600CE
:109B30002F00CA45DBD14346012B00DCE3E0039A4A
:109B400013005B441E685F68029BDB0099464A4431
:109B5000904610E0FFFFFF000000E03F0000F03FF4
:109B6000FFFFFF3F0000703EC8F20000FB21F93FFD
:109B7000FFFFFF1F984643465C681B6818002100E2
:109B800032003B000090019100F0FAFD04000D004E
:109B900002000B000098019901F08AFF32003B009F
:109BA00000F0EEFD4346039A9860D9601C605D604A
:109BB000083B26002F009A42DCD14D4694460026F1
:109BC00000244746083565442A686B683000210048
:109BD00000F0D6FD083D06000C00AF42F4D1039B17
:109BE0004A9F5D689968D868089B002B65D08022E1
:109BF000120694460D9B6544604464441F605D609A
:109C00009960D8601E615C61EEE69A464B46079308
:109C1000059B30005A423900089500F0CFF9002228
:109C20003A4B06000F0000F0FBFB002824D0384B15
:109C300000223000390001F0C9FC02F09DFA5246C2
:109C40000400950002F0CEFA0022304B01F0BEFC79
:109C500002000B003000390001F02AFF02F08CFAFC
:109C60000EAA50510122059B524418339046059389
:109C700093000EAAD45023E65346300039009C00CE
:109C800002F07AFA0EAB1851D04619E680230D9AED
:109C90001B06CB18106053600B0002004A984B99CA
:109CA00001F006FF434607000C00002B00DDD5E65F
:109CB00080231B069C466444E4E62B003A000D9D7D
:109CC0002A606B600A000300AA60EB603200230088
:109CD0002A616B6188E6099BDB00009372AB0493F9
:109CE00032E4A49B022B00DDE8E6002B00DD92E6C7
:109CF00000D079E6002700246AE6002600246EE7FB
:109D00000020002198E60026340068E7000070413A
:109D10000000703EF0B5CE46474680B587B0009251
:109D20000193474A4B00814688465B08934207DC13
:109D30004146484602F020FA4146031E484666D096
:109D40004A4643464846414601F040FC04000D00A7
:109D500002000B004846414601F038FC394A3A4BB4
:109D600006000F002000290001F030FC374A384B74
:109D700001F09EFE22002B0001F028FC354A364BF4
:109D800000F0FEFC22002B0001F020FC334A344B93
:109D900001F08EFE22002B0001F018FC314B324AFC
:109DA00000F0EEFC0E9B02900391002B34D0009843
:109DB000019900222D4B01F009FC029A039B0490AB
:109DC00005913000390001F001FC02000B000498FD
:109DD000059901F06DFE22002B0001F0F7FB009ABF
:109DE000019B01F065FE224A04000D00214B30006A
:109DF000390001F0EBFB02000B002000290000F00D
:109E0000BFFC02000B004846414601F051FE07B07E
:109E10000CBC90469946F0BD02000B0020002900C2
:109E200001F0D4FB124A134B01F042FE32003B001A
:109E300001F0CCFB4A46434600F0A2FCE7E7C046EF
:109E4000FFFF3F3E7CD5CF5A3AD9E53DEB9C2B8AAC
:109E5000E6E55A3E7DFEB157E31DC73ED561C11907
:109E6000A0012A3F1111813FA6F810110000E03F28
:109E7000495555555555C53F49004B081900704780
:109E8000474AF0B54F4691464B005B0D9944464614
:109E9000D6464A46C0B505000C000E0088460700AD
:109EA000132A27DC002A4BDB3E4B13419A460B005A
:109EB00052461340034318D03B4A3C4B2800210034
:109EC00000F05EFC0022002300F0A0FA002847D03A
:109ED000002C04DA80234A465B031341984446462B
:109EE000534600279E43380031001CBC90469946DB
:109EF000A246F0BD332A08DD8023DB009945F4D16A
:109F000002000B0000F03CFCEFE7294A94460122D6
:109F100063445242DA4092460242E6D0224A234B40
:109F20002800210000F02CFC0022002300F06EFA33
:109F3000002815D0002C1EDB534646469F430FE0F9
:109F4000194A1A4B2800210000F01AFC00220023B5
:109F500000F05CFA002803D0002C04DB0027002668
:109F600038003100C1E76400640825430027002D54
:109F7000F6D0104EF4E74B46142B0BD03422D21AF5
:109F8000012393405D19BD4208D201239C462F0056
:109F9000E044D1E7133B9C46E044CDE72F00CBE7FC
:109FA00001FCFFFFFFFF0F009C7500883CE4377E3B
:109FB000EDFBFFFF0000F0BF002070474B0070B5C5
:109FC0005B0D14000A00002B1AD14B005B08034301
:109FD00015D0234B002201F0F9FA224B9C422DDBD5
:109FE0000A004B005B0D363B1F4DE318AB422ADCE9
:109FF000002B0DDD1D4C1B0522401A43110070BDC6
:10A000001B4DAB42F0D102000B0000F0B9FBF6E7AC
:10A010001D00353519DA174B02009C4209DD0B0093
:10A020001548164900F032F8134A144B01F0CEFAE5
:10A03000E5E70B001248134900F028F8104A114BCD
:10A0400001F0C4FADBE70200E9E7084C36332240AE
:10A050001B051343190000220B4B01F0B7FACEE7A2
:10A0600000005043B03CFFFFFE070000FFFF0F80E1
:10A07000FF07000050C300009C7500883CE4377E59
:10A0800059F3F8C21F6EA5010000903C30B54A009C
:10A09000DB0FDB0752081A43110030BD02B47146D2
:10A0A00049084900095C49008E4402BC7047C0461B
:10A0B000002243088B4274D303098B425FD3030A07
:10A0C0008B4244D3030B8B4228D3030C8B420DD31A
:10A0D000FF22090212BA030C8B4202D312120902A8
:10A0E00065D0030B8B4219D300E0090AC30B8B42E6
:10A0F00001D3CB03C01A5241830B8B4201D38B0394
:10A10000C01A5241430B8B4201D34B03C01A524138
:10A11000030B8B4201D30B03C01A5241C30A8B427B
:10A1200001D3CB02C01A5241830A8B4201D38B0266
:10A13000C01A5241430A8B4201D34B02C01A52410A
:10A14000030A8B4201D30B02C01A5241CDD2C3097C
:10A150008B4201D3CB01C01A524183098B4201D3F8
:10A160008B01C01A524143098B4201D34B01C01AE3
:10A17000524103098B4201D30B01C01A5241C3085B
:10A180008B4201D3CB00C01A524183088B4201D3CA
:10A190008B00C01A524143088B4201D34B00C01AB6
:10A1A0005241411A00D20146524110467047FFE722
:10A1B00001B5002000F0F0F802BDC0460029F7D03C
:10A1C00076E7704703460B437FD4002243088B4257
:10A1D00074D303098B425FD3030A8B4244D3030B2E
:10A1E0008B4228D3030C8B420DD3FF22090212BAF3
:10A1F000030C8B4202D31212090265D0030B8B426F
:10A2000019D300E0090AC30B8B4201D3CB03C01A58
:10A210005241830B8B4201D38B03C01A5241430B33
:10A220008B4201D34B03C01A5241030B8B4201D323
:10A230000B03C01A5241C30A8B4201D3CB02C01A8E
:10A240005241830A8B4201D38B02C01A5241430A06
:10A250008B4201D34B02C01A5241030A8B4201D3F5
:10A260000B02C01A5241CDD2C3098B4201D3CB019C
:10A27000C01A524183098B4201D38B01C01A52414B
:10A2800043098B4201D34B01C01A524103098B424F
:10A2900001D30B01C01A5241C3088B4201D3CB003A
:10A2A000C01A524183088B4201D38B00C01A52411D
:10A2B00043088B4201D34B00C01A5241411A00D2CD
:10A2C00001465241104670475DE0CA0F00D0494236
:10A2D000031000D34042534000229C4603098B42A6
:10A2E0002DD3030A8B4212D3FC22890112BA030A2E
:10A2F0008B420CD3890192118B4208D389019211B0
:10A300008B4204D389013AD0921100E08909C30934
:10A310008B4201D3CB01C01A524183098B4201D336
:10A320008B01C01A524143098B4201D34B01C01A21
:10A33000524103098B4201D30B01C01A5241C30899
:10A340008B4201D3CB00C01A524183088B4201D308
:10A350008B00C01A5241D9D243088B4201D34B0023
:10A36000C01A5241411A00D20146634652415B1065
:10A37000104601D34042002B00D549427047634646
:10A380005B1000D3404201B5002000F005F802BD8B
:10A390000029F8D016E770477047C046D0400B1C24
:10A3A0001141203A03D49C4613411843634652425C
:10A3B000934018437047C0468446101C62468C4642
:10A3C000191C634600E0C0461FB501F097F800284D
:10A3D00001D40021C8421FBD10B500F0EFFF40427C
:10A3E000013010BD10B501F089F8002801DB002014
:10A3F00010BD012010BDC04610B501F07FF8002847
:10A4000001DD002010BD012010BDC04610B501F0D7
:10A4100011F8002801DC002010BD012010BDC0464D
:10A4200010B501F007F8002801DA002010BD012066
:10A4300010BDC046F0B5CE46474615042D0C2E0083
:10A4400080B50704140C3F0C9946030C7E435D4312
:10A45000674363437F19340CE4199C46A54203D932
:10A4600080235B029846C4444B4643435143250C2A
:10A4700036046544360C2404A4195B1959182000CD
:10A480000CBC90469946F0BDF0B54E465746454641
:10A49000DE46E0B543025B0A450083B00F1C9946D7
:10A4A0002D0EC60F002D57D0FF2D24D08020DB00AD
:10A4B000C0041843002381469A469B467F3D7C0298
:10A4C0007A00FB0F640A120E984623D0FF2A4BD065
:10A4D000E30080240020E4047F3A1C43AD186B1C89
:10A4E00047460193534677403A000F2B48D87D49A1
:10A4F0009B00CB589F46002B00D085E008339A463E
:10A50000063B9B467C027A00FB0FFF25640A120E75
:10A510009846DBD1002C00D090E0524601231A432C
:10A5200092460120DBE74C4658461700022824D00B
:10A53000032800D1CFE00022002301284DD158028A
:10A54000D205400AFF071043384303B03CBC904695
:10A550009946A246AB46F0BD002B5BD104239A4638
:10A56000033B00259B46AAE7FF35002C60D15246ED
:10A5700002231A4392460220B1E7FF220023DEE7BE
:10A580004B461B0C9C464B462604360C1804614671
:10A590003300220C6446000C43434E435043544363
:10A5A00080191A0C1218964203D9802149028C4650
:10A5B00064441B041B0C1004C01883015E1EB341CD
:10A5C000800E1843130C1B199B0103431C0023012D
:10A5D00079D5012362081C401443019A7F32002A76
:10A5E0004DDD630704D00F232340042B00D0043437
:10A5F000230103D53C4B019A1C408032FE2ABCDC6F
:10A60000A3015B0AD2B29AE70C239A46093BFF25C5
:10A610009B4654E7180001F071FE4A46431F762519
:10A620009A4000236D4291462D1A9A469B4646E772
:10A63000524603231A439246032050E7200001F0BC
:10A640005DFE431F2D1A9C40763D002047E7802386
:10A650000027DB03FF2272E7424666E74C463200E2
:10A66000584662E780234A46DB031A4222D01C4246
:10A6700020D123435B025B0A4746FF225FE70123A9
:10A680009A1A1B2A21DC23000199D3409E318C4069
:10A690001A0023005C1EA34113435A0704D00F2263
:10A6A0001A40042A00D004335A0111D49B015B0ADA
:10A6B000002244E780234A46DB0313435B025B0A24
:10A6C0003700FF223BE7019587E70022002336E7AA
:10A6D0000122002333E78023DB0323435B025B0A71
:10A6E000FF222CE718F30000FFFFFFF770B50028EA
:10A6F0003DD0C317C5185D40C40F280001F0FEFD12
:10A700009E22121A962A07DCD2B2082833DD0838B6
:10A7100085406802400A23E0992A0BDD05232900C1
:10A720001B1AD94003001B339D402B005D1EAB411B
:10A7300019430D00052801DD431F9D402B000F49E3
:10A740000B406E0709D00F263540042D05D0043389
:10A750005D0102D59F220B40121A9B01580AD2B20A
:10A760004002D205400AE4071043204370BD002494
:10A7700000220020F4E76802400AF1E7FFFFFFFB38
:10A78000F0B54F464646D6460C000903C0B5490A07
:10A79000470F5E0039431F03DB0F9C4665007B0AB1
:10A7A000570F1F436D0DE40F760DA146C000B8464C
:10A7B000D200AB1B64457BD0002B5FDD002E00D0A8
:10A7C000A4E03E00164300D112E15E1E002E00D030
:10A7D0009EE1871A4346B84280410125C91A40428A
:10A7E000091A0B0200D431E149024E0A002E00D1B1
:10A7F0006EE1300001F082FD0300083B1F2B00DDFD
:10A8000061E120223900D21A9E40D1409F400E4380
:10A810009D4200DD51E15D1B6B1C1F2B00DD7CE1C7
:10A820002021C91A3D0030008F408840DD40791E4C
:10A830008F41310007222843D940002507433A4081
:10A84000002A09D00F233B40042B05D03B1DBB42FF
:10A85000BF417F42C9191F000B0200D426E26A1CC7
:10A86000C64B55056D0D9A4200D106E1C44AFF085A
:10A870000A40530752023B43120B8EE0002B00D0DC
:10A88000B8E06B1C5B055B0D012B00DC30E1871A27
:10A890004346B842B641CB1A76429E1B330200D5DE
:10A8A0004CE13B003343A1D100220024002570E09D
:10A8B000002B00DCE5E0002E00D183E0AF4EB54276
:10A8C00060D0802636043743B846382B00DC3EE1A2
:10A8D000434613431F007A1E97413F188742804129
:10A8E000404209180B0200D4B0E0A44B01359D4250
:10A8F00000D1C3E0A24A7B080A4001210F401F4358
:10A900005108D30707221F433A4099E79B4EB542AF
:10A9100038D0802636043743B846382B00DDDCE0DB
:10A920001F2B00DC30E11E004746203EF740BC46AE
:10A93000202B04D04026F31A46469E40324317008F
:10A9400063467A1E97411F43CCE0002B00D104E2FE
:10A950004346134300D159E14B07C00818438023F5
:10A96000C9081B03194208D04546ED081D4204D111
:10A970004346D008590708432900420FC9007F4DBC
:10A980001143C0004B07CA087C49C00803438D42ED
:10A9900068D012036D05120B6D0D00211203180013
:10A9A000130B0A0D12051A43764B2D0513402B434A
:10A9B0005B00E4075B08234319001CBC90469946E2
:10A9C000A246F0BD3E00164312D05E1E002E00D0FF
:10A9D00000E187188742804141444042091801251F
:10A9E0000B0233D5022585E764463300414610004B
:10A9F0001D00C7E7002D00D0DAE00C000443F3D0BF
:10AA00005C1C00D19FE15D4CA64200D12FE1DB43ED
:10AA1000382B00DD66E11F2B00DD83E120240500DB
:10AA2000E41A0F00DD40D940A0404346A7405B1A1E
:10AA3000441EA04198462F433843171ABA42924108
:10AA400043465242991A64463500CAE607223A4004
:10AA5000002A00D0F6E64B07CA084849FF083B43E6
:10AA60008D4296D11900114300D19EE18021090346
:10AA70000A431203120B414D8FE7150000220023F9
:10AA80008BE7002B00D0C7E06B1C5F057F0D012F0B
:10AA900000DCF1E0394DAB4200D1B9E085180A0085
:10AAA000854289414244494251180722CF076D0827
:10AAB0002F4349083A401D00C2E607223049ED1AEB
:10AAC00031403A40BCE63E002838864000279FE6E9
:10AAD000380001F013FC20308EE6434613431F007C
:10AAE0007A1E9741C71BB84280414042091A78E656
:10AAF0000E003B0006431343002D61D1002E00D011
:10AB0000F4E0002B00D11BE164463900100039E766
:10AB10001A4FBB427AD03300FFE630001F3DE840B9
:10AB2000202B03D04021CB1A9E4037437B1E9F41F0
:10AB3000072207433A400021002589E7171A4346B8
:10AB4000BA42B641591A76428E1B64464EE61F2B16
:10AB500000DDADE020264746F61AB740B94617009B
:10AB6000B246DF404E463E4337005646B240561E80
:10AB7000B24117434246DA408918AEE6FF070000AB
:10AB8000FFFF7FFFFFFF0F8020264746F61AB740E2
:10AB9000B9461700B246DF404E463E4337005646A0
:10ABA000B240561EB24117434246DA40891A99E72D
:10ABB0007F4CA6425BD0802424045B42214327E7DC
:10ABC000002E0CD1002B00D1CBE0644639001000E0
:10ABD000774DD7E6764FBB4218D0330075E6002B91
:10ABE00014D04B07C00818438023C9081B0319421F
:10ABF00007D0FC081C4204D17907D0080843E1467D
:10AC000021004C46420FC9001143C000684DB9E60F
:10AC10001D0000220023C0E6002D5BD10D0005437E
:10AC200000D1E2E65D1C00D1B0E0614DAE421FD024
:10AC3000DB43382B71DC1F2B00DD96E020250F0055
:10AC4000ED1AAF40B9460700AA46DF404D463D43E6
:10AC50002F005546A840D940451EA84188440743C7
:10AC6000BF18974292415142414435003AE664464A
:10AC700035004146100085E60B000343002D00D04F
:10AC800063E6002BF5D04346134300D17AE68718DC
:10AC90008742804107224144404209183A400B0252
:10ACA00000D4D5E6434B01351940C9E5380069E6C3
:10ACB0001E004746203EF740BC46202B04D04026CD
:10ACC000F31A46469E403243170063467A1E974168
:10ACD0001F4302E6364DAE42CAD080252D045B42AA
:10ACE0002943A6E70843411E8841A6E6002B00D170
:10ACF00048E6871A4346B842B641CB1A76429E1BB5
:10AD000033024BD5171A4346BA429241591A52425E
:10AD1000891A072264463A4092E501430F00791EE2
:10AD20008F419DE71C000F00203CE740202B03D003
:10AD30004024E31A99400843411E884138437CE689
:10AD40000022002425E6171A4346BA429241591AB6
:10AD50005242891A6446350043E541461000144DBD
:10AD600010E680220024120380E61D000F00203D23
:10AD7000EF40BC46202B03D04025EB1A99400843F6
:10AD800007006346781E87411F4369E7871897428B
:10AD90009B4141445B42C9183500A3E53B00334366
:10ADA000CED0072231003A4052E600231A00F4E5E3
:10ADB000FF070000FFFF7FFFF0B55746DE464E4617
:10ADC0004546E0B5834607000E03480085B092462D
:10ADD0001C00360B400DCD0F002800D19DE0954B97
:10ADE000984239D08023F6001B041E43924A7B0F01
:10ADF000334399469446030063440093002300269E
:10AE0000FF00029323031B0B98466300E40F524696
:10AE10005B0D019400D1B3E086498B4200D19EE0E6
:10AE20004246D100802212040A435146490F114381
:10AE30008B46814952468C4600996344CB1A0021C7
:10AE4000D20000932B0063409A460F2E00D905E1F3
:10AE50007A4BB6009B599F465B463343994600D0D8
:10AE6000B8E002230826002700900293CAE7CB46E9
:10AE70003A0002990195019B9A46022927D003299D
:10AE800000D180E2012944D06D49009B8C46634487
:10AE90001C00002C38DD530700D013E2D2085B46BB
:10AEA000DB0109D55946674B19408B468021C90003
:10AEB0008C46009B63441C00634B9C4207DC5B4652
:10AEC00064055F075B0217431B0B620D02E0002362
:10AED0000027584A00211B031C0B0B0D1B052343A5
:10AEE00014055A4A380013401C4353466400DB07DC
:10AEF00064081C43210005B03CBC90469946A2461C
:10AF0000AB46F0BD0122524201231B1B382B00DC53
:10AF1000ADE1002200230027DCE75B46334399467E
:10AF20005ED0002E00D18AE1300001F0E7F9030085
:10AF30000B3B1C2B00DD7BE11D22D31A5A4601007E
:10AF4000DA4008398E4013005F46334399468F40FC
:10AF50003F4B00261B1A00930023029352E7414601
:10AF600053460B433B499B468C46009B63440093EE
:10AF70005B46002B3BD1022300221E43022161E7E6
:10AF8000434613439B4637D04346002B00D162E132
:10AF9000404601F0B3F903000B3B1C2B00DD53E1ED
:10AFA00002004146083A914088461D21CB1A51467D
:10AFB000D9400B0041460B439B46534693401A0031
:10AFC000009B25499C46604403008C4663440093E3
:10AFD000002137E70323B14600900C26029311E7C6
:10AFE0000023009301330426002702930AE703237A
:10AFF000C3461E43032125E701331E4300220121DE
:10B0000020E700239A46802300271B03094A61E7B3
:10B01000802349461B03194200D1E2E059461942F8
:10B0200000D0DEE00B431B0317001B0BA246014AB6
:10B0300050E7C046FF07000001FCFFFF58F3000087
:10B04000FF030000FFFFFFFEFE070000FFFF0F8071
:10B050000DFCFFFF01F8FFFFF3030000D94500D905
:10B06000CBE000D1C6E03C0048460027009B013BF6
:10B0700000935B46160E1B021E43130298463304D0
:10B080001B0C9946310C0191FFF798F84A46424350
:10B090000B04210C050019438A4207D98919013D87
:10B0A0008E4203D88A4201D9851E8919881A0199CE
:10B0B000FFF784F809048C464A462104644642435B
:10B0C000090C030021438A4204D98919013B8E42AD
:10B0D00000D8F1E02D041D43AB464346891A424691
:10B0E000280C12041D0C5B46140C22001B041B0CC4
:10B0F0005A4303946B434443029568431B19150C50
:10B10000EB189C4203D980246402A44660441C0CC2
:10B1100015041B042D0C20185D19814277D373D0C0
:10B120000C1AA24A7D1BAF42BF419446009B7F424E
:10B130006344E01B1C00864200D1DBE00199FFF76D
:10B140003DF84A4642430B04290C070019438A4242
:10B1500007D98919013F8E4203D88A4201D9871E37
:10B160008919881A0199FFF729F809044A4689467E
:10B1700029044D464243090C030029438A4207D95A
:10B180008919013B8E4203D88A4201D9831E89194D
:10B190003F04891A3A00039F1A43380013041B0C1A
:10B1A000584381460298150C6F4343434543484634
:10B1B000000C8446DB1963449F4203D9802040027F
:10B1C0008446654448461F0C00041B04000C7D198E
:10B1D0001818A94200D284E000D17FE001231A436D
:10B1E00057E680234A461B0313431B031B0BAA4647
:10B1F0006F4A6FE6BA4200D935E74B46DC0758087C
:10B200007B081C43FF0734E70024AF4289D2474440
:10B210004745A4415B466442A4196418013BA64219
:10B220001ED2A0426DD800D1B6E0241A9B4678E722
:10B2300003005A46283B9A400027914688E6584624
:10B2400001F05CF8203072E603005246283B9A4039
:10B2500093460022B4E6504601F050F820309AE6BA
:10B26000A642E2D1B845DCD9341A9B4659E71F2BD8
:10B2700065DC504C0099A4465C46614408008C4053
:10B2800011008240D940501E82410C4314435A465B
:10B29000DA401300620709D00F222240042A05D0A9
:10B2A0002200141D9442894149425B181A0262D55A
:10B2B0000122002300270DE68A4200D80AE7831EF8
:10B2C000891907E70F231340042B00D1E6E5171D6A
:10B2D0009742924153429B44FA08E0E5002800D18E
:10B2E000D7E57118531EB14227D3A94215D358D0C0
:10B2F0001A0073E7002B00DC04E6012300229B44C4
:10B30000CDE502234744474589415B429C4649427B
:10B3100089190C19E344241A03E743465F004745A3
:10B320009B41B8465B429E19023A8919A94200D056
:10B3300054E7404500D051E7ABE51A00F6E71F217E
:10B340005F4649420C1BE740202B07D01A49009B5F
:10B350008C46634418005B4683401A43501E82416A
:10B360003A4307270023174009D00F21002311403B
:10B370001400042995D122005F075B021B0BD20841
:10B3800017430022A6E5802359461B030B431B03EA
:10B3900017001B0B064A9DE5BD42B2D89B46002410
:10B3A000BFE68045B9D31A00C3E7C046FF030000DB
:10B3B000FF0700001E0400003E040000F0B54F46E9
:10B3C0004646D6468446C0B58046194E18030F033C
:10B3D0004D00000B5C0082463F0B6D0DC90F91467E
:10B3E000640DDB0F0120B5420AD0B44203D0A54260
:10B3F00001D157450CD01CBC90469946A246F0BDE1
:10B4000066463E43F7D1AC42F5D154461443F2D1DF
:10B410000120C845EFD1994207D0002DEBD16346FA
:10B420001F433800471EB841E5E70020E3E7C04668
:10B43000FF070000F0B54F464646D6464D00C0B562
:10B440000E03C90F8A462C491F035C008046360B49
:10B450006D0D91463F0B640DDB0F8D421ED08C426B
:10B4600016D0002D1ED130438446002C01D13A4322
:10B4700023D06246002A1AD09A4529D0514602208C
:10B480000139084001381CBC90469946A246F0BDDF
:10B4900039001143E5D002204042F4E73043FAD1AD
:10B4A000AC420FD0002C0FD13A43E7D00CE0012280
:10B4B000013B934318000130E5E763460020002B71
:10B4C000E1D0DBE73A43E6D19A45D7D1A542D5DCB6
:10B4D000A54205DBBE42D1D808D00020BE42D2D260
:10B4E00050460123013898430130CCE7C845C5D800
:10B4F0000020C845F4D3C6E7FF070000F0B54F466B
:10B500004646D6464D00C0B50E03C90F8A462E49A1
:10B510001F035C008046360B6D0D91463F0B640D9A
:10B52000DB0F8D4218D08C4211D0002D18D1304342
:10B530008446002C1ED13A431CD163460020002BC8
:10B5400030D0514602200139084001382AE0390044
:10B550001143EAD0022025E03043FBD1AC4226D093
:10B56000002C26D13A4324D151460220013908400B
:10B57000013817E06246002A0FD09A45E1D1A54272
:10B5800005DBBE42DDD819D00020BE420AD25046AB
:10B59000012301389843013004E00122013B934329
:10B5A000180001301CBC90469946A246F0BD3A43B3
:10B5B000D0D19A45C5D1A542C3DCE0E7C845C0D883
:10B5C0000020C845E3D3EDE7FF070000F0B557467C
:10B5D000DE464E464546E0B5834606000F0348006A
:10B5E00087B092461D003F0B400DCC0F002800D1C4
:10B5F0006FE0DE4B984238D08023FF001B041F43CE
:10B60000730F3B430193DA4B0027994600239B4677
:10B61000F60081442B0369001B0B52469846490DE6
:10B62000ED0F002900D185E0D04B994200D173E0A5
:10B630004346DA0080231B0413435246CC48520F82
:10B6400084461343524600206144D20089442100BD
:10B65000694000918C46012149448A460F2F00D948
:10B6600090E0C449BF00CF59BF465B463B430193BE
:10B6700000D06AE102230827002681469B46C9E7DD
:10B6800032005846019B61460091022800D175E0C6
:10B69000032800D1FEE1012800D02CE1002300277F
:10B6A000002600253F032A0D3F0BB34812053A43FD
:10B6B00002401B051343009A5B00D1075B080B4354
:10B6C0003000190007B03CBC90469946A246AB46F4
:10B6D000F0BD5B463B43019300D12FE1002F00D129
:10B6E000A5E1380000F00AFE03000B3B1C2B00DD37
:10B6F00096E11D22D31A5A460100DA405E46083907
:10B700008F4013008E403B4301939C4B00271B1A34
:10B71000994600239B467DE7414653460B43934998
:10B720008C46E144002B00D01AE10222022017438C
:10B7300000228CE7134300D10DE14346002B00D1DA
:10B7400081E1404600F0DAFD02000B3A1C2A00DDE0
:10B7500072E10100434608398B4098461D239A1A2E
:10B760005346D3401A004346134352468A40494643
:10B77000081A824989468144002068E77B4B0027EC
:10B7800000268EE7140C1204120C1100370C36043C
:10B79000350C794328008C462E0060436044834674
:10B7A00056432100300C804658467943404402916C
:10B7B000844506D98846802149028C46E0444146AA
:10B7C00002913604010C360C00048B4681191E0CC4
:10B7D0001B041B0C0391190079438C462800754308
:10B7E0006544A8465843050C45447743A94203D90C
:10B7F000802149028C466744290C8C46390000049C
:10B80000000C2D042D186144AB4405915946049158
:10B8100001990F043F0C080C3900514342439046F4
:10B8200002008C46090C8B4662437C4344445C44D2
:10B83000A04503D98021490288464244210C88460C
:10B8400061460904090C8C4639005943434370434F
:10B850007E430F0CF6182404BE19644442448C46FF
:10B86000B34203D980235B0298464044029B614661
:10B870009846049B370443449B46AB45AD416B421D
:10B880000D0405992D0C8C467F196744FD18A846B8
:10B890005D462D19A542A44193466442A446C34483
:10B8A000DC448F42BF4198459B4193459241A4455A
:10B8B000A4415B427F421F43360C52426442BF198F
:10B8C0002243BF18624638184302D20D039913432E
:10B8D0006A020A43501E82416146ED0D2A434E0220
:10B8E0003243D90100D4B3E001265008324002436C
:10B8F000DE0732435B08224C5444002C62DD5107C2
:10B9000009D00F201040042805D0101D904292410C
:10B9100052429B180200D90104D580241948E40042
:10B92000034054441848844200DD27E75E075B0269
:10B93000D2081F0B630516435B0DB2E60023994640
:10B940000133042700269B4664E6032301978146C2
:10B950000C279B465EE6012201201743002276E673
:10B96000032303201F43434671E6C046FF07000040
:10B9700001FCFFFF98F30000FFFF0F800DFCFFFFAD
:10B98000FF030000FFFFFFFEFE07000000238027EB
:10B9900000933F030026434B83E6019B3200A446FD
:10B9A000584670E6AC466EE6802701993F0339425F
:10B9B0002DD03B422BD11F433F033F0B0095160078
:10B9C000384B6EE601252D1B382D00DD66E61F2D58
:10B9D00040DC35481C005044160082408440EE4054
:10B9E000501E824134431443EB40620709D00F22BA
:10B9F0002240042A05D02200141D94428041404276
:10BA00001B181A023ED501230027002649E680278D
:10BA1000019B3F031F433F033F0B0094214B40E634
:10BA200003005A46283B9A40002601926DE658468C
:10BA300000F064FC203057E603005246283B9A4051
:10BA40001300002293E6504600F058FC20307BE6BD
:10BA5000CA4650E71F201E004042041BE640202D2E
:10BA600003D0124C5444A3401A43501E8241324327
:10BA700007260027164009D00F200023104014008D
:10BA80000428B9D122005E075B021F0BD2081643BF
:10BA9000002306E680273F031F433F033F0B1600AA
:10BAA000004BFEE5FF0700001E0400003E040000FE
:10BAB000F8B557464E464546DE460C000903E0B54C
:10BAC000490A460F5F0031431E03DB0F760A9B468F
:10BAD000530F3343C84E6500C000E40FD2006D0D14
:10BAE000A24681467F0D9C469046B74200D1B9E000
:10BAF0005B46012673409B46EE1BA34500D183E0C5
:10BB0000002E63DD002F00D0B1E06346134300D167
:10BB100023E1731E002B00D0BAE1861A6346B042BF
:10BB200080410125C91A4042091A0B0200D447E19D
:10BB300049024B0A98464346002B00D189E1404612
:10BB400000F0DCFB0300083B1F2B00DD7CE1202222
:10BB50003000D21A4146D040994002009E400A432C
:10BB60009D4200DD6AE15D1B6B1C1F2B00DD94E133
:10BB7000202110003500C91A8E40DA408840DD408F
:10BB8000711E8E41110007222843002506433240D2
:10BB9000002A09D00F233340042B05D0331DB342B4
:10BBA000B641764289191E000B0200D43DE26A1CA0
:10BBB000914B55056D0D9A4200D119E18F4AF60857
:10BBC0000A40570752023743120B9BE0002E00D069
:10BBD000C5E06E1C7605760D012E00DC48E1674657
:10BBE000861ACB1BB042BF417F42B8461F00434676
:10BBF000FF1A3B00B8461B0200D55FE137439AD1DC
:10BC000000220024002579E0002E00DCFAE0002F5D
:10BC100000D18DE0784B9D4267D0802367461B049E
:10BC20001F43BC46382E00DC52E1634613435A1EC4
:10BC300093411E1886428041404209180B0200D4ED
:10BC4000BEE06D4B01359D4200D1D2E06B4A7308D6
:10BC50000A4001210E401E435108D30707221E430C
:10BC6000324095E71E00164300D045E740E7624B9F
:10BC70009D423AD0802367461B041F43BC46382EA2
:10BC800000DDEBE01F2E00DC3AE133006746203B8D
:10BC9000DF403B00202E05D04027BF1B6646BE403C
:10BCA000324390464646721E96413343DAE0002BFB
:10BCB00000D114E26346134300D168E180234E07AC
:10BCC000C008C9081B030643194208D06046C008D3
:10BCD000184204D163460100D2085E071643F30000
:10BCE0009946C900720F444D11434B46DE08424B42
:10BCF0004F073743CA089D4200D16EE012036D051D
:10BD0000120B6D0D00211203130B0A0D12051A43BD
:10BD10003B4B2D0513402B435B00E4075B0823439B
:10BD2000380019003CBC90469946A246AB46F8BD87
:10BD30006346134311D0731E002B00D007E1861811
:10BD40008642804161444042091801250B0237D5E3
:10BD500002257BE73E00614691463500C5E75C461B
:10BD6000002D00D0E1E00B000343F3D0731C00D1A1
:10BD7000ACE1214B9F4200D13AE1F343382B00DD87
:10BD80006FE11F2B00DD8CE120250E00ED1AAE4087
:10BD9000B0460600AA46DE40454635432E005546CD
:10BDA000D940A8406346451EA8415B1A9C463043D3
:10BDB000161AB242924163465242991A3D00B4E6C5
:10BDC00007223240002A00D0E4E60B4BF6084F076A
:10BDD0003743CA089D4200D090E73B00134300D18F
:10BDE000A6E180231B031A431203120B024D89E7BD
:10BDF00015000022002785E7FF070000FFFF7FFFF7
:10BE0000FFFF0F80002E00D0C7E06B1C5E05760D93
:10BE1000012E00DCF0E0C84DAB4200D1B9E085183E
:10BE20000A00854289416244494251180722CE07DF
:10BE30006D082E43490832401D00A9E6BF49ED1A9E
:10BE4000114007223240A3E6320028388240002603
:10BE500086E6300000F052FA203073E66346134362
:10BE60005A1E9341C61AB04280414042091A5CE60C
:10BE70000E00674606431743002D5ED1002E00D00A
:10BE8000F3E0002F00D11EE15C46614691462CE7AD
:10BE9000A94FBE427BD01E00F1E610001F3DE840D6
:10BEA000202B03D04021CB1A9A401643731E9E418B
:10BEB0000722064332400021002583E7161A634615
:10BEC000B2428041591A40420B1A98465C4632E60B
:10BED0001F2E00DDABE02027BB1B9A46634657466A
:10BEE000BB40994613004F46F3401F433B00574663
:10BEF000BA40571EBA4113436246F240891898E689
:10BF00002027BB1B9A4663465746BB409946130001
:10BF10004F46F3401F433B005746BA40571EBA41B5
:10BF200013436246F240891A9CE7834B9F425FD0DD
:10BF300080252D047342294320E7002E0CD1002FC9
:10BF400000D1D0E05C46614691467B4DCDE67A4F0C
:10BF5000BE421CD01E0065E6002F18D0C0084E0758
:10BF600006438020C9080003014208D06346DC086C
:10BF7000044204D12100DA46D2085E071643F300DA
:10BF8000994601245346C900720F11431C406A4D63
:10BF9000ABE61D0000220027B4E6002D59D10B00AE
:10BFA000034300D1D6E6731C00D1B2E0624B9F423E
:10BFB0001ED0F343382B6FDC1F2B00DD97E02025CC
:10BFC0000E00ED1AAE40B0460600AA46DE404546D9
:10BFD00035432E005546A840D940451EA8418C4403
:10BFE0000643B61896429241514261443D0025E60F
:10BFF0003D006146914678E60B000343002D00D0DA
:10C0000055E6002BF5D06346134300D16DE6861844
:10C010008642804161444042091800220B0200D44C
:10C02000D0E6464B01351940B2E5B1465DE6330036
:10C030006746203BDF403B00202E05D04027BF1B3A
:10C040006646BE40324390464646721E9641334392
:10C05000EFE5394B9F42CBD080252D047342294315
:10C06000A8E70843411E8841A2E6002F00D13CE624
:10C070006346861ACF1AB0429B415B42FB1A984630
:10C080001B024ED5161A6346B2429241591A5242C9
:10C09000891A5C4600227BE501430E00711E8E4129
:10C0A0009FE71D000E00203DEE40B046202B04D03F
:10C0B0004025EB1A99400843814648464346411EB5
:10C0C0008841184374E60022002417E6161A6346D6
:10C0D000B2429241591A5242891A3D0025E5614601
:10C0E0009146154D01E680220024120379E61D00D9
:10C0F0000E00203DEE40B046202B04D04025EB1A28
:10C100009940084381464E464346711E8E411E4368
:10C1100067E7861896429B4161445B42C9183D001F
:10C120008CE547463743CED007224146324049E6A8
:10C1300000273A00E6E5C046FF070000FFFF7FFF4B
:10C1400070B50C4E0D031C0349005B002D0B490D0F
:10C15000240B5B0DB14208D0064900208B4203D16D
:10C1600014432000441EA04170BD05430120002D52
:10C17000FAD1F1E7FF07000030B5144D0A034B0078
:10C18000120B5B0DC90F0024AB4211DD104CA34212
:10C1900010DC8024640322430E4CE41A1F2C0CDDB7
:10C1A0000D48C31ADA4013005C42002900D11C007C
:10C1B000200030BD094BCC18FAE7094DE040AC46F1
:10C1C00063449A4013000343EEE7C046FE030000B9
:10C1D0001D0400003304000013040000FFFFFF7F74
:10C1E000EDFBFFFF70B500282DD0C317C5185D40CB
:10C1F000C40F280000F082F8154B1B1A5B055B0D7D
:10C200000A2815DD0B38854000222D032D0B002157
:10C2100010002D030A0D2D0B12052A430D4D1B0591
:10C220002A4013435B00E4075B082343190070BDF9
:10C2300002002900153291400A000B21081AC5405E
:10C240002D032D0BE3E70024002300250022DEE769
:10C250001E040000FFFF0F804100090E4B1C70B54B
:10C26000DBB24602750AC40F012B14DDE0239B00EC
:10C270006D07360BCB1800210A0D280012051C4D46
:10C2800032435B052A405B0813435B00E4075B080D
:10C290002343190070BD002914D1002D1ED02800A1
:10C2A00000F02CF80A281CDC0B232A001B1ADA40A9
:10C2B000030015339D400F4B12031B1A5B05160B31
:10C2C0005B0DD8E7002D06D0320B802636036D07B4
:10C2D0001643094BCFE7084B0026CCE70023002686
:10C2E000C9E703002A000B3B9A400025E3E7C0465C
:10C2F000FFFF0F8089030000FF0700001C210123BE
:10C300001B04984201D3000C10391B0A984201D338
:10C31000000A08391B09984201D30009043902A216
:10C32000105C40187047C04604030202010101017D
:10C33000000000000000000030B51C00094B0500A3
:10C340001B6885B0D868084B002A01D1074B1A003A
:10C350000292019300912B002200054900F026F87B
:10C3600000F0A6FD8C000020D8F300001AE00000C9
:10C37000E5F30000014B18687047C0468C000020B0
:10C38000084B10B50400002B02D0002100E000BFD4
:10C39000054B1868836A002B00D09847200001F0F5
:10C3A0005DFBC0460000000014F400000EB403B5AD
:10C3B000010003AB044804CB0068019300F076F859
:10C3C00002B008BC03B018478C00002070B50026EE
:10C3D0000C4D0D4C641BA410A64209D1002601F09F
:10C3E0003FFB0A4D0A4C641BA410A64205D170BD48
:10C3F000B300EB5898470136EEE7B300EB58984787
:10C400000136F2E75C0200205C0200205C020020A2
:10C410006C020020002310B59A4200D110BDCC5C04
:10C42000C4540133F8E710B5884202D98B189842FA
:10C4300003D3002307E08B5C8354013AFBD210BD89
:10C44000CC5CC45401339A42FAD1F8E703001218C5
:10C45000934200D1704719700133F9E7936810B522
:10C46000013B9360002B04DA9469A34207DB0A299D
:10C4700005D01368581C10601970080010BD00F03A
:10C480004BFC0100F9E7F8B506000F001400D518C1
:10C49000AC4201D1002007E021783A003000FFF7DC
:10C4A000DDFF0134431CF3D1F8BD0000F0B59FB0AF
:10C4B00002900F0016000593002805D083690493AD
:10C4C000002B01D100F0F4FD7B4B9F425BD1029B1E
:10C4D0005F68BB891B0762D53B69002B5FD00023D7
:10C4E00006AC6361203363761033A37635002B7876
:10C4F000002B01D0252B5CD1AB1B04930CD0320058
:10C5000039000298FFF7BFFF431C00D1C4E0626905
:10C51000049B9446634463612B78002B00D1BBE0FD
:10C52000012200235242626002A9543252186E1C4A
:10C530002360E360A3601370A365317805225F4830
:10C5400000F0D4FE751C002835D12268D30604D52E
:10C55000532302A95B1820211970130704D5532314
:10C5600002A95B182B21197033782A2B2CD03500A7
:10C5700000210A20E3682A786E1C303A092A64D91F
:10C5800000292ED026E04E4B9F4202D1029B9F688D
:10C590009FE74C4B9F429CD1029BDF6899E7390093
:10C5A000029800F00FFC002899D0012040421FB0F3
:10C5B000F0BD01359BE7414B2268C01A012383403F
:10C5C000134323602E00B8E7059B191D1B680591D6
:10C5D000002B01DB099304E05B42E3600223134379
:10C5E00023602B782E2B0AD16B782A2B35D1059B13
:10C5F00002351A1D1B680592002B2BDB0793324E68
:10C6000029780322300000F071FE002806D0402374
:10C61000801B83402268013513432360297806225A
:10C620002A486E1C217600F061FE00283AD0284B83
:10C63000002B25D10722059B07339343083305932D
:10C640006369039A9B18636150E7434301219B1878
:10C65000350090E701235B42D0E700230A201A004F
:10C660000135636029786E1C3039092903D9002B04
:10C67000C5D00792C3E74243012352183500F1E7C2
:10C6800005AB00933A00134B2100029800E000BF75
:10C690000390039B0133D3D1BB895B0600D584E7AC
:10C6A0000B9884E705AB00933A000A4B21000298EF
:10C6B00000F080F8ECE7C0466CF4000018F40000CD
:10C6C0008CF400004CF400001EF4000022F4000082
:10C6D0000000000087C40000F7B5150001938A68C8
:10C6E0000B6900900C00934200DA130022002B60CB
:10C6F00043321278002A01D001332B6023689B0655
:10C7000002D52B6802332B60062723681F4027D0F1
:10C71000230043331B785A1E93412268920630D47B
:10C720002200019943320098089EB047431C25D04F
:10C73000062320682A68E16803400025042B03D102
:10C740008D1AEB43DB171D40A3682269934201DD7C
:10C750009B1AED180027BD4220D1002010E00137C0
:10C76000E3682A689B1ABB42D2DD220001231932FA
:10C7700001990098089EB047431CF0D10120404227
:10C78000FEBD3020E1184331087021005A1C4531AC
:10C790000978A218433202331170C1E72200012345
:10C7A0001A3201990098089EB047431CE6D0013721
:10C7B000D1E70000F0B589B004920A004332059336
:10C7C000039002920A7E0C000E9B6E2A00D186E036
:10C7D0001FD8632A33D008D8002A00D18CE0582A09
:10C7E0004DD0250042352A7030E0642A01D0692AF4
:10C7F000F7D1196825680A1D280629D508681A6026
:10C80000002803DA2D23029A404213706B4E0A2748
:10C810004FE0732A74D008D86F2A1FD0702AE0D155
:10C82000202209680A43226003E0752A16D0782A7C
:10C83000D7D12200782145321170614E22E02500C7
:10C840001A684235111D196013682B70012365E0C9
:10C8500008681A606906D3D500B2D1E7196825685F
:10C86000081D186008682E0605D5544E08276F2A43
:10C870001BD00A2719E06D06F7D580B2F5E74531E0
:10C880004E4E0A7018682268011D0068196015066E
:10C8900021D5D30702D520231A4322601027002870
:10C8A00003D1202322689A432260230000224333CD
:10C8B0001A706368A360002B58DB0422216891433F
:10C8C0002160002854D1029D002B5AD025003378D6
:10C8D00042352B7055E05506DBD580B2D9E71A6892
:10C8E0000D68101D4969186013682E0601D519607E
:10C8F00002E06D06FBD519800023029D23614FE005
:10C900001A68111D1960156800216268280000F07E
:10C91000EDFC002801D0401B6060636823610023A8
:10C92000029A13703CE023692A0004990398059D3C
:10C93000A847431C3ED023689B0715D4079BE0689B
:10C94000984239DA180037E022000123193204999D
:10C950000398059EB047431C2CD00135E368079A25
:10C960009B1AAB42F0DCE9E70025F7E70028ADD0E1
:10C97000029D3900FDF722FC735C013D2B700028FD
:10C98000F7D1082F09D12368DB0706D56368226930
:10C99000934202DC3023013D2B70029B5B1B236121
:10C9A000059B07AA00932100049B0398FFF794FEC0
:10C9B000431CB8D10120404209B0F0BD29F4000069
:10C9C0003AF400000D4B70B51C680500A36B002BFA
:10C9D0000FD1182000F06EFC094BA0630360094BD7
:10C9E00001224360084B83600B2383810023026193
:10C9F00043610022A36B1D615A6170BD8C00002051
:10CA00000E33CDAB34126DE6ECDE0500124B10B5E3
:10CA10001C68A36B002B0FD1182000F04BFC0F4BB0
:10CA2000A06303600E4B012243600E4B83600B2317
:10CA30008381002302614361A46B0B4A2069616911
:10CA40000A4BFDF7F7FC01220023801859412061B1
:10CA500061614800400810BD8C0000200E33CDAB52
:10CA600034126DE6ECDE05002D7F954C2DF4515807
:10CA70000CB430B5164B9DB00C1E1D6808DA8B2324
:10CA800001202B6040421DB030BC08BC02B01847EA
:10CA9000822302A99B008B810023029008619C42A3
:10CAA00000D0631E8B604B6101235B42CB81209AD7
:10CAB00021AB2800019300F055FD431C01DA8B23C4
:10CAC0002B60002CDFD00023029A1370DBE7C046F6
:10CAD0008C0000200EB400B50B499CB01DAB029039
:10CAE0000690079104910948094904CB0591006813
:10CAF00002A9019300F036FD0023029A13701CB0C6
:10CB000008BC03B01847C046FFFFFF7F8C00002021
:10CB10000802FFFF020010B51378541C002B05D14A
:10CB2000CC5CD4540133002CFAD110BD2200F3E7C1
:10CB3000C9B20378002B04D08B4200D1704701307A
:10CB4000F7E74B42594149420840F7E702780B7832
:10CB5000002A03D0013001319A42F7D0D01A704731
:10CB60000023C25C0133002AFBD1581E704700230A
:10CB700030B59A420AD0013AC45CCD5CAC4204D1D3
:10CB8000934202D00133002CF6D1631B180030BD54
:10CB900030B50500002A00D130BD0C78013A6B1C7D
:10CBA0002C700131002C05D19A189A42F4D01C70D7
:10CBB0000133FAE71D00EDE710B50378002B0FD124
:10CBC0000B785A4253415B42184010BD0023CA5CA7
:10CBD000002AFAD0C45C944201D10133F7E7013056
:10CBE0000378002BF2D11800EFE70000F0B51F002A
:10CBF0000E0087B00590019102920C98347800F0F5
:10CC0000EAFA082200194378751C134036D12D2CFE
:10CC100036D1B51C74780126002F62D0102F09D1AF
:10CC2000302C07D120222B789343582B54D1102736
:10CC30006C7802352D4B3900F31818000393FDF77B
:10CC4000BDFA049101210023494202008C461800DC
:10CC50002100303909291AD80C00A74223DD591CBC
:10CC600009D06346824206D302D10499A14202DB75
:10CC70000123784320182C780135E9E72E00BCE722
:10CC80002B2C01D01E00C7E7B51C7478FAE72100F1
:10CC90004139192901D8373CDFE7210061391929C9
:10CCA00001D8573CD9E75A1C08D1059A23331360A1
:10CCB000029B0398002B09D107B0F0BD002E00D0D5
:10CCC0004042029A002AF7D0002B01D06B1E01933C
:10CCD000029B019A1A60EFE73024002FAAD108279F
:10CCE000A8E7302C9ED00A27A4E7C046FFFFFF7FAD
:10CCF00037B51300064A05001068046A002C00D1FD
:10CD0000044C0A0000942900FFF770FF3EBDC046A6
:10CD10008C000020F0000020F8B505000E00140083
:10CD2000002804D08369002B01D100F0C1F9224B07
:10CD30009C422DD16C68A369A360A3891B0731D5E0
:10CD40002369002B2ED023682269F7B2981A6369F1
:10CD5000F6B2834205DC2100280000F03BF90028F0
:10CD600026D1A3680130013BA36023685A1C2260CE
:10CD70001F706369834204D0A389DB071AD50A2E8A
:10CD800018D12100280000F025F9002812D00FE06A
:10CD90000A4B9C4201D1AC68CDE7094B9C42CAD1F9
:10CDA000EC68C8E72100280000F00CF80028CAD081
:10CDB000012676423000F8BD6CF400008CF40000CF
:10CDC0004CF40000364B70B51D6806000C00002DB9
:10CDD00005D0AB69002B02D1280000F069F9314B76
:10CDE0009C420FD16C680C23E25E93B219072DD4DC
:10CDF000D90611D409230120336037331343A381AB
:10CE0000404270BD284B9C4201D1AC68EBE7274BF8
:10CE10009C42E8D1EC68E6E75B0713D5616B00291B
:10CE200008D023004433994202D0300000F06AFA5F
:10CE3000002363632422A3899343A38100236360B7
:10CE4000236923600823A2891343A3812369002B4C
:10CE50000BD1A0218022A389890092000B4093422C
:10CE600003D02100300000F0E1F90123A289134032
:10CE700011D00023A36063695B42A3610020236992
:10CE80008342BED10C23E25E1306BAD5402313437E
:10CE9000A3810138B5E7920700D46369A360EDE789
:10CEA0008C0000206CF400008CF400004CF40000B6
:10CEB00010B5062000F090FC012000F0CFFD00002E
:10CEC000F7B58A8905000C00130760D44B68002B66
:10CED00004DC0B6C002B01DC0020FEBDE76A002F98
:10CEE000FAD000232E682B6080235B01216A1A4050
:10CEF00034D0606DA3895B0706D56368C01A636B85
:10CF0000002B01D0236CC01A0200216A00232800E4
:10CF1000E76AB847A189431C06D12B681D2B30D87E
:10CF20002B4ADA40D3072CD50023636023692360A2
:10CF3000CB0405D5431C02D12B68002B00D16065C2
:10CF4000616B2E600029C7D023004433994202D080
:10CF5000280000F0D7F900206063BEE70123280015
:10CF6000B847431CC6D12B68002BC3D01D2B01D062
:10CF7000162B01D12E60AFE74023A2891343A38172
:10CF8000ABE740230B430120A3814042A5E70F6993
:10CF9000002FA1D00B680F60DB1B019300239207C9
:10CFA00000D14B69A360019B002B00DC94E7019B3F
:10CFB0003A00216A2800A66AB047002803DC402313
:10CFC000A2891343DFE7019B3F181B1A0193EAE78D
:10CFD000010040200B6970B505000C00002B01D149
:10CFE000002070BD002804D08369002B01D100F01F
:10CFF0005FF80B4B9C4209D16C680C22A35E002B9E
:10D00000EED021002800FFF75BFFEAE7054B9C42CA
:10D0100001D1AC68F1E7044B9C42EED1EC68ECE73F
:10D020006CF400008CF400004CF40000002310B5F8
:10D03000040003604360836081814366C2810361B1
:10D0400043618361190008225C30FFF7FFF9054B4B
:10D0500024626362044BA362044BE362044B2363C8
:10D0600010BDC04619D8000041D8000079D8000092
:10D07000A5D8000010B5024900F08CF810BDC046DC
:10D08000D5CF000070B568254A1E55430E00290013
:10D09000743100F081F9041E08D000212A000160DB
:10D0A00046600C30A0606832FFF7D0F9200070BDF8
:10D0B000836913B50400002B28D18364C36403651E
:10D0C000134B144A1B6882620193984201D10123D9
:10D0D0008361200000F020F86060200000F01CF860
:10D0E000A060200000F018F80022E06004216068D1
:10D0F000FFF79CFF01220921A068FFF797FF02229A
:10D100001221E068FFF792FF0123A36113BDC0461F
:10D1100014F4000075D00000F8B51C4B07001E6821
:10D12000B369002B02D13000FFF7C2FF4836B46864
:10D130007368013B04D53368002B07D03668F6E7E7
:10D140000C22A55E002D0DD06834F2E704213800D2
:10D15000FFF798FF30600028F0D10C2304003B60FB
:10D160002000F8BD20000A4B656625606560A5605B
:10D17000E36025616561A561082229005C30FFF745
:10D1800065F96563A563A564E564E9E714F4000047
:10D190000100FFFFF7B504000700002601914834A5
:10D1A000002C01D13000FEBD6368A5680093009B90
:10D1B000013B009301D52468F2E7AB89012B08D924
:10D1C0000E22AB5E013304D029003800019B984742
:10D1D00006436835EBE7EC300068704770B50E0029
:10D1E0001D000E23C95E96B01400002907DA002343
:10D1F0002B60B3891B0611D48023DB000FE06A4645
:10D2000000F088FB0028F2DBF022019B12021340A1
:10D21000054A9B185A4253412B60EDE740230020FA
:10D22000236016B070BDC04600E0FFFFF7B50226D0
:10D230008B8905000C00334206D02300473323605E
:10D24000236101236361F7BD01AB6A46FFF7C6FFA7
:10D2500000990700280000F09FF8002808D10C2250
:10D26000A35E9A05EFD4032293431E43A681E4E70D
:10D270000F4BAB628023A28920601343A381009BE4
:10D2800020616361019B002B0DD00E23E15E28001D
:10D2900000F052FB002806D00322A38993431A0012
:10D2A00001231343A381A0893843A081CBE7C04663
:10D2B00075D0000010B5034B0100186800F06CF841
:10D2C00010BDC0468C00002082B0002900D101A909
:10D2D000101E06D0002B06D013780B601078431E6A
:10D2E000984102B0704702204042FAE7C9B2821862
:10D2F000904201D10020704703788B42FBD001306F
:10D30000F6E7000070B50500002910D00C1F236857
:10D31000002B00DAE418280000F034FB1D4A1368E3
:10D32000002B05D163601460280000F02CFB70BD59
:10D33000A34209D9216860188342F3D118685B6859
:10D3400041182160EEE713005A68002A01D0A2427A
:10D35000F9D919685818A0420BD120680918581833
:10D3600019608242E0D110685268411819605A6011
:10D37000DAE7A04202D90C232B60D5E721686018B8
:10D38000824203D1106852684118216062605C607B
:10D39000CAE7C046341C0020032370B5CD1C9D4352
:10D3A000083506000C2D1ED20C25A9421DD83000D0
:10D3B00000F0E8FA254A14682100002919D1244C0C
:10D3C0002368002B03D1300000F0CAF92060290047
:10D3D000300000F0C5F9431C2BD10C233000336022
:10D3E00000F0D1FA03E0002DDFDA0C2333600020D7
:10D3F00070BD0B685B1B19D40B2B03D90B60CC18C9
:10D40000256003E04B688C420DD11360300000F0C2
:10D41000BAFA200007220B30231D9043C31AE7D02D
:10D420005A42E250E4E763600C00EFE70C00496801
:10D43000C3E70323C41C9C43A042E1D0211A30005F
:10D4400000F08EF9431CDBD1C7E7C046341C002036
:10D45000381C0020F8B507000D001600002905D182
:10D460001100FFF799FF04002000F8BD002A03D146
:10D47000FFF748FF3400F7E700F086FA2C00B042CF
:10D48000F2D231003800FFF787FF041EECD02900EC
:10D490003200FEF7BFFF29003800FFF733FFE3E754
:10D4A000F0B58E6885B007000C00039201939E4290
:10D4B0003CD890238A89DB001A4234D003250969BD
:10D4C00023685B1A0293636902985D43EB0F5D1951
:10D4D000019B6D1001331B18AB4200D91D00530591
:10D4E00032D529003800FFF757FF061E09D10C235B
:10D4F0003B6040230120A28940421343A38105B031
:10D50000F0BD029A2169FEF785FFA389144A1A40EB
:10D5100080231343A381029B2661F6182660656170
:10D52000019EED1AA560019B9E4200D9019E32002A
:10D5300003992068FEF777FFA36800209B1BA36078
:10D5400023689E192660DAE72A003800FFF782FF79
:10D55000061EE0D121693800FFF7D4FEC7E7C046B8
:10D560007FFBFFFFF0B59FB0029005938B890F0002
:10D5700016001B0611D50B69002B0ED14021FFF7B9
:10D580000BFF38603861002805D10C23029A01385E
:10D5900013601FB0F0BD40237B61002306AC6361C4
:10D5A000203363761033A37635002B78002B01D01F
:10D5B000252B46D1AB1B04930CD0320039000298C6
:10D5C000FFF76EFF431C00D1AEE06269049B9446F6
:10D5D000634463612B78002B00D1A5E00122002376
:10D5E0005242626002A9543252186E1C2360E360FA
:10D5F000A3601370A365317805225448FFF776FEC7
:10D60000751C00281FD12268D30604D5532302A914
:10D610005B1820211970130704D5532302A95B1846
:10D620002B21197033782A2B16D0350000210A20BF
:10D63000E3682A786E1C303A092A4ED9002918D09E
:10D6400010E00135B1E7414B2268C01A0123834045
:10D65000134323602E00CEE7059B191D1B6805911F
:10D66000002B01DB099304E05B42E36002231343D8
:10D6700023602B782E2B0AD16B782A2B35D1059B72
:10D6800002351A1D1B680592002B2BDB0793304EC9
:10D69000297803223000FFF729FE002806D0402316
:10D6A000801B8340226801351343236029780622BA
:10D6B00028486E1C2176FFF719FE00283CD0264B27
:10D6C000002B25D10722059B07339343083305938D
:10D6D0006369039A9B18636166E7434301219B18C2
:10D6E0003500A6E701235B42D0E700230A201A0099
:10D6F0000135636029786E1C3039092903D9002B64
:10D70000C5D00792C3E74243012352183500F1E721
:10D7100005AB00933A00114B2100029800E000BFD6
:10D720000390039B0133D3D1BB890B985B0600D4D4
:10D730002FE7012040422CE705AB00933A00074B4E
:10D7400021000298FFF736F8EAE7C04618F4000017
:10D750001EF4000022F4000000000000A1D400002C
:10D76000002370B5064C05000800236000F060F946
:10D77000431C03D12368002B00D02B6070BDC04632
:10D78000C82F002070B504000D001F2904D91623EE
:10D7900003600120404270BD436C002B04D08A001E
:10D7A0009B181A68002A08D1200000F031F82A00DE
:10D7B0000100200000F01AF8EDE70020012AEAD06D
:10D7C000511C03D1162301302360E4E70024280014
:10D7D0001C6090472000DEE710B5034B010018687D
:10D7E000FFF7D0FF10BDC0468C000020002370B5AD
:10D7F000064C050008001100236000F001F9431CED
:10D8000003D12368002B00D02B6070BDC82F0020EF
:10D8100010B500F0E5F810BD70B50C000E25495F9D
:10D8200000F0BAF8002803DB636D1B18636570BD58
:10D83000A389024A1340A381F9E7C046FFEFFFFF27
:10D84000F8B51F008B8905000C001600DB0505D517
:10D850000E23C95E0022022300F080F8A389054A46
:10D8600028001340A38132000E23E15E3B0000F04C
:10D870002BF8F8BDFFEFFFFF70B50C000E25495FD8
:10D8800000F06CF8A389421C03D1054A1340A38120
:10D8900070BD802252011343A3816065F8E7C04642
:10D8A000FFEFFFFF10B50E23C95E00F021F810BD99
:10D8B0000B1E04D0FF2A04D98A2303608B3B180077
:10D8C00070470A700123FAE770B5050008001100DF
:10D8D0000022064C22601A0000F0B8F8431C03D165
:10D8E0002368002B00D02B6070BDC046C82F0020DD
:10D8F000002370B5064C05000800236000F060F8B6
:10D90000431C03D12368002B00D02B6070BDC046A0
:10D91000C82F0020002370B5064C05000800110038
:10D92000236000F055F8431C03D12368002B00D07E
:10D930002B6070BDC82F0020002370B5064C050079
:10D940000800236000F054F8431C03D12368002B27
:10D9500000D02B6070BDC046C82F002070B50500F8
:10D96000080011000022064C22601A0000F050F856
:10D97000431C03D12368002B00D02B6070BDC04630
:10D98000C82F0020704770470B1F1B68181F002B03
:10D9900001DA0B58C018704770B505000800110077
:10D9A0000022064C22601A0000F03AF8431C03D112
:10D9B0002368002B00D02B6070BDC046C82F00200C
:10D9C00058220120014B40421A607047C82F0020A6
:10D9D00058220120014B40421A607047C82F002096
:10D9E00058220120014B40421A607047C82F002086
:10D9F0005822024B00201A607047C046C82F0020F2
:10DA000058220120014B40421A607047C82F002065
:10DA100058220120014B40421A607047C82F002055
:10DA200058220120014B40421A607047C82F002045
:10DA3000044A1368002B00D1034B1818106018001B
:10DA40007047C0463C1C0020D02F002058220120E7
:10DA5000014B40421A607047C82F0020FEE7C046C5
:10DA6000F8B5C046F8BC08BC9E467047F8B5C0463D
:10DA7000F8BC08BC9E4670476461746100000000F9
:10DA80000EDB0000EF01000017DB0000E3020000E6
:10DA90001FDB0000090B000026DB0000450C000026
:10DAA0002BDB00000905000031DB0000F50600005B
:10DAB0003CDB00005303000041DB00009D0E000032
:10DAC0004DDB00001F02000057DB0000D5090000FD
:10DAD00065DB00009506000072DB00008108000095
:10DAE0007EDB00005506000072616E646F6D0061A0
:10DAF0006C6C006C61737400300066616C7365005F
:10DB00007472756500252E3135732E2E2E006D61D1
:10DB10006B654C697374006164644C617374006478
:10DB2000656C657465006A6F696E0073706C69740A
:10DB300000636F707946726F6D546F0066696E6432
:10DB4000006A6F696E537472696E677300756E69EF
:10DB5000636F6465417400756E69636F64655374C7
:10DB600072696E67006E65774279746541727261A1
:10DB700079006173427974654172726179006672ED
:10DB800065654D656D6F727900000000F1DB000086
:10DB900091130000F6DB0000AF1300001FDB000054
:10DBA000B3130000FCDB00009513000006DC00004E
:10DBB000B71300000FDC0000BB13000019DC0000ED
:10DBC000BF13000024DC0000C313000030DC0000A1
:10DBD0009913000039DC0000A713000043DC0000AB
:10DBE0009D1300004EDC0000AB13000066696C65FD
:10DBF000006F70656E00636C6F736500656E644FD7
:10DC00006646696C6500726561644C696E65007298
:10DC1000656164427974657300617070656E644C0F
:10DC2000696E6500617070656E6442797465730039
:10DC300066696C6553697A650073746172744C69C6
:10DC40007374006E657874496E4C697374007379EF
:10DC50007374656D496E666F0000000084170000E4
:10DC600094170000AE1700002A1800006218000088
:10DC700096180000CE180000F418000038190000B3
:10DC80007A190000CE190000121A0000741A000060
:10DC9000BC1A0000E21A00001A1B0000601B000002
:10DCA000861B0000B41B0000E21B0000BE32000017
:10DCB0009A1C00006C1D0000E21D0000521E0000B6
:10DCC0009E1E0000BE1E0000E01E00003820000066
:10DCD0007C200000F42000002221000054210000DC
:10DCE00086210000062200006E220000CA220000E9
:10DCF000282300009A2300000C2400006824000060
:10DD0000C2240000F8240000482500008E250000F1
:10DD1000D62500002A2600007E260000BC26000032
:10DD2000282700005E270000A6270000EE2700003D
:10DD30003628000070280000B828000008290000DC
:10DD40006A2A0000B41B00001A1B000070290000A2
:10DD500084170000A6290000D2290000082A00002C
:10DD6000342A000084170000841700008417000084
:10DD700084170000E62A0000282B00006E2B00000C
:10DD8000BE2B0000EA2B0000622C0000B42C000027
:10DD9000182D000084170000841700003C2D00009F
:10DDA0006C2D00009C2D0000D22D0000FC2D0000E9
:10DDB000322E00005C2E0000842E0000AC2E0000ED
:10DDC000DC2E00000C2F0000362F0000602F00001A
:10DDD000902F0000BA2F0000841700008417000065
:10DDE000841700008417000084170000EA2F000049
:10DDF00016300000423000006E3000009A30000003
:10DE0000D030000010310000463100007C310000AD
:10DE1000A8310000D43100000A320000841700004D
:10DE20008417000084170000841700008417000086
:10DE30008417000084170000841700008417000076
:10DE40008417000084170000841700003632000099
:10DE500036320000583300008E3300005B2564200A
:10DE60006974656D206C6973745D00282564206297
:10DE7000797465732900286F626A65637420747908
:10DE800070653A2025642900537461636B20756EB8
:10DE9000646572666C6F7700626F6F6C65616E00AF
:10DEA0006E756D62657200737472696E67006C697D
:10DEB0007374006279746520617272617900000088
:10DEC00007000000030000004ADF0000B534000036
:10DED00052DF0000653500005BDF00008F37000077
:10DEE00064DF0000B93400006DDF000093370000EC
:10DEF00075DF00007D3700007EDF0000AD360000DA
:10DF000089DF00001D39000094DF0000F5350000B6
:10DF10009FDF000091380000ABDF000059360000A1
:10DF2000B7DF0000ED380000000000000100000035
:10DF30000200000003000000040000000A000000CE
:10DF40006D6963726F3A62697400686173546F6ED1
:10DF50006500706C6179546F6E650068617353651C
:10DF600072766F00736574536572766F00646163D7
:10DF7000496E6974006461635772697465007371F6
:10DF80007561726557617665007365745573657266
:10DF90004C454400616E616C6F675265616400615D
:10DFA0006E616C6F67577269746500646967697444
:10DFB000616C52656164006469676974616C577271
:10DFC00069746500474320746F6F6B20256420756A
:10DFD000736563733B206672656520256420776FE7
:10DFE000726473003C496E74656765723E003C4C18
:10DFF0006973743E003C4F626A6563743E003C4244
:10E0000079746541727261793E000D0A564D205057
:10E01000616E69633A2025730D0A006D69736300B0
:10E0200055E00000ED4300005EE000007D4300008D
:10E0300062E00000D14200006AE000007742000088
:10E0400074E000000D42000080E000000F4100007D
:10E050006E756C6C00686578546F496E74007369F6
:10E060006E006A736F6E476574006A736F6E436FFC
:10E07000756E74006A736F6E56616C7565417400DD
:10E080006A736F6E4B6579417400000050E10000C7
:10E090005944000058E100005D44000062E10000C6
:10E0A0007B4400006BE100008544000076E1000045
:10E0B0008F44000082E100009944000090E10000DC
:10E0C000A344000098E10000AD4400009EE1000080
:10E0D000B7440000B3E10000C1440000C8E1000003
:10E0E000CB440000D4E10000D5440000E4E100008E
:10E0F000DF440000F0E10000E9440000FDE1000021
:10E10000F34400000CE20000FD4400001FE20000A8
:10E110000745000035E200001145000041E2000023
:10E120001B45000051E200002545000060E20000B0
:10E130002F4500006EE200003945000076E2000045
:10E14000674400007EE20000714400006E657400C8
:10E1500068617357694669007374617274576946E0
:10E16000690073746F70576946690077696669530F
:10E170007461747573006D7949504164647265739C
:10E1800073007374617274535349447363616E0016
:10E1900067657453534944006D794D414300687479
:10E1A00074705365727665724765745265717565F2
:10E1B000737400726573706F6E64546F487474701A
:10E1C000526571756573740068747470436F6E6E18
:10E1D00065637400687474704973436F6E6E656331
:10E1E0007465640068747470526571756573740049
:10E1F00068747470526573706F6E736500776562D2
:10E20000536F636B65745374617274007765625306
:10E210006F636B65744C6173744576656E740077DB
:10E220006562536F636B657453656E64546F436CC2
:10E2300069656E74004D515454436F6E6E6563741E
:10E24000004D5154544973436F6E6E656374656439
:10E25000004D515454446973636F6E6E656374006E
:10E260004D5154544C6173744576656E74004D5134
:10E270005454507562004D515454537562004D51C1
:10E280005454556E737562001A1B1C03040607096B
:10E290000A171819000000000008080800080A4AB8
:10E2A0004000000A5FEA5FEA0ED92ED36E193244AD
:10E2B00089330C924C924D0808000000048808082D
:10E2C000040804848488000A448A4000048EC480C0
:10E2D000000000048800000EC000000000080001DB
:10E2E000224488100C9252524C048C84848E1C82DE
:10E2F0004C901E1EC244924C06CA525FE21FF01E92
:10E30000C13E02448ED12E1FE24488100ED12ED180
:10E310002E0ED12EC4880008000800000480048856
:10E320000244880482000EC00EC008048244880E95
:10E33000D126C0040ED135B36C0C925ED2521C9221
:10E340005C925C0ED010100E1C9252525C1ED01CBF
:10E35000901E1ED01C90100ED013712E12525ED241
:10E36000521C8808081C1FE242524C125498149206
:10E37000101010101E113B75B131113935B3710CED
:10E380009252524C1C925C90100C92524C861C92F1
:10E390005C92510ED00C825C1FE484848412525231
:10E3A000524C1131312A44113135BB7112524C9209
:10E3B00052112A4484841EC488101E0EC808080EF8
:10E3C00010080482410EC242424E048A40000000FE
:10E3D0000000001F0804800000000ED2524F1010F1
:10E3E0001C925C000ED0100E02424ED24E0C925C7B
:10E3F000900E06C81C88080ED24EC24C10101C92FB
:10E40000520800080808024002424C101498149266
:10E410000808080806001B75B131001C9252520012
:10E420000C92524C001C925C90000ED24EC2000E18
:10E43000D010100006C8049808080EC80700125231
:10E44000524F0011312A4400113135BB00124C8C5F
:10E450009200112A4498001EC4881E06C48C84862B
:10E46000080808080818080C881800000C836000C9
:10E470000000000001000000020000000300000096
:10E480000400000005000000060000000700000076
:10E4900008000000090000000A0000000B00000056
:10E4A0000C0000000D0000000E0000000F00000036
:10E4B0001000000012000000140000001600000010
:10E4C000180000001A0000001C0000001E000000E0
:10E4D00020000000230000002600000029000000AA
:10E4E0002C0000002F000000320000003600000069
:10E4F0003A0000003E00000042000000460000001C
:10E500004B00000050000000550000005A000000C1
:10E5100061000000680000006F000000760000004D
:10E520007D000000840000008B00000092000000CD
:10E5300099000000A0000000A7000000AE0000004D
:10E54000B5000000BC000000C3000000CA000000CD
:10E55000D1000000D8000000DF000000E60000004D
:10E56000ED000000F4000000FB000000FF000000D0
:10E57000C0E500005D450000CBE50000D54A000085
:10E58000D5E5000015470000E2E500004548000021
:10E59000E9E5000095480000F2E50000E5480000CC
:10E5A000FEE50000DD4700000FE60000D549000051
:10E5B0001CE600006D470000646973706C617900AF
:10E5C0006C696768744C6576656C006D624469734C
:10E5D000706C6179006D62446973706C61794F662B
:10E5E00066006D62506C6F74006D62556E706C6F7A
:10E5F00074006D62447261775368617065006D628A
:10E600005368617065466F724C6574746572006E14
:10E61000656F506978656C53656E64006E656F5008
:10E620006978656C53657450696E004E6F7420652F
:10E630006E6F75676820726F6F6D206576656E20EE
:10E64000616674657220636F6D70616374696F6E6B
:10E6500000436F6D70616374656420466C6173681C
:10E6600020636F64652073746F72650A256420628D
:10E6700079746573207573656420282564252529C0
:10E68000206F6620256400426164207265636F72AA
:10E690006420666F756E6420647572696E672069A8
:10E6A0006E697469616C697A6174696F6E00256462
:10E6B0002025642025642028256420776F726473E8
:10E6C00029002564207265636F7264732C202564B1
:10E6D00020776F7264732C206D6178494420256423
:10E6E0002C20636F6D70616374696F6E2063796352
:10E6F0006C657320256400526573746F72656420C5
:10E70000256420736372697074730053746172744A
:10E71000656400726164696F00000000ACE700008E
:10E72000B9540000B9E7000055570000C9E70000E0
:10E73000D5560000D7E70000E9580000E2E70000E6
:10E74000E1540000F2E700006955000006E800000F
:10E750005155000015E80000CB5A000021E80000E8
:10E76000495A00002AE80000ED59000035E8000091
:10E770003559000040E800007159000049E80000E8
:10E78000A559000052E80000F154000061E80000C3
:10E79000D15400006AE80000015500006E6F6E65FC
:10E7A000006F7468657200706169720064697361FA
:10E7B000626C65526164696F006D65737361676552
:10E7C0005265636569766564007061636B65745258
:10E7D000656365697665007061636B657453656E2A
:10E7E00064007265636569766564496E7465676522
:10E7F000720072656365697665644D657373616700
:10E8000065547970650072656365697665645374F3
:10E8100072696E670073656E64496E7465676572D0
:10E820000073656E64506169720073656E64537441
:10E8300072696E67007365744368616E6E656C0023
:10E8400073657447726F757000736574506F776588
:10E8500072007369676E616C537472656E67746879
:10E86000006465766963654944006C6173744D6545
:10E870007373616765494400556E6B6E6F776E20E8
:10E880007072696D6974697665205B25733A2573CA
:10E890005D00000000000000963007772C610EEE4E
:10E8A000BA51099919C46D078FF46A7035A563E9E7
:10E8B000A395649E3288DB0EA4B8DC791EE9D5E00E
:10E8C00088D9D2972B4CB609BD7CB17E072DB8E70D
:10E8D000911DBF906410B71DF220B06A4871B9F362
:10E8E000DE41BE847DD4DA1AEBE4DD6D51B5D4F49B
:10E8F000C785D38356986C13C0A86B647AF962FD00
:10E90000ECC9658A4F5C0114D96C0663633D0FFA4C
:10E91000F50D088DC8206E3B5E10694CE44160D552
:10E92000727167A2D1E4033C47D4044BFD850DD23C
:10E930006BB50AA5FAA8B5356C98B242D6C9BBDB4F
:10E9400040F9BCACE36CD832755CDF45CF0DD6DC4A
:10E95000593DD1ABAC30D9263A00DE518051D7C8F1
:10E960001661D0BFB5F4B42123C4B3569995BACF7C
:10E970000FA5BDB89EB802280888055FB2D90CC69D
:10E9800024E90BB1877C6F2F114C6858AB1D61C116
:10E990003D2D66B69041DC760671DB01BC20D29835
:10E9A0002A10D5EF8985B1711FB5B606A5E4BF9FC2
:10E9B00033D4B8E8A2C9077834F9000F8EA80996B5
:10E9C00018980EE1BB0D6A7F2D3D6D08976C649120
:10E9D000015C63E6F4516B6B62616C1CD830658539
:10E9E0004E0062F2ED95066C7BA5011BC1F4088216
:10E9F00057C40FF5C6D9B06550E9B712EAB8BE8B57
:10EA00007C88B9FCDF1DDD62492DDA15F37CD38CDF
:10EA1000654CD4FB5861B24DCE51B53A7400BCA3DD
:10EA2000E230BBD441A5DF4AD795D83D6DC4D1A40F
:10EA3000FBF4D6D36AE96943FCD96E34468867ADE6
:10EA4000D0B860DA732D0444E51D03335F4C0AAA85
:10EA5000C97C0DDD3C710550AA41022710100BBE88
:10EA600086200CC925B56857B3856F2009D466B9CF
:10EA70009FE461CE0EF9DE5E98C9D9292298D0B004
:10EA8000B4A8D7C7173DB359810DB42E3B5CBDB7B1
:10EA9000AD6CBAC02083B8EDB6B3BF9A0CE2B60332
:10EAA0009AD2B1743947D5EAAF77D29D1526DB04E7
:10EAB0008316DC73120B63E3843B64943E6A6D0D32
:10EAC000A85A6A7A0BCF0EE49DFF099327AE000A7D
:10EAD000B19E077D44930FF0D2A3088768F2011E10
:10EAE000FEC206695D5762F7CB67658071366C19A7
:10EAF000E7066B6E761BD4FEE02BD3895A7ADA10C8
:10EB0000CC4ADD676FDFB9F9F9EFBE8E43BEB717A8
:10EB1000D58EB060E8A3D6D67E93D1A1C4C2D83832
:10EB200052F2DF4FF167BBD16757BCA6DD06B53F98
:10EB30004B36B248DA2B0DD84C1B0AAFF64A0336D7
:10EB4000607A0441C3EF60DF55DF67A8EF8E6E3156
:10EB500079BE69468CB361CB1A8366BCA0D26F259F
:10EB600036E2685295770CCC03470BBBB9160222EC
:10EB70002F260555BE3BBAC5280BBDB2925AB42B01
:10EB8000046AB35CA7FFD7C231CFD0B58B9ED92C16
:10EB90001DAEDE5BB0C2649B26F263EC9CA36A757B
:10EBA0000A936D02A906099C3F360EEB8567077232
:10EBB00013570005824ABF95147AB8E2AE2BB17B99
:10EBC000381BB60C9B8ED2920DBED5E5B7EFDC7C20
:10EBD00021DFDB0BD4D2D38642E2D4F1F8B3DD6877
:10EBE0006E83DA1FCD16BE815B26B9F6E177B06F72
:10EBF0007747B718E65A0888706A0FFFCA3B06665F
:10EC00005C0B0111FF9E658F69AE62F8D3FF6B61EB
:10EC100045CF6C1678E20AA0EED20DD75483044E8D
:10EC2000C2B30339612667A7F71660D04D4769491B
:10EC3000DB776E3E4A6AD1AEDC5AD6D9660BDF402E
:10EC4000F03BD83753AEBCA9C59EBBDE7FCFB247E1
:10EC5000E9FFB5301CF2BDBD8AC2BACA3093B353C6
:10EC6000A6A3B4240536D0BA9306D7CD2957DE54CF
:10EC7000BF67D9232E7A66B3B84A61C4021B685DA8
:10EC8000942B6F2A37BE0BB4A18E0CC31BDF055A21
:10EC90008DEF022D416C6C207461736B7320737463
:10ECA0006F70706564007631343200202573202542
:10ECB00073004D656D6F727920636C656172656478
:10ECC000004E6F2066726565207461736B20656EFF
:10ECD000747269657300000050ED0000F57100006A
:10ECE0005DED00006D6B000069ED0000C571000076
:10ECF0006FED0000D571000075ED0000E5710000BA
:10ED00007BED00009D70000091ED00006D73000030
:10ED10009FED0000A16B0000A9ED0000F973000059
:10ED2000B1ED0000C16E0000BAED0000656D00009D
:10ED3000C6ED00007D6C0000CFED0000C96C000046
:10ED4000D7ED0000156E000073656E736F7273006F
:10ED5000616363656C65726174696F6E0074656D83
:10ED600070657261747572650074696C74580074B2
:10ED7000696C74590074696C745A007365744163EA
:10ED800063656C65726F6D6574657252616E6765FF
:10ED9000006D61676E657469634669656C640074D3
:10EDA0006F756368526561640069326352656164BE
:10EDB00000693263577269746500737069457863DE
:10EDC00068616E6765007370695365747570007271
:10EDD000656164444854006D6963726F70686F6E5A
:10EDE00065000000F1DB0000D9740000F6DB0000D4
:10EDF000857400001BEE00001D76000020EE000070
:10EE0000A174000029EE0000A57500002FEE00009F
:10EE1000FD74000073657269616C00726561640065
:10EE200072656164496E746F00777269746500770A
:10EE3000726974654279746573000000B8EE000071
:10EE40004D760000C6EE00005D760000D3EE0000B7
:10EE500051760000DCEE000061760000E6EE000076
:10EE600065760000EFEE000069760000F4EE000029
:10EE70006D760000F9EE00007176000005EF0000ED
:10EE8000757600000CEF00007976000015EF0000A9
:10EE90007D7600001AEF00008176000025EF00006B
:10EEA000857600002FEF00005576000039EF000056
:10EEB0005976000074667400656E61626C65446921
:10EEC00073706C6179007365744261636B6C696720
:10EED000687400676574576964746800676574488E
:10EEE000656967687400736574506978656C006C57
:10EEF000696E65007265637400726F756E64656437
:10EF00005265637400636972636C65007472696151
:10EF10006E676C65007465787400746674546F7500
:10EF20006368656400746674546F75636858007430
:10EF30006674546F7563685900746674546F7563B2
:10EF40006850726573737572650076617273000044
:10EF500070EF0000157B00007AEF0000F57A0000EA
:10EF600083EF0000D17A00008FEF00005F7A00008D
:10EF7000766172457869737473007661724E616D63
:10EF80006564007365745661724E616D65640076E8
:10EF900061724E616D65466F72496E6465780057A7
:10EFA000656C636F6D6520746F204D6963726F428D
:10EFB0006C6F636B732100705F73706920213D205B
:10EFC0004E554C4C002F686F6D652F6769742F2E5E
:10EFD000706C6174666F726D696F2F7061636B61C5
:10EFE0006765732F6672616D65776F726B2D6172E5
:10EFF0006475696E6F6E6F726469636E7266352FC9
:10F000006C69627261726965732F5350492F535056
:10F01000492E63707000535049436C6173733A3AE0
:10F02000535049436C617373284E52465F535049A5
:10F030005F547970652A2C2075696E74385F742C62
:10F040002075696E74385F742C2075696E74385F32
:10F05000742900000000000000000000E97C0000AE
:10F06000A57C0000CB7C0000D57C0000DF7C00008C
:10F07000C97C000003000000020000000100000045
:10F080000400000005000000110000000C0000005A
:10F090000B000000120000000A0000000600000043
:10F0A0001A00000014000000170000001600000005
:10F0B0001500000010000000FFFFFFFFFFFFFFFF33
:10F0C000000000001E0000001900000018000000F1
:10F0D0000700000008000000090000000D0000000B
:10F0E0000E0000000F0000001C0000001B000000CC
:10F0F0001D000000130000000000000000000000E0
:10F10000D580000009890000558100006981000058
:10F110005F810000D1800000C58000007581000083
:10F12000F1800000C18000000000000000003043BA
:10F1300000000000000030C3737172740000000012
:10F14000FB21F93FFB2109407CD91240FB211940EA
:10F150007A6A1F407CD92240BBFD2540FB21294013
:10F160003A462C407A6A2F405C4731407CD9324085
:10F170009C6B3440BBFD3540DB8F3740FB21394071
:10F180001BB43A403A463C405AD83D407A6A3F4028
:10F190004C7E40405C4741406C1042407CD942402C
:10F1A0008CA243409C6B4440AC344540BBFD454081
:10F1B000CBC64640DB8F4740EB584840FB214940D7
:10F1C00083F9A200444E6E00FC291500D157270098
:10F1D000DD34F50062DBC0003C99950041904300AE
:10F1E0006351FE00BBDEAB00B761C5003A6E240080
:10F1F000D24D42004906E00009EA2E001C92D100DF
:10F20000EB1DFE0029B11C00E83EA700F535820089
:10F2100044BB2E009CE98400B4267000417E5F0050
:10F22000D6913900538339009CF439008B5F8400F8
:10F2300028F9BD00F81F3B00DEFF97000F9805007E
:10F24000112FEF000A5A8B006D1F6D00CF7E360024
:10F2500009CB2700464FB7009E663F002DEA5F00AE
:10F26000BA277500E5EBC7003D7BF100F7390700D1
:10F2700092528A00FB6BEA001FB15F00085D8D00AF
:10F28000300356007BFC4600F0AB6B0020BCCF0087
:10F2900036F49A00E3A91D005E619100081BE600A8
:10F2A00085996500A0145F008D40680080D8FF003C
:10F2B00027734D0006063100CA561500C9A8730011
:10F2C0007BE260006B8CC00000000040FB21F93F36
:10F2D000000000002D44743E000000809846F83C79
:10F2E0000000006051CC783B00000080831BF039A7
:10F2F0000000004020257A38000000802282E3369A
:10F30000000000001DF3693502000000030000004A
:10F31000040000000600000080A500002AA50000EF
:10F320002AA5000058A6000026A5000026A500007A
:10F330004EA6000058A6000026A500004EA600001C
:10F3400026A5000058A600005CA600005CA60000F0
:10F350005CA6000064A600005CB00000CEAE000019
:10F3600012AF000076AE000012AF000002B0000045
:10F3700012AF000076AE0000CEAE0000CEAE0000B0
:10F3800002B0000076AE00006EAE00006EAE00006F
:10F390006EAE000010B0000084B7000086B600001A
:10F3A00086B60000A4B9000080B6000080B6000058
:10F3B0008CB90000A4B9000080B600008CB9000030
:10F3C00080B60000A4B900009AB900009AB9000004
:10F3D0009AB90000A8B900002C2066756E637469A4
:10F3E0006F6E3A2000617373657274696F6E2022CC
:10F3F000257322206661696C65643A2066696C65D4
:10F4000020222573222C206C696E652025642573CB
:10F4100025730A0090000020232D302B2000686CFB
:10F420004C00656667454647003031323334353627
:10F430003738394142434445460030313233343560
:10F440003637383961626364656600000000000089
:10F4500000000000000000000000000000000000AC
:10F46000000000000000000000000000000000009C
:10F47000000000000000000000000000000000008C
:10F48000000000000000000000000000000000007C
:10F49000000000000000000000000000000000006C
:10F4A000000000000000000000000000504F534921
:10F4B0005800002020202020202020202828282834
:10F4C0002820202020202020202020202020202034
:10F4D0002020208810101010101010101010101084
:10F4E0001010100404040404040404040410101094
:10F4F0001010101041414141414101010101010140
:10F5000001010101010101010101010101011010CD
:10F510001010101042424242424202020202020213
:10F52000020202020202020202020202020210109F
:10F53000101020000000000000000000000000008B
:10F5400000000000000000000000000000000000BB
:10F5500000000000000000000000000000000000AB
:10F56000000000000000000000000000000000009B
:10F57000000000000000000000000000000000008B
:10F58000000000000000000000000000000000007B
:10F59000000000000000000000000000000000006B
:10F5A000000000000000000000000000000000005B
:08F5B000000000000000000053
:08F5B800500BFF7F0100000071
:10F5C000FFFFFFFFE803000001000000E803DC0587
:10F5D000DC05DC05DC050000FFFFFFFFFFFFFFFF90
:10F5E0001800000019FCFFFFFFFFFFFF02000000F2
:10F5F00040420F00FFFF01FF0024F4000200000062
:10F6000003000000FFFFFFFF0000000001000000FA
:10F610000000020001000000FFFFFFFF00000000EB
:10F62000020000000000040002000000FFFFFFFFD6
:10F6300000000000030000000000080003000000BC
:10F640000A000000080000000100000090000020F7
:10F65000000000006CF400008CF400004CF400008A
:10F66000000000000000000000000000000000009A
:10F67000000000000000000000000000000000008A
:10F68000000000000000000000000000000000007A
:10F69000000000000000000000000000000000006A
:10F6A000000000000000000000000000000000005A
:10F6B0004300000000000000000000000000000007
:10F6C000000000000000000000000000000000003A
:10F6D00043000000000000000000000000000000E7
:10F6E000000000000000000000000000000000001A
:10F6F00043000000000000000000000000000000C7
:10F7000000000000000000000000000000000000F9
:10F7100043000000000000000000000000000000A6
:10F7200000000000000000000000000000000000D9
:10F730004300000000000000000000000000000086
:10F7400000000000000000000000000000000000B9
:10F750004300000000000000000000000000000066
:10F760000000000000000000000000000000000099
:10F770004300000000000000000000000000000046
:10F780000000000000000000000000000000000079
:10F79000B1D80000C9D2000000000000B2F400009F
:10F7A0000CDB00001AE000001AE000001AE0000084
:10F7B0001AE000001AE000001AE000001AE0000061
:10F7C0001AE000001AE00000FFFFFFFFFFFFFFFF4D
:10F7D000FFFFFFFFFFFF00000100415343494900C5
:10F7E0000000000000000000000000000000000019
:10F7F00000000000000000000000415343494900A0
:10F8000000000000000000000000000000000000F8
:10F81000000000000000000000000000E9000000FF
:10F82000757C0000C97F000021840000C100000039
:040000030000806514
:00000001FF
